:1000000000400020F98C0000398D00003B8D00007D
:1000100000000000000000000000000000000000E0
:100020000000000000000000000000003D8D000006
:1000300000000000000000003F8D0000418D000026
:10004000438D000061650000A5900000438D000015
:10005000438D000000000000438D0000438D000030
:100060007941000079940000438D0000438D000029
:10007000438D0000438D0000438D0000438D000040
:10008000438D000029910000438D0000438D000046
:10009000438D0000438D0000438D0000438D000020
:1000A000438D0000438D00000000000000000000B0
:1000B0000000000000000000000000000000000040
:1000C00010B5064C2378002B07D1054B002B02D02E
:1000D000044800E000BF0123237010BD740200201B
:1000E000000000009C130100044B10B5002B03D04E
:1000F0000349044800E000BF10BDC04600000000F6
:10010000780200209C130100164B002B00D1144BE9
:100110009D46402292029A1A924600218B460F4633
:100120001348144A121A0DF015FF0F4B002B00D084
:1001300098470E4B002B00D0984700200021040068
:100140000D000D48002802D00C4800E000BF0DF063
:10015000C1FE2000290008F0F7FF0DF095FEC04613
:100160000000080000400020000000000000000027
:1001700074020020B42F00200000000000000000E6
:1001800002000120104011D1042A0ED91368180969
:1001900080B2002809D001388000031D11180979A8
:1001A000002902D001309842F8D170470020FCE7C6
:1001B0000378002B03D05AB2002A01DB01307047CC
:1001C0003F229343C03B59424B41C01803789343AD
:1001D000802BF4D10130F9E710B500240378002B0F
:1001E00001D1200010BDFFF7E3FF0134F6E770B541
:1001F000002204000D00411C092004F0E5FA00284B
:1002000006D001236200134343600023A34200DBB6
:1002100070BD9A00A958821891600133F6E770B555
:10022000012803DC1C2001F0D7FA70BD01230D6802
:1002300011201D42F7D04868184206D1042804D97D
:100240000F2302681340042B01D00E20EBE704F0CB
:1002500019F96D100400002D03DDFFF7BDFFA84262
:1002600006DA1220DFE72000FFF7A2FF0400013DBD
:10027000012DF8D120787F2809DDDF280BDCF82359
:100280003F22DB00800118406378134018430123AC
:1002900040001843C9E7EF280BDCFC226378120109
:1002A0009B0113403F220007000C0343A07810403D
:1002B000ECE7F72812DCFC22637892021B03134060
:1002C000E0228004520310403F221843E378134099
:1002D000FC220343A07812018001E8E7012040429C
:1002E000D5E7F8B54D680F00EB0706D4042D04D907
:1002F0000F232E683340092B03D00B2001F06CFA3A
:10030000F8BD6B683609B6B25C10731EA3420FD8F5
:10031000032120000BF0DAFC6421642803DC0100D7
:10032000032800DA03212800891904F07FFA050068
:100330002B6800201B099BB2013B9C42E0D23A682B
:10034000A31C9B005A510123013464001C436C60C0
:10035000D6E7F0B585B0012803DC1C2001F03CFA9B
:1003600012E001274B683A000093022806D08B6800
:100370003B4203D05F10002F00DC17000125009BDB
:100380002B4203D00120404205B0F0BD009B042B5E
:10039000F8D91B680C680F261900314004292DD1AB
:1003A0002C4205D1042C03D923681E40042E01D011
:1003B0000E20D3E70098FFF7E3FEB842E2DB009897
:1003C00004F060F80600200004F05CF803780100F7
:1003D000002BD7D0781E30180EF072F9041ED1D041
:1003E0003378002B01D0A64202D36800012521E01A
:1003F0003000FFF7DDFE01350600F1E709293ED1A7
:10040000009B5B685B1001939F42BBDC2C422ED1AA
:10041000042C2CD923683340042B28D1200004F06D
:1004200031F8039602907E1C009AB300D0588442A3
:1004300002D178002843A7E728420ED104280CD91E
:100440000368039A1340042B07D104F01BF8010042
:1004500002980EF0FFF80028EBD0019B37009E4277
:10046000E1DD8FE71F00019B9F4200DD8AE77B1CD7
:1004700000999A008A58A242F4D17800B6E703297D
:1004800000D07FE71A0992B25B0F92000B40D31A9B
:1004900001939F4200DD75E72C4229D1042C27D916
:1004A00022681640032E19D1100980B2520F800025
:1004B0003240251D801A019B2E181B1A0193009BA8
:1004C000781E0433019A904200DD5BE72A00191878
:1004D000B2420FD316D10130400087E7042E07D176
:1004E000200003F0CFFF05002000FFF749FEE2E700
:1004F0000F2033E70C78A4461478A44502D10131CB
:100500000132E5E70130DDE7F0B50D0085B00128E7
:1005100004DC1C2001F060F905B0F0BD012708687B
:10052000384206D1042804D90F2102680A40042A5F
:1005300001D00E20EEE76A681740FAD1042AF8D9F4
:1005400013680B40042BF4D103F09CFF040068688F
:1005500003F098FF02900EF087F8039000280FD167
:100560002000FFF739FE0190019B0122591C092050
:1005700004F02AF9364E3060002815D10020CBE770
:10058000029920000EF09CF8001B434243412000DA
:100590000193019B5E1C0028E6D0039B0299C018C2
:1005A0000EF08EF80196F4E70122019B5B001343E5
:1005B0004360039B002B18D12000FFF7F9FD019B3E
:1005C0000500BB4201DC3068A6E7291B200004F0CF
:1005D00079F90028D2D0BB1C32689B0098502800C3
:1005E000FFF7E6FD01372C00E9E7019B012B02D163
:1005F0002B68836090E7029920000EF061F80125D6
:100600000700019B002F13D0AB42DCDB391B20001D
:1006100004F058F90028B1D032680135AB00985089
:10062000039B0299FC1820000EF04AF80700E8E747
:10063000AB42C8DB20000EF017F80100200004F0E8
:1006400041F900289AD001353368AD00E850BAE787
:10065000A40F002010B503F0F9FE43000120184359
:1006600010BD0000C30711D404280FD90F2302685E
:100670001340032B0AD119400133591AC0234907EB
:10068000DB051940024B1A40114301607047C04618
:10069000FFFFFF9F70B5002805DC1C2001F09CF8CF
:1006A0000500280070BD01220C68144201D10D2004
:1006B000F4E701281CD04B681342F8D05B101320DC
:1006C000FF2BEBD81A0619040A431A431B021343E3
:1006D0006410E243D2171440E11C89101A00032071
:1006E00004F072F8051EDCD02100FFF7BBFFD8E74D
:1006F0000023EDE7F7B507000E001C20012F06DDF3
:100700004C68012322001A40009203D10D2001F011
:1007100063F853E0022F02D08A681A42F6D0012310
:1007200035681D4200D0A9E0042D00D8A6E01C4188
:10073000002C00DC1C000F2029680840092828D163
:100740006B685B100093022F05D0B368009A5B10B2
:100750009A4200DD0093009B01221D1B0135EB43F3
:10076000DB171D40691C092004F02EF8071E09D074
:1007700001236D001D430300326808334560009972
:10078000A14201DA3800FEBD0134A100515802C374
:10079000F5E7042845D1280003F074FEFFF71CFD9F
:1007A0000190022F04D0B3685B10984200DD0193E2
:1007B000019BA34204DA002004F078F80700E1E787
:1007C000280003F05FFE0700009BA34221DB280006
:1007D000009703F057FE05003800FFF7E9FC019B86
:1007E00001340700A342F7DA009BC41A200004F08A
:1007F0005DF8071EC6D003F045FE0190306803F097
:1008000041FE2200009B591B411801980DF086FB08
:10081000B8E73800FFF7CCFC009B070001330093DA
:10082000D2E703282AD10B099BB2490F9B00014054
:10083000591A022F04D0B2685210914200DD110003
:10084000A14205DA00220320110003F0BDFFB5E745
:1008500003200E1B331DD9170140C918891000222F
:1008600003F0B2FF071E00D18CE7013631000334DC
:10087000FFF7F8FE381D29193200C7E7212046E7A7
:10088000F7B5002804DC1C2000F0A6FF040014E0EB
:100890000D6801272E003E4011D03D41FF2D01D9AA
:1008A0001320F1E700223900032003F08DFF041E1E
:1008B00003D03900FFF7D6FE25712000FEBD042DC0
:1008C000EED90F232A681340042B1BD12800FFF711
:1008D00057FCC31C07000320D9170140C918891011
:1008E000320003F071FF041EE7D03900FFF7BAFEB3
:1008F000280003F0C7FD231D01003A0018000DF089
:100900000DFBDAE7092B1FD103206B6832005B1067
:1009100001930333D9170140C918891003F054FF1C
:10092000041ECAD00199FFF79DFE019B9E42C4DAC6
:10093000B300EB189B683B4204D05B10FF2BAFD891
:10094000A21913710136F0E7032BA9D12C00B4E7EB
:1009500010B57F2902DC0170013010BD1A4B99429D
:100960000CDC40238A115B42134303703F230B408E
:1009700080214942194341700230EEE7134B9942FE
:1009800010DC20230A135B4213433F2480220370B0
:100990008B1152422340214013430A43437082701B
:1009A0000330DAE70A4B9942D7DCF0230370603B4F
:1009B0004370113B8A11FF3B1A4382703F22114062
:1009C0001943C1700430C8E7FF070000FFFF0000B3
:1009D000FF0F010010B50124044002D04410200094
:1009E00010BD042810D90F2302681340042B07D12F
:1009F00003F048FD21000A220DF0FEFE0400EEE7A0
:100A0000032B01D10430F5E70D2000F0E5FEE6E709
:100A1000F0B50E0085B0002803DC1C2000F0DCFEE1
:100A200017E00F6801243D00254006D1042F1ED990
:100A30000F233A681340042B0DD13800FFF7CAFF8B
:100A400002AC01002000FFF783FF011B200003F030
:100A500039FF040032E0092B09D17B685B10019358
:100A6000019B9C4205DD00F0BDFE002819D02A2024
:100A7000D4E70134A300F858FFF7ACFF01237F2827
:100A80000DDD154ADB18904209DD144A013390420E
:100A900005DD0021124AC30F82424B419B00ED1835
:100AA000DEE7280003F002FF041E07D0376803F0DA
:100AB000E9FC01250600019B9D4202DD200005B0F6
:100AC000F0BD0135AB00F858FFF784FF010030009E
:100AD000FFF73EFF0600EEE7FF070000FFFF000004
:100AE000FF0F0100F7B5030001900E001C20012B41
:100AF00011DD0868FFF76EFF07007068FFF76AFFF7
:100B0000019B05000124022B08D0B068FFF762FFAB
:100B1000041E03DC292000F05FFEFEBDAF421CDC9A
:100B2000E81B21000BF0D2F8451C691C00220920AB
:100B300003F04AFE0028F0D001226B00134343600B
:100B40009440002379009D42E7DD17009E000F438B
:100B50008619B76001330919F5E7781B21000BF0FE
:100B6000B5F86442451CE0E710B5040001200840D8
:100B700010D104290DD90F230A681340042B08D182
:100B8000080003F07FFC010020000DF063FD4342EC
:100B9000584110BD0020FCE7F7B50E00012803DC2A
:100BA0001C2000F019FEFEBD4D68EB0706D4042D95
:100BB00004D90F222B681A40092A01D00B20F0E734
:100BC0006A681B099BB25410A34200D85C1E01271F
:100BD00031680F404810002F35D12648FFF7C4FF79
:100BE00001230190002813D131682348FFF7BCFF8F
:100BF000002811D0002C0DD00122631C013C944030
:100C00009B005A5114436C6004E00137BA00AB50AA
:100C1000BC42FADA0020C6E701233068184223D12B
:100C2000042821D902680E331340042B1CD1FFF78E
:100C3000D1FE002807D131681048FFF795FF002842
:100C400012D01220ADE70028FBDD8442F9DB8300DF
:100C5000EB180433844209DC0123621C013C9C40F4
:100C6000920053511C43CEE711209AE75A68013095
:100C70001A60EEE7FFF5000003F6000008F600003A
:100C8000002310B50C000B70C30705D50D494210A9
:100C900020000DF0A3FC08E00B49002802D0042836
:100CA00004D10A4920000DF0B9FC10BD0428FCD97C
:100CB0000F2302681340042BF7D103F0E3FB044930
:100CC0000200E5E71F0401000AF6000010F600002C
:100CD00015F60000F0B593B0060002911C20012E1D
:100CE0001DDD029B01251B681C002C4000D0ADE0DF
:100CF000042B00D8E6E01A680F231A40092A4AD1CB
:100D00000394039A029992008A5817002F4005D144
:100D1000042A03D910681840092806D0222000F0C0
:100D20005BFD0190019813B0F0BD52685210A418F9
:100D3000039A013203929642E3D1611C012203F02F
:100D400043FD0190002802D100230193EAE7019BB3
:100D50006400190025435D600831029ABB00D05839
:100D600002684368120992B25B109A4200D8531E7F
:100D70000022934209DCDA43D21713409B00C918C2
:100D8000039B01379F42E8DBCCE794000519AD686F
:100D900001320D51EDE72700032A59D10193029A40
:100DA000BB00D3582B42B9D1042BB7D9186801998D
:100DB0000140032939D1020992B2430F92000B403E
:100DC000D31A1C190137BE42E9D10320E31CD917FD
:100DD0000140C9188910002203F0F6FC0190002898
:100DE000B2D000252100FFF73DFC019B1E1D029A99
:100DF000AB00D45801231C421FD1042C1DD90F2154
:100E000023681940032918D1180980B25B0F8000AC
:100E10000B40C01A0023834213DBC343DB17184087
:100E200001353618BD42E2DB7CE7042900D075E7C6
:100E30001800FFF7A5F92418C4E72000FFF7A0F970
:100E4000E8E7E2181279F2540133E4E700273C00A6
:100E50000F25029ABB00D3580122134234D1042B30
:100E600032D9186801002940042935D11800FFF74C
:100E700087F924180137BE42EBD1200003F016FD9C
:100E80000190002800D15FE7029FB600BB19041D46
:100E9000029301233D681D4229D1042D27D90F2635
:100EA0002B681E40042E37D12800FFF769F9060091
:100EB000280003F0E7FA0100200032000DF02EF8C0
:100EC000A41922E02700C3E7180005A9FFF7D8FE00
:100ED00005A80DF0C9FBCCE7032900D01EE70209E5
:100EE00092B2430F92000B40D31A1C19C2E705A916
:100EF0002800FFF7C5FE05A80DF0B6FB05A9050003
:100F0000020020000DF00AF86419029B0437BB426E
:100F1000BFD10023237005E7032EF6D11A0992B240
:100F20005B0F92001E40961B291DC5E7F0B50D0012
:100F300097B0002806DC1C2000F04EFC07003800AB
:100F400017B0F0BD0C68012123000B40009306D1BF
:100F5000042C04D922680F331A40092A01D00B202F
:100F6000EAE7626852100392002A03DC009803F05B
:100F70009DFCE3E7504A019201280BD068680842C3
:100F800008D1042806D902681340042B02D103F0CB
:100F900079FA019001980DF067FB06000F27039B7B
:100FA0000834013B05935E43039B02909B00E318CA
:100FB000049301232068184273D1042871D9016871
:100FC0000B003B409C46042B03D1FFF7D9F8861950
:100FD00009E0032B6CD162460B099BB2490F9B00C1
:100FE00011405A1A9619049B0434A342E1D13000EF
:100FF00003F05CFC071EA2D02B680793029B002B1A
:1010000003D0686803F03EFA0190380003F03AFA22
:101010000400009B079A9B00D3189E68300003F0E1
:1010200031FA0123334005000693002B01D1042E31
:1010300004D809A93000FFF723FE09AD28000DF000
:1010400013FB069B0490002B0ED1042E0CD90F210C
:1010500033681940032907D11A0992B25B0F920035
:101060000B40D31A351D04932000049A29000CF07C
:1010700055FF049BE418029B002B0AD0059B009AA5
:10108000934206DD2000029A01990CF047FF029B73
:10109000E418009B01330093009A039B9342B8D15C
:1010A0004DE709A9FFF7ECFD09A80DF0DDFA8EE781
:1010B00003F0E8F9F9E7C046F7FB000010B501229C
:1010C000002400280BDD0B681A40141E03D05C10AE
:1010D000E343DB171C400122904200D04A68611CA8
:1010E000092003F071FB002803D0012364001C4396
:1010F000446010BD0A6870B510000125284034D145
:10110000042A32D90F24136849681C40092C17D1CE
:1011100054681B099BB22C41A34200D85C1E844238
:1011200005DC02200133984206DB00200FE0850039
:101130005519A9600130F2E7840011510130F2E73E
:10114000032C12D1294203D1132000F045FB70BDBE
:101150004910FF29F8D81B099BB204329B00D31811
:101160009342E2D911700132FAE70B2000F034FB10
:10117000DBE700000123F7B500254E680C00334083
:101180000193AB420ED11D00042E0BD90F22336800
:101190001A40092A26D172681B099BB25510AB422E
:1011A00000D85D1E27687C10FB0746D439003D48F7
:1011B000FFF7DAFC002826D00DF0ACF929000AF080
:1011C0006BFE4C1C019B002B00D069E0042E67D9FC
:1011D00032680F331340092B3BD10134A400A459CA
:1011E0002000FEBD042A04D13000FEF7C9FF05002F
:1011F000D8E7019D032AD5D11D09ADB25B0FAD0023
:101200001340ED1ACEE739002748FFF7ADFC002860
:101210001DD1042F16D90F233A681340042B11D186
:101220003800FFF7D7FB041E07D139001F48FFF72E
:101230009BFC002806D0122005E0002CFBDDA54217
:10124000C0DAF8E7112000F0C7FA0400C8E72C0064
:10125000B8E7042B1CD1300003F014F90500012C71
:101260000EDCFEF7A5FF461B300003F01FFB041E3B
:10127000B6D003F007F9320029000CF04FFEAFE7BB
:101280002B78013C002BD6D02800FEF791FFE5E734
:10129000032B05D13419E37801245B001C439FE73D
:1012A0000B20D0E7F8F5000003F6000008F6000078
:1012B000F7B54D680E002A0001210A402FD1042DF8
:1012C0002DD90F242B68B7681C40092C14D16968EC
:1012D0001B099BB24C100192A34200D85C1E3168DE
:1012E0003448FFF741FC00282DD00F232A68134013
:1012F000092B1DD1012317E0032C10D10F4203D17C
:10130000132000F069FAFEBD7A100192FF2AF7D887
:101310001A0992B25B0F92001C40141BDFE70B20EE
:10132000EFE701339A00AF509C42FADA0020EAE777
:10133000032BFBD12B0001335A1BA242F6DC6A4679
:101340001279DA70F7E736687010F30719D43100B4
:101350001948FFF709FC002822D1042E1ED90F23BB
:1013600032681340042B19D13000FFF733FB0028FB
:1013700007D131001148FFF7F7FB00280ED01220EB
:10138000BFE70028FBDD8442F9DB0F232A68134006
:10139000092B07D1013080004751C7E71120B0E782
:1013A0002000F2E7032BC1D16B461B792D18EB709F
:1013B000BCE7C046FFF5000003F6000008F6000099
:1013C00070B501240868204207D1042805D90F25EB
:1013D00001680D40092D02D14468200070BD032D25
:1013E00008D10A0992B24B0F92002B40D31A5B002E
:1013F0001C43F2E7042DF0D103F044F8FEF7ECFEB5
:1014000040000443E9E7000010B5034A0E210348F9
:1014100005F098F910BDC04688F5000080F5000081
:1014200000207047042070470120704710B500204D
:1014300003F03CFA10BD00207047002070470020E8
:101440007047002070470020704700207047002040
:1014500070470020704700207047000010B5034A15
:101460000D21034805F06EF910BDC046A0F600003E
:1014700008F70000704700207047002070470020E8
:101480007047002070470020704700207047002000
:10149000704700207047000010B5034A0821034838
:1014A00005F050F910BDC04680F70000C0F70000FD
:1014B0000378002B03D05AB2002A01DB01307047B9
:1014C0003F229343C03B59424B41C018037893439A
:1014D000802BF4D10130F9E7F8B50127060014009C
:1014E0000800394227D104293FD90F230A681A403E
:1014F000042A3AD13C4213D1042C11D9226813405A
:10150000042B0DD102F0BEFF0500200002F0BAFF4F
:10151000010028000DF09EF800282EDB1FD127E0E7
:10152000E30722D502F0AEFF0A2200210DF064F994
:101530000500601010E0174015D1042A15D90F23BB
:1015400012681340042B10D120004D1002F09AFFB6
:101550000A2239000DF050F985420EDB08DD002E1D
:1015600009DC00200CE04D10E3E70F22054B1A7058
:101570000136022EF5D8042002E004207617304010
:10158000F8BDC046B4020020F8B5060000252C4B7B
:10159000EC00E4182379032B09D00135FF2DF6D197
:1015A000300005F0E3F8002848D1013846E030006B
:1015B0000DF05AF8EBB202003100180005F05AF9AC
:1015C000002839D1226851688842E6D08300D318B8
:1015D0009B680130F02BF7D10123800008301218EE
:1015E0001A42DAD1042AD8D90F21136819400429E4
:1015F000D3D11B0998B20123013080001018184282
:10160000CBD10428C9D90F2203681340042BC4D1BD
:1016100002F038FF03270400092120000DF00CF828
:101620000028BAD0013F441C002FF5D13100200022
:101630000DF046F88442B0D102482843F8BDC046B8
:101640006425002000FFFFFF10B50124044002D0F4
:101650004410200010BD042810D90F230268134045
:10166000042B07D102F00EFF21000A220DF0C4F86E
:101670000400EEE7032B01D10430F5E70D22014B06
:101680001A70E6E7B4020020012210B5024018D11A
:10169000042802D903681A0992B201230B4012D11F
:1016A000042902D90B681B099BB20024934206D17E
:1016B00004309B000431C318984206D30124200053
:1016C00010BD0022E9E70023EFE704780A78002C38
:1016D00001D1002AF2D0013001319442ECD0002433
:1016E000EDE70000F7B50700009101933049314B59
:1016F000002A02D002220A70013A00261A601B68F2
:10170000CE54BE4200DBF7BD009AB300D058294B3F
:10171000274D1C68C8239B0065191C1B0123184218
:1017200006D0254A4310210028000CF025FF09E0CF
:10173000224A002802D004281BD1214A2100280077
:101740000CF01AFF1A4C20000CF08EFF194A019B76
:101750001060002B0BD07B1EB34208DD194B984262
:1017600005D8431C1360202222540022E254013683
:10177000C7E7042819D90F2301680B40042B04D1B3
:1017800002F080FE104A0300CDE7092B03D1436825
:101790000E4A5B10C7E7032B08D10A0992B2490F22
:1017A00092000B40D31A0A4ABDE70123094ABAE75F
:1017B000B5020020D80500201F0401000AF6000031
:1017C00010F600001F0300004B0A01001CFA000085
:1017D0002BFA000036FA0000014B18700020704709
:1017E000B4020020024B1878431E98417047C0464F
:1017F000B4020020002310B51A00FFF773FF034B5B
:101800000348196805F04EFD002010BDD8050020E2
:10181000B502002070B502F0C1FB094C0100251D86
:101820001F2228000CF038FF28000CF01DFF0423B5
:1018300004308008000118432060200070BDC046BD
:1018400090020020C368F0B59F00836889B0DF195B
:10185000030018330193036901999A00019B0090DA
:101860009C18436902939B00CB180393CA4B1B78C7
:10187000002B51D192103B6802617F221D12C74993
:1018800013409B005B58043702929F46009B9B6865
:101890000293FA1A009B92109B7812021A43009B43
:1018A000587805F0EBF90023009A2B701370009B19
:1018B000009A9B680293FB1A9B10D360019BE41A69
:1018C000A4101461039B019A9B1A009A9B10536108
:1018D00009B0F0BD009B587805F0C8F90023009AC4
:1018E0001370E4E7AC4B1B78002B15D1019A0099DB
:1018F000A21A92103B680A61029A1D121340A74A6D
:101900009B009B580437C0E7019B221DD11AA24BB4
:10191000D82918DD1A221A709F4D2978FF29B5D1D0
:1019200000232B709E4D2B68002BC0DD0123009AF5
:10193000137002F01BFBFA232A689B00534318180C
:10194000009B5860B3E71B782560002B01D0140082
:10195000E2E7009889103B68016102991D120B4073
:101960008E499B005B58140004378EE7019B221DB3
:10197000D11A894BD82902DD1A221A70CCE73D68AA
:101980001B78381D2560002B02D014000700C3E728
:10199000009889107B68016102991D120B407F49F4
:1019A0009B005B58140008376FE7019B221DD11A7A
:1019B000794BD82902DD1A221A70ADE7AD001B78E9
:1019C0007D192560002B01D01400A5E7009889102F
:1019D0003B68016102991D120B4070499B005B58E6
:1019E0001400043751E7019B221DD11AD82903DDC9
:1019F0001A22694B1A708FE76A4BAD00EB582360CF
:101A0000654B1B78002B01D0140085E700988910E6
:101A10003B68016102991D120B4060499B005B58B5
:101A20001400043731E7043C5E4B2268AD00EA50F5
:101A3000594B1B78002B00D06EE7019A0099A21A2F
:101A400092103B680A61029A1D121340534A9B0090
:101A50009B58043719E7534BAE00F058FFF7F4FDDD
:101A60004D4B05001B78002B09D1043C2068FFF783
:101A7000EBFD451901206D004A4B0543F550464BDF
:101A80001B78002B00D047E7019A0099A21A921008
:101A90003B680A61029A1D121340404A9B009B5802
:101AA0000437F2E6019B221DD11A3B4BD82902DDF7
:101AB0001A221A7030E70198039D0121A84202D230
:101AC00029000C3909681B782160002B01D0140013
:101AD00022E701990098511A89103B680161029927
:101AE0001D120B402D499B005B5814000437CCE6B7
:101AF000019A231D9A1A2849D82A02DD1A230B704D
:101B00000AE70198039EB0421BD231000C390968E4
:101B1000254849102D186D1AAD00A95921601C00E7
:101B20001D4B1B78002B00D0F6E6009992103B6805
:101B30000A61029A1D121340184A9B009B580437F1
:101B4000A3E6182008700021E8E7019B039A93425E
:101B50001ED213000C3B1B68134A5B10AD18043CEB
:101B6000ED1A2268039BAD00EA500B4B1B78002B4B
:101B700000D0D1E6019A0099A21A92103B680A613E
:101B8000029A1D121340054A9B009B5804377CE6BD
:101B90001822014B1A70E8E7B40200201CF800007C
:101BA000E00500205C2D0020FDFFFF3F019B039A14
:101BB00093422DD2D34B043CEE1815000C3D2B68FC
:101BC0005B10F31A9B009858FFF73EFD04902068C5
:101BD000FFF73AFD2D68049B6D10751B1E18012040
:101BE0007600039BAD000643EE50C74B1B78002BDD
:101BF00000D091E6019A0099A21A92103B680A61FE
:101C0000029A1D121340C14A9B009B5804373CE6C0
:101C10001822BD4B1A70E8E7019B221DD11ABA4B5E
:101C2000D82902DD1A221A7076E60398AD002858EA
:101C30001B782060002B01D014006DE600988910FD
:101C40003B68016102991D120B40B0499B005B5833
:101C50001400043719E6043C039B2268AD00EA50E7
:101C6000A94B1B78002B00D056E6019A0099A21AC6
:101C700092103B680A61029A1D121340A34A9B000E
:101C80009B58043701E6039BAD005D192B68043CAB
:101C900020685E10FFF7D8FC361801209A4B7600BA
:101CA0001B7806432E60002B00D035E6019A009980
:101CB000A21A92103B680A61029A1D121340934ABD
:101CC0009B009B580437E0E5AD00019B641BE61ABE
:101CD0008D4DA3420FD82B78002B00D01CE6009A24
:101CE000B6103B681661029A1D121340874A9B008A
:101CF0009B580437C9E5864802F0B4FB2B78002BCB
:101D000000D009E6009AB6103B681661029A1D12CF
:101D100013407E4A9B009B580437B6E5AB00FF1882
:101D2000002D00DAC3E5784B1B78002B00D0F3E5DB
:101D3000019A0099A21A92103B680A61029A1D1238
:101D40001340724A9B009B5804379EE5043C23686D
:101D5000042B04D1AB00FF18002D00DAA7E56A4B75
:101D60001B78002B00D0D7E5019A0099A21A921097
:101D70003B680A61029A1D121340644A9B009B58FB
:101D8000043782E5043C2368042B04D0AB00FF1821
:101D9000002D00DA8BE55C4B1B78002B00D0BBE5F7
:101DA000019A0099A21A92103B680A61029A1D12C8
:101DB0001340564A9B009B58043766E5261F30683F
:101DC000C3070AD540100138002809DB0123400071
:101DD000AD0018437F19306069E5FFF735FCF2E785
:101DE000494B1B78002B01D0340095E5019A0099EE
:101DF000B21A92103B680A61029A1D121340434ABC
:101E00009B009B58340004373FE52600019A039B52
:101E10000C369B1A9B100793B21AD82A02DD1A239C
:101E20000B7079E520006C00FF2501236D00254033
:101E30001D43009C0560A468009D03943C1BAD7885
:101E4000A41024022C43079D9C409D401C432B431F
:101E5000836044606846009B007E09789870634602
:101E600004983400C358009892108360002903D06E
:101E700008331F0003964FE51F0000999B680A6115
:101E8000029A1D121340214A9B000C379B5803965F
:101E9000FBE4231F1D68039A019B93423AD10A2059
:101EA000EB0711D4042D18D90F232A681340042BF3
:101EB00016D1280002F0E6FA0CF0D6FBC8239B00EE
:101EC000984200D918000630643004F007FD00285D
:101ED0000FD1043F019B0393E9E40720042DF3D0C5
:101EE0002800431E9841FA234042FF331840073030
:101EF000EAE7009B2900587804F0D2FE0023009AFC
:101F00001370E7E7FDFFFF3FB40200201CF800005C
:101F100048FA0000039B039A0C3B1B6800995B1076
:101F20009B00D31A0C3B1D601C1D1300083B1B6853
:101F30005A108A70FF210A40CE49D2005B005758E0
:101F40009B0A009A9B009760FF18039B019A043B31
:101F50001B685B109B00D3180393C74BA21A1B7816
:101F60009210002B00D0D7E400993B680A61029AD6
:101F70001D121340C14A9B009B58043785E4231F60
:101F80001868FFF761FBAD000600641B1E2831DCFA
:101F9000002812DCB84B1B78002B00D0BCE4019A5F
:101FA0000099A21A92103B680A61029A1D1213400E
:101FB000B24A9B009B58043767E401F0D7FF033E09
:101FC000361801F0D3FFAE4B801B9842F9D8AA4BCC
:101FD0001B78002B00D09FE4019A0099A21A92105E
:101FE0003B680A61029A1D121340A44A9B009B5849
:101FF00004374AE40123009A137001F0B7FF009BF5
:102000000A3886195E6052E4231F1868FFF71CFB2C
:10201000AD000600641B002812DC974B1B78002BD8
:1020200000D079E4019A0099A21A92103B680A61E3
:10203000029A1D121340914A9B009B58043724E4D6
:10204000904B984203DD1D228B4B1A7064E40123F0
:10205000009A137001F08AFFFA239B005E430A3E48
:1020600030186DE4AB00E41A002328001A002100A8
:10207000FFF738FB844E854D3168280002F022FCC2
:10208000834B31681860280004F0D6FF31682800BF
:1020900005F008F9784B1B78002B00D03CE4019A3E
:1020A0000099A21A92103B680A61029A1D1213400D
:1020B000724A9B009B580437FFF7E7FB6E4BAD005D
:1020C0001B78641B002B00D026E4019A0099A21A09
:1020D00092103B680A61029A1D121340674A9B00E6
:1020E0009B580437FFF7D1FB009804F05BFC624B70
:1020F0001B78002B00D00FE4019A0099A21A9210CD
:102100003B680A61029A1D1213405C4A9B009B586F
:102110000437FFF7BAFB231F1E68002E47D1083B88
:102120001868013606401FD04610220001237100B6
:10213000083A0B431360002E00DC99E00123720083
:102140001A43211F0A602200083A12681A41921BA2
:10215000049222000C3A106818422BD0049AAD0069
:10216000D2189A40134331E004281BD90F22036888
:102170001A40092A02D146687610D6E7042A08D107
:1021800002F080F90378002BCFD0FFF791F90136E8
:10219000F8E7032A06D1180980B25E0F80001640C6
:1021A000861BC2E71922344B1A70FFF7B5FB761075
:1021B000013EC0E7042856D90F2201680A40092AC7
:1021C0001BD1049BAD0002339B001B58039AAB50FC
:1021D000294B1B78002B01D0FFF79EFB019A009939
:1021E000A21A92103B680A61029A1D121340234AF8
:1021F0009B009B580437FFF748FB042A2BD1039B15
:10220000AD005B19069302F03DF90600049D01350F
:10221000012D10DC3000FFF74BF9831B18000493ED
:1022200002F044FB051E0ED002F02CF9049A310096
:102230000BF074FE07E03178013D002906D112222F
:102240000D000D4B1A70069B1D60C1E73000FFF7B3
:102250002FF90600DCE7032A05D1049AAD008218A5
:10226000127952007EE71922034B1A70FFF754FBD4
:102270000437ADE764250020B40200201CF80000FC
:102280007F96980080EE3600D8050020B502002029
:1022900008000020AB00019AE3189B1AD82B18DC29
:1022A00001226B1E002D19DCCF4B1B78002B01D0B7
:1022B000FFF732FB019A0099A21A92103B680A615B
:1022C000029A1D121340C94A9B009B580437FFF71E
:1022D000DCFA1A22C44B1A70FFF71EFB22601D00A5
:1022E0000434DEE7019A231D9B1ABF4ED82B03DD71
:1022F0001A233370FFF710FB019B039AAD00934242
:102300002FD2231F1868FFF79FF9011E26DD039BBC
:102310000C3B1A685210824220DB9007801AB44BA3
:102320004018C018039B8000C258631B1A60AE4B54
:10233000641B1B780434002B01D0FFF7EDFA019ADF
:102340000099A21A92103B680A61029A1D1213406A
:10235000A64A9B009B580437FFF797FA2023337057
:10236000E5E71823FBE7A34BAD001A68631B1C00CD
:102370001A609D4B04341B78002B01D0FFF7CCFA78
:10238000019A0099A21A92103B680A61029A1D12E2
:102390001340964A9B009B580437FFF776FA221F9A
:1023A0001368042B02D12200AD007F198E4B1B78DD
:1023B000002B02D01400FFF7AFFA01990098511AD0
:1023C00089103B68016102991D120B4087499B00EF
:1023D0005B5814000437FFF758FA043C2368042BB9
:1023E00004D00023AD0023607F1904347E4B1B789A
:1023F000002B01D0FFF790FA019A0099A21A9210CF
:102400003B680A61029A1D121340784A9B009B5850
:102410000437FFF73AFAAB009C46E61A002D1CDCA5
:102420001C22714B1A70002333606346E41A6E4B12
:1024300004341B78002B01D0FFF76EFA019A009943
:10244000A21A92103B680A61029A1D121340674A51
:102450009B009B580437FFF718FA002033685A1086
:102460008300F15801230B4003D10D215E4A117006
:10247000DAE749108A4200DD0A0001308542EFDCCC
:10248000012352001343CFE7AB009C46E61A002D10
:102490001CDC1C22544B1A70002333606346E41A80
:1024A000514B04341B78002B01D0FFF735FA019A09
:1024B0000099A21A92103B680A61029A1D121340F9
:1024C0004A4A9B009B580437FFF7DFF90020336826
:1024D0005A108300F15801230B4003D10D21424AC9
:1024E0001170DAE749108A4200DA0A0001308542A9
:1024F000EFDC012352001343CFE723000122083B06
:102500001968AE00114222D0231F1B6813421ED04F
:10251000114113410022994200DA0432A31B1A60D0
:10252000314BA41B1B780434002B01D0FFF7F4F9C6
:10253000019A0099A21A92103B680A61029A1D1230
:1025400013402A4A9B009B580437FFF79EF902204C
:10255000231F1A684042FEF7BFFFA51B2860DFE774
:102560002300083B19680123AE00194223D0221F23
:1025700012681A421FD019415010CB0FD21788424F
:102580005341A21B9B001360174BA41B1B78043400
:10259000002B01D0FFF7C0F9019A0099A21A9210FE
:1025A0003B680A61029A1D121340104A9B009B5817
:1025B0000437FFF76AF90120231F1A684042FEF72B
:1025C0008BFFA51B2860DFE72300083B1868231F4B
:1025D0001968AE00A61B0423814202D004280BD840
:1025E000002333601FE0C046B40200201CF8000046
:1025F000FCFFFF3F0800002001231842F0D10F2309
:1026000002681A40042AEBD1033A1142E8D10429A6
:10261000E6D90A681340042BE2D1FFF735F8431ED0
:10262000984180003060EA4BAD001B78641B043495
:10263000002B01D0FFF770F9019A0099A21A9210AD
:102640003B680A61029A1D121340E24A9B009B58A4
:102650000437FFF71AF92300083B1868231F19688D
:10266000AE00A61B0023814202D0042802D8042316
:10267000336016E001231842F9D10F2302681A4093
:10268000042AF4D1033A1142F1D10429EFD90A689E
:102690001340042BEBD1FEF7F7FF43425841800073
:1026A0003060CB4BAD001B78641B0434002B01D091
:1026B000FFF732F9019A0099A21A92103B680A6159
:1026C000029A1D121340C34A9B009B580437FFF720
:1026D000DCF823000122083B1968AE00114223D028
:1026E000231F1B6813421FD05B104A10D80FC91755
:1026F0009A424141A31B89001960B54BA41B1B786A
:102700000434002B01D0FFF707F9019A0099A21AAF
:1027100092103B680A61029A1D121340AD4A9B0059
:102720009B580437FFF7B1F8231F1A680120FEF702
:10273000D3FEA51B2860E0E723000122083B1968AF
:10274000AE00114222D0231F1B6813421ED011413C
:1027500013410022994200DD0432A31B1A609C4BF6
:10276000A41B1B780434002B01D0FFF7D5F8019A85
:102770000099A21A92103B680A61029A1D12134036
:10278000944A9B009B580437FFF77FF8231F1A6871
:102790000220FEF7A1FEA51B2860E0E7231F1B68AF
:1027A000AD00043B5A1E9341621B14009B00136052
:1027B000874B04341B78002B01D0FFF7ADF8019A4A
:1027C0000099A21A92103B680A61029A1D121340E6
:1027D000804A9B009B580437FFF757F82300083BBB
:1027E0001868FEF731FF231F06001868FEF72CFF5C
:1027F00036180120AD00631B1C00760006431E60E6
:10280000734B04341B78002B01D0FFF785F8019A35
:102810000099A21A92103B680A61029A1D12134095
:102820006C4A9B009B580437FFF72FF82300083BA6
:102830001868FEF709FF231F06001868FEF704FF5B
:10284000361A0120AD00631B1C00760006431E6093
:102850005F4B04341B78002B01D0FFF75DF8019A21
:102860000099A21A92103B680A61029A1D12134045
:10287000584A9B009B580437FFF707F82300083B92
:102880001868FEF7E1FE231F06001868FEF7DCFE5D
:1028900046430120AD00631B1C00760006431E600A
:1028A0004B4B04341B78002B01D0FFF735F8019A0D
:1028B0000099A21A92103B680A61029A1D121340F5
:1028C000444A9B009B580437FEF7DFFF231F18681C
:1028D000FEF7BAFE061E1CD11F233D4A1370AD0041
:1028E000631B1C001E603A4B04341B78002B01D084
:1028F000FFF712F8019A0099A21A92103B680A6138
:10290000029A1D121340334A9B009B580437FEF76E
:10291000BCFF2300083B1868FEF796FE310009F063
:10292000D5F9012640000643D9E7231F1868FEF7B2
:102930008BFE061E1CD11F23254A1370AD00631B9E
:102940001C001E60224B04341B78002B01D0FEF7C4
:10295000E3FF019A0099A21A92103B680A61029A59
:102960001D1213401B4A9B009B580437FEF78DFF36
:102970002300083B1868FEF767FE310009F08CFA67
:10298000012649000E43D9E7231F1868FEF75CFEB5
:10299000C217801850400122AD00631B1C0040008C
:1029A000104318600A4B04341B78002B01D0FEF74B
:1029B000B3FF019A0099A21A92103B680A61029A29
:1029C0001D121340034A9B009B580437FEF75DFF1E
:1029D000B40200201CF80000AB000793E31A069332
:1029E000012D32D11868FEF72FFEC617AE430490B2
:1029F0000136049B9E4201DC04961E00049B0136B6
:102A0000F61A0BF087FD310009F046FA049B069A8E
:102A1000CB1801215B000B431360079BE41AF04BBA
:102A200004341B78002B01D0FEF776FF019A009941
:102A3000A21A92103B680A61029A1D121340E94AD9
:102A40009B009B580437FEF720FF022D0AD1069BFE
:102A50001868FEF7F9FD069B06005868FEF7F4FDBE
:102A60000490C6E7012364260493C7E7AB00E61A87
:102A700031002800049302F07BF8049B3060E41AD4
:102A8000D74B04341B78002B01D0FEF745FF019A89
:102A90000099A21A92103B680A61029A1D12134013
:102AA000D04A9B009B580437FEF7EFFE2300083BFB
:102AB0001868FEF7C9FD231F06001868FEF7C4FD5D
:102AC00006400120AD00631B1C00760006431E601B
:102AD000C34B04341B78002B01D0FEF71DFF019A75
:102AE0000099A21A92103B680A61029A1D121340C3
:102AF000BC4A9B009B580437FEF7C7FE2300083BE7
:102B00001868FEF7A1FD231F06001868FEF79CFD5C
:102B100006430120AD00631B1C00760006431E60C7
:102B2000AF4B04341B78002B01D0FEF7F5FE019A61
:102B30000099A21A92103B680A61029A1D12134072
:102B4000A84A9B009B580437FEF79FFE2300083BD2
:102B50001868FEF779FD231F06001868FEF774FD5C
:102B600046400120AD00631B1C00760006431E603A
:102B70009B4B04341B78002B01D0FEF7CDFE019A4D
:102B80000099A21A92103B680A61029A1D12134022
:102B9000944A9B009B580437FEF777FE231F186862
:102BA000FEF752FDC0430122AD00631B1C00400034
:102BB000104318608A4B04341B78002B01D0FEF7B9
:102BC000ABFE019A0099A21A92103B680A61029A20
:102BD0001D121340834A9B009B580437FEF755FE95
:102BE0002300083B1868FEF72FFD231F0600186816
:102BF000FEF72AFD86400122AD00631B1C00760013
:102C000016431E60764B04341B78002B01D0FEF770
:102C100083FE019A0099A21A92103B680A61029AF7
:102C20001D1213406F4A9B009B580437FEF72DFE80
:102C30002300083B1868FEF707FD231F06001868ED
:102C4000FEF702FD06410122AD00631B1C00760069
:102C500016431E60624B04341B78002B01D0FEF734
:102C60005BFE019A0099A21A92103B680A61029ACF
:102C70001D1213405B4A9B009B580437FEF705FE6C
:102C800023000C3B1868FEF7DFFC2300083B06001E
:102C90001868FEF7D9FCF1170200C317300009F0DD
:102CA0004DF9231F049005911868FEF7CDFC020032
:102CB0000498059909F0F6F843000120AD00661B61
:102CC00034001843464B30601B780434002B01D08D
:102CD000FEF722FE019A0099A21A92103B680A613F
:102CE000029A1D1213403F4A9B009B580437FEF77F
:102CF000CCFDAB00E61A310028000493FEF7DEF9A4
:102D0000049B3060E41A364B04341B78002B01D04E
:102D1000FEF702FE019A0099A21A92103B680A611E
:102D2000029A1D1213402F4A9B009B580437FEF74E
:102D3000ACFDAB00E41A21002800FEF7DBF9284BBC
:102D40001B78002B01D0FEF7E7FD019A0099A21A2B
:102D500092103B680A61029A1D121340214A9B009F
:102D60009B580437FEF791FDAB00E61A31002800AE
:102D70000493FEF7FFF9049B3060E41A184B043407
:102D80001B78002B01D0FEF7C7FD019A0099A21A0B
:102D900092103B680A61029A1D121340114A9B006F
:102DA0009B580437FEF771FDAB00E41A21002800A0
:102DB000FEF77EFA0A4B1B78002B01D0FEF7ACFD24
:102DC000019A0099A21A92103B680A61029A1D1298
:102DD0001340044A9B009B580437FEF756FDC0463B
:102DE000B40200201CF80000AB00E61A31002800F5
:102DF0000493FEF7E5FA049B3060E41AE54B0434D3
:102E00001B78002B01D0FEF787FD019A0099A21ACA
:102E100092103B680A61029A1D121340DE4A9B0021
:102E20009B580437FEF731FD231F186801F02AFB79
:102E30002200083A12680300AD00D1072ED4042AFC
:102E40000CD910680F221040013808280FD808F05C
:102E50009FFE05252B270E0E0E0E2900CF491800C8
:102E60000BF0F8FB43425841631B80001860C94BCC
:102E7000641B1B780434002B01D0FEF74DFD019A32
:102E80000099A21A92103B680A61029A1D1213401F
:102E9000C14A9B009B580437FEF7F7FCC049DEE7A8
:102EA000C049DCE7C049DAE7C049D8E7019A231DE9
:102EB00004939E1AD82E04DD1A22B64B1A70FEF720
:102EC0002BFD01F05DF8430001201843B14B206059
:102ED0001B78002B02D0049CFEF71EFD009AB61052
:102EE0003B681661029A1D121340AB4A9B009B5827
:102EF000049C0437FEF7C9FC019B261DF31A0493BA
:102F0000D82B04DD1A22A34B1A70FEF705FD01F041
:102F10002DF8A74B40001840012318439D4B20601B
:102F20001B78002B02D03400FEF7F6FC049A0099BF
:102F300092103B680A61029A1D121340964A9B0048
:102F40009B5834000437FEF7A0FC019B261DF31AA2
:102F5000904DD82B03DD1A232B70FEF7DDFC01F01A
:102F60000FF8944B1A68831A904201D2924A9B1828
:102F700001205B00034323602B78002B02D0340038
:102F8000FEF7CAFC019A0099B21A92103B680A61D6
:102F9000029A1D121340804A9B009B58340004374C
:102FA000FEF773FC00F0ECFF824BAD001860794B2C
:102FB000641B1B78002B01D0FEF7AEFC019A009930
:102FC000A21A92103B680A61029A1D121340724ABB
:102FD0009B009B580437FEF758FC03F019FFAE0026
:102FE000002815D16B4BA41B1B78002B01D0FEF7DA
:102FF00093FC019A0099A21A92103B680A61029A06
:103000001D121340644A9B009B580437FEF73DFC99
:103010000123A61B28001A003100FEF763FB674D51
:103020002868643003F05AFC002802D1043FFEF700
:103030003EFC009B29685A78614803F038FE012362
:10304000009A3400137000F091FF5E4B2A681B68F1
:10305000063253431818009B5860FEF728FC03F013
:10306000D7FEAE00002815D14A4BA41B1B78002BBD
:1030700001D0FEF751FC019A0099A21A92103B6808
:103080000A61029A1D121340434A9B009B58043761
:10309000FEF7FBFBA61B2800012300223100FEF7F0
:1030A00021FB464D2868643003F018FC0028BDD091
:1030B000434803F0BFFDC2E7AD00661BFEF7AAFB65
:1030C0003400344B30601B780434002B01D0FEF701
:1030D00023FC019A0099A21A92103B680A61029A95
:1030E0001D1213402C4A9B009B580437FEF7CDFB62
:1030F000284BAD001B78641B002B01D0FEF70CFCA5
:10310000019A0099A21A92103B680A61029A1D1254
:103110001340214A9B009B580437FEF7B6FBAD00D5
:10312000661B300000F065FF34001A4B30601B78DE
:103130000434002B01D0FEF7EFFB019A0099A21A8C
:1031400092103B680A61029A1D121340124A9B00BA
:103150009B580437FEF799FBAD00661B300000F06A
:103160004AFF34000B4B30601B780434002B01D035
:10317000FEF7D2FB019A0099A21A92103B680A61ED
:10318000029A1D121340044A9B009B580437FEF715
:103190007CFBC046B40200201CF8000058FA000076
:1031A00060FA000067FA00006EFA000073FA00008F
:1031B000FEFFFF7FE405002037894100D80500208D
:1031C000B502002004000020AB00E61A3100280000
:1031D000049300F05BFD049B3060E41AF44B04346C
:1031E0001B78002B01D0FEF797FB019A0099A21AD9
:1031F00092103B680A61029A1D121340ED4A9B002F
:103200009B580437FEF741FBAD00641B200000F023
:10321000F5FEE74B1B78002B01D0FEF77DFB019AF2
:103220000099A21A92103B680A61029A1D1213407B
:10323000E04A9B009B580437FEF727FBAB00E61AD9
:1032400031002800049300F085FC049B3060E41AF0
:10325000D74B04341B78002B01D0FEF75DFB019A9D
:103260000099A21A92103B680A61029A1D1213403B
:10327000D04A9B009B580437FEF707FBAD00641B48
:10328000200000F015FFCA4B1B78002B01D0FEF781
:1032900043FB019A0099A21A92103B680A61029AB4
:1032A0001D121340C34A9B009B580437FEF7EDFAEA
:1032B0000121280000F0D6FEBD4B1B78002B01D069
:1032C000FEF72AFB019A0099A21A92103B680A6144
:1032D000029A1D121340B74A9B009B580437FEF711
:1032E000D4FA0021280000F0BDFEB14B1B78002B62
:1032F00001D0FEF711FB019A0099A21A92103B68C7
:103300000A61029A1D121340AA4A9B009B58043777
:10331000FEF7BBFAAD00661B300000F0F7FE34008C
:10332000A34B30601B780434002B01D0FEF7F4FA75
:10333000019A0099A21A92103B680A61029A1D1222
:1033400013409C4A9B009B580437FEF79EFAAD0041
:10335000661B300000F0EEFE3400954B30601B78A9
:103360000434002B01D0FEF7D7FA019A0099A21A73
:1033700092103B680A61029A1D1213408D4A9B000D
:103380009B580437FEF781FAAD00641B200000F063
:10339000A5FE874B1B78002B01D0FEF7BDFA019AE2
:1033A0000099A21A92103B680A61029A1D121340FA
:1033B000804A9B009B580437FEF767FAAD00641BF8
:1033C000200004F07BFB7A4B1B78002B01D0FEF72A
:1033D000A3FA019A0099A21A92103B680A61029A14
:1033E0001D121340734A9B009B580437FEF74DFA99
:1033F000AD00661B300004F057FC34006C4B3060AD
:103400001B780434002B01D0FEF786FA019A00994C
:10341000A21A92103B680A61029A1D121340654A73
:103420009B009B580437FEF730FAAD00641B200068
:1034300004F0BEFA5E4B1B78002B01D0FEF76CFA4D
:10344000019A0099A21A92103B680A61029A1D1211
:103450001340584A9B009B580437FEF716FAAD00FC
:10346000661B300004F0BEFA3400514B30601B780C
:103470000434002B01D0FEF74FFA019A0099A21AEA
:1034800092103B680A61029A1D121340494A9B0040
:103490009B580437FEF7F9F9AB00E41A2100280025
:1034A00002F010F8424B1B78002B01D0FEF734FAE3
:1034B000019A0099A21A92103B680A61029A1D12A1
:1034C00013403C4A9B009B580437FEF7DEF9AB00E3
:1034D000E41A2100280001F0FBFD354B1B78002B7E
:1034E00001D0FEF719FA019A0099A21A92103B68CE
:1034F0000A61029A1D1213402E4A9B009B58043702
:10350000FEF7C3F9AB00E41A2100280001F092FE97
:10351000274B1B78002B01D0FEF7FEF9019A00998A
:10352000A21A92103B680A61029A1D121340214AA6
:103530009B009B580437FEF7A8F9AB00E41A210062
:10354000280001F09FFE1A4B1B78002B01D0FEF7DC
:10355000E3F9019A0099A21A92103B680A61029A53
:103560001D121340134A9B009B580437FEF78DF938
:10357000AB00E61A31002800049304F005FC049B1C
:103580003060E41A0A4B04341B78002B01D0FEF79C
:10359000C3F9019A0099A21A92103B680A61029A33
:1035A0001D121340034A9B009B580437FEF76DF928
:1035B000B40200201CF80000AB00E61A310028001D
:1035C000049304F0E9FB049B3060E41AD44B043408
:1035D0001B78002B01D0FEF79FF9019A0099A21ADF
:1035E00092103B680A61029A1D121340CD4A9B005B
:1035F0009B580437FEF749F9AB00E61A3100280062
:10360000049304F0D1FB049B3060E41AC44B0434EF
:103610001B78002B01D0FEF77FF9019A0099A21ABE
:1036200092103B680A61029A1D121340BD4A9B002A
:103630009B580437FEF729F9AB00E61A3100280041
:10364000049304F0B9FB049B3060E41AB44B0434D7
:103650001B78002B01D0FEF75FF9019A0099A21A9E
:1036600092103B680A61029A1D121340AD4A9B00FA
:103670009B580437FEF709F9AB00E41A2100280033
:1036800001F0A0FEA64B1B78002B01D0FEF744F9F9
:10369000019A0099A21A92103B680A61029A1D12BF
:1036A0001340A04A9B009B580437FEF7EEF8AB008E
:1036B000E41A2100280001F00DFE994B1B78002B25
:1036C00001D0FEF729F9019A0099A21A92103B68DD
:1036D0000A61029A1D121340924A9B009B580437BC
:1036E000FEF7D3F8AB00E61A31002800049301F08E
:1036F0006DFD049B3060E41A894B04341B78002B69
:1037000001D0FEF709F9019A0099A21A92103B68BC
:103710000A61029A1D121340824A9B009B5804378B
:10372000FEF7B3F8AB00E41A2100280001F0FCFC1E
:103730007B4B1B78002B01D0FEF7EEF8019A009925
:10374000A21A92103B680A61029A1D121340754A30
:103750009B009B580437FEF798F8002D00DC8AE0A8
:10376000231F1E68012D0CD12E4207D1042E05D92E
:103770000F23326830001340042B10D001235B422A
:1037800012E0022DFAD12300083B1868C307F5D4D4
:103790000428F3D90F2302681340042BEED100F064
:1037A00071FEFDF7F1FE0300AA00A41A5A1C62D0B4
:1037B0000020022D12D101223240824235D1042E46
:1037C00033D90F213068014009292ED17168481082
:1037D000FF2108408100914222D16418019A00998A
:1037E000A21A92100A61FF251A004F49AA438A4281
:1037F00023D11D062D0C05432B120693FF232A12FD
:1038000013404A4ADB009446049363441B794449BD
:10381000032B01D1FEF7F9FA02230B70FEF77CF8B7
:10382000B518AD68A5500432D5E70B223C4B1A7091
:10383000002323600434FEF76FF88600A61B3100D6
:10384000984700223A4B341D1A60354B30601B7884
:10385000934201D0FEF760F8019A0099A21A9210E3
:103860003B680A61029A1D1213402E4A9B009B5826
:103870000437FEF70AF800232360294B221D1B782A
:10388000002B02D01400FEF747F801990098511A56
:1038900089103B68016102991D120B4021499B0070
:1038A0005B5814000437FDF7F0FFAB00E41A210069
:1038B000280003F0E9FA1A4B1B78002B01D0FEF721
:1038C0002BF8019A0099A21A92103B680A61029A99
:1038D0001D121340134A9B009B580437FDF7D5FF78
:1038E000AB00E61A31002800049303F0CDFA049BE4
:1038F0003060E41A0A4B04341B78002B01D0FEF729
:103900000BF8019A0099A21A92103B680A61029A78
:103910001D121340034A9B009B580437FDF7B5FF67
:10392000B40200201CF8000000FFFFFF6425002007
:10393000A40F00200023F7B55A1E0192002B07DACE
:1039400001F0D6FD03F0B8FB03F0C4FC192301938A
:1039500000263000194B1968B14212DD184B1A6865
:1039600001328A420FDAF0241A601D68154F6C4349
:10397000E35D002B1FD0E419022B06D12000FDF7D8
:1039800061FF019BD8E70022EDE7012B0DD1002854
:1039900001D100F0EBFAF0226A43BB185B680A49D8
:1039A000C31A8B4201D80223BB54F0235D43054B5D
:1039B000EB5C022BE2D00136CCE7C046DC050020F0
:1039C00000000020041C00207F96980080220B4BF2
:1039D00052001A600121A822A920094BD2001964C3
:1039E0009A58C00005321A5006481A50C122C02009
:1039F000920000039850044B1970704700E100E0FA
:103A0000008000404C05000025060020042070477F
:103A1000F8B550C9012322001A40101E2DD03340A2
:103A2000181E2AD0641000201A2C26D81D4B7610A0
:103A300035009E4200DD1D001B4F3B5D012B05D074
:103A40000121200005F064FD01233B55174B1B7835
:103A5000002B01D1FFF7BAFF0023154A9E420DDC6F
:103A6000FF2514491448D65CB44202D15E0070525E
:103A7000D5540133042BF6D10420F8BDD15C8C421F
:103A800003D10C4A5B009D52F6E70133042BF5D1BC
:103A90000023D15CFF2901D1D454F2E70133042B78
:103AA000F7D1E9E78813000008060020250600206A
:103AB0001C0000200E000020DC05000070B530C99D
:103AC000012322001A40101E1FD02B40181E1CD0AC
:103AD00064101A2C00D91924174E335D012B05D020
:103AE0000121200005F014FD012333556910080061
:103AF000124A1038124B904208D90122002152423A
:103B000020001A6005F022FD042070BD1C600D48E5
:103B100008F0DCF80C4B040018800C4B1B78002BD1
:103B200001D1FFF753FF0122094B9A64A922D20069
:103B3000995864189C50E7E7080600209086010019
:103B40001800002020A107000C00002025060020FE
:103B50000080004070B501240D68254204D10D207D
:103B6000FDF73AFE200070BD6D101A2D17D8002405
:103B7000012804DD4C68043C63425C416400094E4A
:103B8000735DA34204D02100280005F0C1FC7455E8
:103B9000280005F0F1FC03000420012BE3D00020F5
:103BA000E1E7C04608060020F8B501260D6834009C
:103BB000B04200DD4C682B003340181E0BD02300B0
:103BC0003340181E07D06D10002D05DCA123002006
:103BD0001E4ADB00D650F8BD641000201A2CFAD81B
:103BE0001B4F3B5D012B04D00121200005F090FC10
:103BF0003E552900174808F069F80A21053008F0F9
:103C000065F8154BA400E258144B12021343A2228C
:103C10001349D2008B50134C0C4B9C50124C195131
:103C2000012412495C50124B196900219950114A24
:103C3000904200DD1000A8228021D200985001227D
:103C400089005A5004201A60C5E7C04600F00140C0
:103C50000806002000B4C4045C0E01000300030049
:103C60000060004040A10040140500000405000071
:103C700000A00040FFFF0000030010B50120002B52
:103C800002DC1B30FDF7A8FD10BD0000F8B50124D3
:103C90000B6806000D00234204D10D20FDF79CFDAA
:103CA0002000F8BD5B1004D103F0AEFE40002043BD
:103CB000F7E72000072BF4D80D4A9B009C580D4FC6
:103CC0003B5D002B05D00021200005F021FC0023E6
:103CD0003B55012E06DD6B68042B03D10221200029
:103CE00005F016FC200005F0C1FA01244000DEE7D3
:103CF000F0FA00000806002010B50124044002D0AC
:103D00004410200010BD042810D90F23026813406E
:103D1000042B07D100F0B6FB21000A220AF06CFD4B
:103D20000400EEE7032B01D10430F5E70D20FDF789
:103D300053FDE6E7F8B50C00022803DC1C20FDF774
:103D40004BFDF8BD0868FFF7D7FF06006068FFF776
:103D5000D3FF0500A068FFF7CFFF0100794807F007
:103D6000B5FF04001A2D01D90020EAE7764F7B5DEC
:103D7000012B05D00121280005F0CAFB01237B554A
:103D80000021280005F0E2FB002C0ED020000138B5
:103D9000C046C046C046C046C046C046C046C046F3
:103DA000C046C046C046C046F1D1012731002800B8
:103DB000394005F0CBFB002C0ED020000138C04666
:103DC000C046C046C046C046C046C046C046C046C3
:103DD000C046C046C046F1D171103940280005F0F8
:103DE000B5FB002C0ED020000138C046C046C046AE
:103DF000C046C046C046C046C046C046C046C04693
:103E0000C046F1D10127B1103940280005F09EFBD2
:103E1000002C0ED020000138C046C046C046C04627
:103E2000C046C046C046C046C046C046C046C04662
:103E3000F1D1F1103940280005F088FB002C0ED09C
:103E400020000138C046C046C046C046C046C046F5
:103E5000C046C046C046C046C046C046F1D1012754
:103E600031113940280005F071FB002C0ED02000E4
:103E70000138C046C046C046C046C046C046C046DF
:103E8000C046C046C046C046C046F1D17111394057
:103E9000280005F05BFB002C0ED020000138C04646
:103EA000C046C046C046C046C046C046C046C046E2
:103EB000C046C046C046F1D10127B11139402800A3
:103EC00005F044FB3900002C0ED020000138C0461C
:103ED000C046C046C046C046C046C046C046C046B2
:103EE000C046C046C046F1D1F6113140280005F069
:103EF0002DFB002C0ED020000138C046C046C04625
:103F0000C046C046C046C046C046C046C046C04681
:103F1000C046F1D10121280005F018FB002C00D18A
:103F200022E720000138C046C046C046C046C04611
:103F3000C046C046C046C046C046C046C046F1D195
:103F400012E7C04640420F000806002004207047D8
:103F500010B5002803DC1C20FDF73EFC10BD0B68EB
:103F60000020DB07FAD40D30F6E700000122034BF6
:103F70001A64A822D20098587047C04600800040BA
:103F80000122054B10B51A64A822FA21D2009858D4
:103F9000890007F011FE10BD008000400048704706
:103FA00010FB00001B20704770B5054E0400335C09
:103FB0000D008B4202D005F0ABFA355570BDC046FE
:103FC0000806002070B50024084D635D012B09D15F
:103FD0000021200005F0BAFA0021200005F098FA2F
:103FE0000023635501341B2CEED170BD0806002060
:103FF000704711207047372070470000F8B501273F
:1040000004683C4202D045683D4203D10D20FDF7D3
:10401000E3FBF8BD64101A2CFBD80C4E335D012B6A
:1040200004D03900200005F073FA375508496D10A7
:104030008D4202DCE943C9172940200005F09CF9B4
:10404000335D012BE5D1034A1355E2E70806002052
:10405000FF030000E805002010B50800FFF7CEFFC1
:10406000002010BD70B505000C001A2814D80E4EA3
:10407000335C012B04D0012105F04AFA012373556A
:104080000A4B5B5D002B08D0611E8C4161428905A3
:10409000890D280005F070F970BD210028004C1E24
:1040A000A14105F053FAF7E708060020E8050020D3
:1040B000036810B5DA0703D40D20FDF78DFB10BDA2
:1040C0004168581004394A425141FFF7CBFFF6E7E7
:1040D00010B50800FFF7ECFF002010BD37B56946AA
:1040E0000A00064B30CB30C203680220042B02D1F9
:1040F00001F0A0F837BD01F0C5F8FBE780FA000039
:1041000010B50800FFF7EAFF002010BD10B5084CFD
:10411000237D002B05D00021142005F0F9F90023A0
:104120002375142005F028FA43425841800010BD41
:104130000806002010B5084CA37D002B05D00021F7
:10414000162005F0E5F90023A375162005F014FAF2
:1041500043425841800010BD08060020A0220023E1
:104160000349D2008B50034910328B507047C04630
:1041700000F0014000600040F7B52F4D2F4EEB6C72
:10418000002B14D0A9240023E4003759EB642C4BF6
:10419000186800280BDB2B4B19784A425141C9B2F1
:1041A000197005F0D3F9284B1B88DF1937512B6D97
:1041B000002B38D00021254B254FF45829653A783B
:1041C0000193244D8A4206D02B68032B03D8224A40
:1041D000D05C05F0BBF92B68204A0133134004D5AD
:1041E0000422013B5242134301331B4900228C46F7
:1041F0002B60042B18D06046C05C591CFF2802D1EC
:104200000B000122F5E7002A00D02B60012105F008
:104210009DF901233B702B68114A5B009B5A0C34BB
:10422000E418019BF450F7BD01235B422B6000238F
:104230003B700C4BF4E7C046FC800040008000401F
:1042400018000020240600200C0000204C0500006F
:1042500023060020040600201C000020030000802C
:104260000E0000205C460000084B094AFF201A801F
:104270005A809A80DA800023064A07491370074A59
:10428000087048708870C870136070470E00002076
:10429000DC050000230600201C000020040600208E
:1042A0000122024B52421A607047C046180000209B
:1042B00010B5034A0D21034802F044FA10BDC04670
:1042C00088FA000053050100E12170B549021A483F
:1042D00004F042FD002401220320184B18491A6102
:1042E0005C50043158508018083158501A6006301C
:1042F00004F0B6FFFF21134AA15401341B2CFBD15B
:1043000001220020104B01001A6004230F4A104DB7
:104310001468002CFCD02C680002013B2043116083
:10432000002BF5D101220B4B1A6004F0D1FE01F0F5
:1043300025FA03F0F3FF70BD8C1B002000800040C5
:10434000040500000806002000D0004000D1004015
:1043500008D5004004D00040F8B50B4E07003000EF
:104360000D0004F041FD0400A84200DD2C003D00DA
:10437000EB1B9C4205DD300004F040FD2870013548
:10438000F6E72000F8BDC0468C1B002010B50100E8
:10439000014804F0E9FC10BD8C1B002010B5054C51
:1043A000200004F0EFFCE1212000490204F0D4FCDD
:1043B00010BDC0468C1B0020C3070CD4064B1B68E5
:1043C000834208D8054B1B68984204D8031F1B681A
:1043D000002B00D018007047300600202C0600206B
:1043E0000023012210B50A48990001334250642B82
:1043F000FAD1084B084C1A609722002112012000C4
:1044000009F0A8FD054B064A6360064B1A6010BD13
:104410005C2D00200800002034060020A0250000AC
:10442000380600202806002010B5044B044A1A6004
:10443000044B054A1A60FFF7D3FF10BD3006002079
:10444000340600202C060020A40F0020044B1B681B
:104450001868000980B20238C343DB171840704760
:104460002806002000B59BB00200054901A80AF00B
:10447000B5F801A802F0E2FC02F02CFFFCE7C04610
:10448000E7FB00000B4BC20704D4042804D80A4BF6
:1044900000D00A4B180070470F2203681A40031D12
:1044A000042AF7D0064B092AF4D0064B032AF1D090
:1044B000054BEFE7C1FB000010F600000AF6000014
:1044C000CBFB0000DBFB0000D2FB00000020064A13
:1044D0000649131F186013681B099BB202339B0027
:1044E000D2188A42F5D3704738060020A40F002066
:1044F000F7B50F240126314B314A1968314B324D43
:10450000186813681F002740072F26D813681B0957
:104510009BB202339B00D218AA42F2D300242B4E46
:10452000A500AD192868FFF747FF01342860642C07
:10453000F6D1274C2068FFF73FFF2060254C20680C
:10454000002802D0FFF738FF20600025224B1B68AF
:104550000093009B9D4214DBF7BD1B099BB29B009F
:10456000D3189A42D2D01F68374208D1B94206D236
:10457000B84204D3043F3F68002F00D01F60043BC3
:10458000EFE7F0236B43154A9B181A78002A01D1F4
:104590000135DEE71F693C2300266B43DB199B00D6
:1045A00001930136BB1BF3D4019BB4001C1B0B4BC6
:1045B0001C19A069FFF700FFA061F2E73006002098
:1045C000380600202C060020A40F00205C2D0020BF
:1045D00008000020A40F0020DC050020041C00209F
:1045E000F7B50124204246D1234B1B689C469842D4
:1045F00041D3224B1B68019398423CD8031F1B6890
:10460000002B38D10200036800941B099BB2002BD9
:104610000FD10099131F196090422CD015682B1FE1
:104620001B68990069180C68013B14600A602A0035
:10463000EDE79D0055192968009C214219D18C4550
:1046400017D8019C8C4214D30E1F3468002C10D153
:104650000F680F343C40072C08D92F60151F2B60C2
:104660000B680A601B099BB20A00D0E70099316011
:10467000CDE7013BCBE7F7BD300600202C0600203C
:104680000D4970B50A000D4D1368141F1B092668EB
:104690009BB2981C002E0BD000238A4200D00B0046
:1046A00023608300C91880001218AA42ECD370BDA1
:1046B0001B011360F7E7C04638060020A40F002056
:1046C000F8B5124C27000F223B681D09ADB213420A
:1046D0000DD06E1CB600A74204D032003900200075
:1046E00009F025FC0022A3190436A4191A6002352A
:1046F000AD00074B7F199F42E5D31B1B9B10013B6D
:104700001B012360034B1C60F8BDC0463806002027
:10471000A40F002028060020F0B59BB0FFF726FC70
:1047200000240700214AA300D0580134FFF758FFA6
:10473000642CF7D11E4B1868FFF752FF1D4B186809
:10474000002801D0FFF74CFF00261B4B1B689E4240
:1047500017DBFFF795FFFFF7CBFEFFF7B1FFFFF782
:1047600005FC164BC21B1B6815491B6801A81B09D9
:104770009BB2023B09F032FF01A802F05FFB1BB0C5
:10478000F0BDF02575430F4BED182B78002B01D1B0
:104790000136DAE72B695C1E002CF9DBA300EB186D
:1047A0009869FFF71DFF013CF6E7C0465C2D00202D
:1047B00008000020A40F0020DC05002028060020AF
:1047C000A1FB0000041C0020F7B5174D4F1C2B68FF
:1047D00006001B680C001B099BB201929F420BDB79
:1047E000FFF79AFF2B681B681B099BB29F4203DBF4
:1047F0000A20FCF7F1FFFEBD2868A71CBA00DB1BEE
:1048000081181B010B6029600021031F19600F2311
:104810001E4003002401264340C3083A9A189A42D6
:10482000E9D9019902C3FAE728060020F7B5030089
:104830000122134004000D000193002B2BD1174BD4
:104840001B68834227D8164B1B68834223D90F234A
:10485000144F386000681840FFF7B6FF019B3C68B2
:10486000061E3B6017D0236804301B099BB29D4293
:1048700000DD1D00AA00211D251F09F04FFBFFF7D9
:1048800025FE2E60FFF734FE00232B602268064BC6
:104890001340236034002000FEBDC04630060020D7
:1048A0002C060020A40F0020F0FF0F00032304308B
:1048B00010B5C11719400918891000220420FFF70C
:1048C00083FF10BD70B5050008000C00FFF7EEFF78
:1048D0000023002804D170BDE95CC21811710133B6
:1048E000A342F9DBE343DB171C40002304192371C7
:1048F000F1E7F0B50C009BB0022804DC1C20FCF7AB
:104900006BFF1BB0F0BD01230868184206D10428D4
:1049100004D90F2601683140042901D00E20EEE7AA
:1049200061680D001D40F9D10429F7D90A683240A9
:10493000042AF3D1A2681A4201D10D20DFE7FFF764
:10494000A1FD06006068FFF79DFDA768010001ACAE
:104950007F103000257003F029FE39006423220007
:1049600003F089FE200009F07FFE01002000FFF720
:10497000A9FFC6E710B51C4CA544041E02D1FFF7E1
:1049800095FF0BE003F02AFD0138062828D807F030
:10499000FFF8090911182904240000208023DB00F6
:1049A0009D4410BD200003F095FD011B2000FFF782
:1049B00089FFF3E7200003F03BFD4300012018438B
:1049C000ECE780226946D200200003F048FD6846EB
:1049D00009F04AFE01006846E9E704210348E6E7DA
:1049E0000020CCE70420D9E700FCFFFF58FC0000C2
:1049F00070B50C00022803DC1C20FCF7EDFE70BD36
:104A000001230868184206D1042804D90F2501683B
:104A10002940042901D00E20EFE761681942FAD13C
:104A20000429F8D90A682A40042AF4D1A2681A4253
:104A300001D10D20E1E7FFF725FD05006068FFF7D4
:104A400021FDA46801006410280003F0AFFD2100DF
:104A500003F0ECFDFFF78EFFD1E770B50D000128E4
:104A600003DC1C20FCF7B8FE70BD0124086820425E
:104A700006D1042804D90F2102680A40042A01D073
:104A80000E20EFE76A682242FAD1042AF8D91368A7
:104A90000B40042BF4D1FFF7F5FC06006868FFF724
:104AA000F1FC0100300003F081FD03F003FE400043
:104AB0002043D9E7F8B507000C001C20012F0BDDBF
:104AC00001250868284206D1042804D90F2102686C
:104AD0000A40042A03D00E20FCF77EFEF8BD62686F
:104AE0002A42F8D1042AF6D913680B40042BF2D1DC
:104AF000FFF7C8FC06006068FFF7C4FC0100022F46
:104B000014D0A4682C4211D06410300003F04EFD84
:104B1000050003F063FC012811D1002C02DD0135F2
:104B2000012C06D12800FFF725FFD7E701246442B6
:104B3000EBE7280003F0DBFC013C0500F0E702286E
:104B4000F0D1002CEEDD0135012CEBD00022280045
:104B5000110003F0FEFC03F0CAFC013C0500F3E782
:104B600010B502F055F9431E9841800010BD0000B9
:104B7000086870B501240500254006D1042804D931
:104B80000F2302681340042B03D00E20FCF724FEF1
:104B900070BDFFF777FC03782900233B5A4253414D
:104BA0001022C01809F028FE80239B05C218044B70
:104BB0009A4201D91420E9E740002043E8E7C046C3
:104BC000FFFFFF3F10B50124044002D04410200035
:104BD00010BD042810D90F2302681340042B07D1FD
:104BE000FFF750FC21000A2209F006FE0400EEE760
:104BF000032B01D10430F5E70D20FCF7EDFDE6E7CE
:104C000010B50868FFF7DEFF09F070F804F0C4FF84
:104C1000054B002208F05EFA04F064FD09F030F85C
:104C200043000120184310BD00408F4010B50868B4
:104C3000FFF7C8FF07F0DEFA094907F0A9F909F004
:104C40008FF804F0A7FD074B002208F043FA04F0A8
:104C500049FD09F015F843000120184310BDC04676
:104C6000D30237390000D040F7B50C00042803DC2C
:104C70001C20FCF7B1FDFEBD0868FFF7A3FF019003
:104C80006068FFF79FFF0600A068FFF79BFF050025
:104C9000E068FFF797FF07002069FFF793FFAE4238
:104CA00001D11F20E5E7019BC01B9B1B5843A91B9B
:104CB00007F00CF8C71901207F003843DBE700003C
:104CC00070B50E00012803DC1C20FCF785FD70BDCB
:104CD0004B68581009F00AF8040030680D004010C5
:104CE00009F004F802000B002000290007F0E8FD9D
:104CF0000B4A0C4B04F096FD02000B0000200A4901
:104D000008F05AFC0022094B08F0E4F9084B002295
:104D100008F0E0F908F0B4FF430001201843D6E79B
:104D20006C45D9CC955BC83F0000F03F40A5E540FD
:104D300000408F4010B5034A0B21034801F002FDEB
:104D400010BDC04600FC0000F8FB000000207047CA
:104D500010B51E20FCF740FD10BD10B51E20FCF75D
:104D60003BFD10BD10B51E20FCF736FD10BD10B583
:104D70001E20FCF731FD10BD10B51E20FCF72CFDE8
:104D800010BD10B51E20FCF727FD10BD10B51E206C
:104D9000FCF722FD10BD10B51E20FCF71DFD10BD57
:104DA00010B51E20FCF718FD10BD10B51E20FCF735
:104DB00013FD10BD10B51E20FCF70EFD10BD10B583
:104DC0001E20FCF709FD10BD10B51E20FCF704FDE8
:104DD00010BD10B51E20FCF7FFFC10BD10B51E2045
:104DE000FCF7FAFC10BD10B51E20FCF7F5FC10BD59
:104DF00010B51E20FCF7F0FC10BD10B51E20FCF70E
:104E0000EBFC10BD10B51E20FCF7E6FC10BD10B584
:104E10001E20FCF7E1FC10BD10B51E20FCF7DCFCE9
:104E200010BD10B51E20FCF7D7FC10BD10B51E201C
:104E3000FCF7D2FC10BD10B51E20FCF7CDFC10BD58
:104E400010B51E20FCF7C8FC10BD10B51E20FCF7E5
:104E5000C3FC10BD10B51E20FCF7BEFC10BD10B584
:104E60001E20FCF7B9FC10BD10B51E20FCF7B4FCE9
:104E700010BD10B51E20FCF7AFFC10BD10B5034AE5
:104E80001F21034801F05EFC10BDC046D0FC0000AD
:104E9000C8FD0000002070470120704701207047C6
:104EA00000207047012070470020704700207047A5
:104EB000002070470020704710B5034A09210348BD
:104EC00001F040FC10BDC04664FF0000ACFF0000D4
:104ED0000120034B1860034B1B6883401843704745
:104EE000C40F0020A80F0020F0B5EFF310810123BC
:104EF000194083F31088134AA1261268124D013A13
:104F00009340A022114FD205F600002B17D02C6839
:104F1000945103420BD0C046C046C046C046C0466E
:104F2000C046C046C0462C68D4515B08EDE7D4515A
:104F3000C046C046C046C046C046C046F5E781F3FD
:104F40001088F0BD20000020B40F00200C050000E8
:104F500030B585B001AD0C220649280008F0DEFF0F
:104F60000024285D01210134FFF71EF80C2CF8D134
:104F700005B030BDF9FF000030B585B001AD0C22A1
:104F80000649280008F0CAFF0024285D00210134EA
:104F9000FFF70AF80C2CF8D105B030BDF9FF00007E
:104FA000F7B56A463B4B01AE1380062393703A4B2C
:104FB00033800F23B370FEF7D9FF384B384DC0183C
:104FC0002B68984201D200232B602C68002C41D121
:104FD000375D01213800FEF7E7FF0134002138007A
:104FE00004F0B4FA032CF3D1002401276B461E5DB4
:104FF00039003000FEF7D8FF01343900300004F0EA
:10500000A5FA032CF2D1C8200138C046C046C046DC
:10501000C046C046C046C046C046C046C046C04660
:10502000C046F1D16B4600211878FEF7BDFF6B46F4
:1050300000215878FEF7B8FF6B4600219878FEF7FC
:10504000B3FFFEF793FFFA2300241B01C01828606A
:105050002000FEBDFEF78AFF2B6800249842F7D39C
:10506000042004F003F90600052004F0FFF83618C8
:10507000062004F0FBF80B4B9B1B181A0A4BA042AE
:1050800006DB18600023094A2B6013600124DFE768
:105090001C60F7E7040500000D0E0000102700005B
:1050A000BC0F002043030000A80F0020C40F002005
:1050B0000B6810B5044A5B101360044B186803F0CA
:1050C00030F9002010BDC04624000020C00F002091
:1050D0000022054B10B51A60044B1B68934201D0A7
:1050E00003F01DF9002010BDC00F0020B01A0020F1
:1050F00010B5041E0CDA1A24084BA400E2581F2332
:105100001A401E3B9340064A1360064A136010BDC6
:10511000FEF748FFA042EEDDEEE7C0465C0E010060
:10512000B40F0020180500500200086810B5C3072E
:105130000FD540101823012A03DD4A68042A00D144
:105140000833054A1360FEF753FFFFF7D1FF002035
:1051500010BD01204042EDE72000002010B50028DE
:105160000CDD0A68131F591E8B4107490B60042A86
:1051700006D0FFF701FF0022044B1A60002010BD8B
:10518000FFF7E6FEFAE7C046B80F0020A80F0020A0
:1051900010B50124044002D04410200010BD0428A2
:1051A00010D90F2302681340042B07D1FFF76AF9C7
:1051B00021000A2209F020FB0400EEE7032B01D1B5
:1051C0000430F5E70D20FCF707FBE6E70868F8B5C3
:1051D000C3071AD5FFF7DCFF0300203B5E2B25D861
:1051E0000520434301221D180020114E9D4219D075
:1051F00005211024F75C3C4200D080180139520090
:1052000064100029F7D10133F0E704280ED90F22EA
:1052100003681A40042A09D11B099BB2002B05D050
:105220000379DAE7012340001843F8BD0120FCE7C9
:105230000500010070B508680D00FFF7A9FF040024
:105240006868FFF7A5FF621E0100042A14D8451EF6
:10525000042D11D805236B439B18012215009D4096
:105260002B00064805682B430360054B1B68002B89
:1052700002D0200003F054F8002070BDC00F0020C1
:10528000B01A002070B508680D00FFF781FF040018
:105290006868FFF77DFF621E0100042A13D8451ECF
:1052A000042D10D805236B439B1801229A40074810
:1052B000036893430360064B1B68002B03D0002256
:1052C000200003F02DF8002070BDC046C00F002064
:1052D000B01A0020F0B5050089B008680C00FFF78F
:1052E00057FF0690022D36DD6068FFF751FF0190F1
:1052F000A068FFF74DFF04000127231D661E0793DA
:10530000731C0293079B9E4235D00523734305937C
:10531000019B019D05330493049BAB421ED0042ED8
:1053200016D86B1E042B13D80122059B2349013B81
:105330005B199A409446224A0B681068069A3A40D4
:1053400003920DD062461A430A60012200280DD153
:105350007F000135E0E701240194CDE7029ECFE70D
:10536000624693430B600028F2D0039A029928000A
:1053700002F0D6FFECE7019B1E1D042E1AD8012C6B
:1053800018D1002505273B0021006B439B1999404C
:105390000B000A4A013511689943094B11601B68DB
:1053A000002B05D0019B0022581D290002F0B8FFF8
:1053B000052DE8D1002009B0F0BDC046C00F002087
:1053C000B01A0020F0B53B4B85B01B680C00002BD9
:1053D00003D101204042FFF78BFE012627683E40A3
:1053E0003CD1042F3AD90F233A681340092B35D109
:1053F0007B685B100293029B9E4258DAB300FB1855
:105400009868FFF7C5FEFF2305000414001218403A
:105410001C4029492B404043019306F057FC0304EC
:10542000200025496043039306F050FC039C0002D2
:10543000044301982049404306F048FC1F4B204399
:105440001B68202B06D1AD00AD0E1D4BAD00EC58F6
:1054500000022043FFF748FD0136CCE73800FFF794
:1054600097FEFF2605000714001230401249404302
:1054700006F02CFC3740040438000F49784306F04E
:1054800025FC2E400002044330000B49704306F017
:105490001DFC0A4B20431B68202B06D1AB009B0E42
:1054A000074A9B009B5800021843FFF71DFD002090
:1054B00005B0F0BDB40F0020590600002000002008
:1054C000E0010100086810B5C30703D5FFF760FECF
:1054D000054B1860054B1B68002B03D0024B186866
:1054E00002F01FFF002010BDC00F0020B01A0020E6
:1054F0009D4B70B51B68002B0DD19C4C2368002B75
:105500000AD19B4A1268002A06D19A4B1B68002BCD
:1055100001D0FFF745FD70BD974D2A68002A1BD1C9
:10552000944A1268002A10D0FFF73AFD0028F2D002
:10553000FFF70EFD8E4B226819681A6000290BD008
:10554000002A09D1FFF718FDE5E7894A1268002A09
:10555000F0D1002BEED0EBE700210D2003F0F6FF99
:1055600000210E2003F0F2FF00210F2003F0EEFFD8
:105570002E68012E5DD0022E00D1A2E0002E51D166
:10558000013631007A4C04202368994303F0DEFF92
:1055900004212368052019404B42594103F0D6FFEE
:1055A00010212368062019404B42594103F0CEFFD9
:1055B00080212368090119404B4259410C2003F016
:1055C000C5FF80212368090219404B4259410B2035
:1055D00003F0BCFF80212368490219404B42594126
:1055E0000A2003F0B3FF80212368890219404B424F
:1055F0005941092003F0AAFF80212368C9021940FC
:105600004B425941082003F0A1FF802321681B036E
:1056100019404B425941072003F098FF31000D20FB
:1056200003F094FF2B680321581C06F035FC296019
:1056300071E702214E4C0720236819404B42594123
:1056400003F084FF0820216801404B42594103F0D8
:105650007DFF80212368C90019404B425941052034
:1056600003F074FF80212368490119404B425941DE
:10567000062003F06BFF80212368C90119404B42CB
:105680005941042003F062FF8021236889031940F7
:105690004B4259410A2003F059FF802321681B0423
:1056A00019404B425941092003F050FF31000C20B2
:1056B00003F04CFF31000B2003F048FF31000E20B7
:1056C000AEE720212A4C0720236819404B4259415C
:1056D00003F03CFF40212368082019404B42594108
:1056E00003F034FF80212368092019404B425941BF
:1056F00003F02CFF80212368490019404B42594197
:105700000A2003F023FF80212368890019404B42BF
:1057100059410B2003F01AFF8021236889011940A9
:105720004B4259410C2003F011FF802123684903AB
:1057300019404B425941062003F008FF802123689D
:10574000C90319404B425941042003F0FFFE802356
:1057500021685B0419404B425941052003F0F6FED5
:1057600001210F205CE7C046B80F0020C00F0020C9
:10577000B00F0020C40F0020AC0F0020012010B596
:105780004042FFF7B5FC0020FFF7AEFB012003F01D
:10579000BDFC10BD10B5034A0B21034800F0D2FF39
:1057A00010BDC046E0020100380301008023F0B5BF
:1057B00002255B051A690A4C0A4BA1261D510327D5
:1057C0008025F600ED00BA43884202D300221A5128
:1057D000F0BD5F59002FFCD098518018F4E7C04607
:1057E0000405000000E0014010B5002806D1C020EB
:1057F000B02140028902FFF7D9FF10BDB0208021FF
:105800008002C902F7E7000043425841064B40427C
:105810001840B0239B02C018036800201A0E532AB8
:1058200001D11B02180A704700C0FEFF30B50124E9
:105830008025054B054AED009C505C59002CFCD09E
:1058400001600021995030BD00E0014004050000D6
:1058500043425841074B40421840B0239B02C018B6
:10586000A62310B50902DB05090A1943FFF7DEFF7D
:1058700010BDC04600C0FEFFF0B5012480260D4BD0
:105880000D4DF6005C51002902DC00225A51F0BD9A
:10589000577814783F022743947824042743D47818
:1058A000043224063C439F59002FFCD010C001391C
:1058B000E9E7C04600E001400405000070B50500BE
:1058C0004B680A009C1C2100A400FFF7D5FF281993
:1058D00070BD0000134B1B68002B0CD08022B0233E
:1058E000D2029B0200280BD11A1D5B681B0E522BA3
:1058F00000D110007047B022C02392025B02F1E792
:1059000082420DD903681B0E522B09D14368023322
:105910009B00C018824203D903681B0E522BE9D0AA
:105920000020E7E7C8100020F0B50020B7B0002441
:10593000FFF7D0FF270005002600002D2ED1284DAF
:105940002868FFF761FF32003B0001900094254971
:1059500004A808F043FE04A801F070FA224B64206A
:105960001C682B68A0215A425341204A5B421340D5
:10597000B02292029B18E41A6043490206F0A6F98D
:10598000A0225202030000921949220004A808F044
:1059900025FE04A801F052FA37B0F0BDFF226B6873
:1059A00029689C460233FF180B12013613409C42B3
:1059B00000DA1C00FF200A140240039262460140F4
:1059C00001920091039A0B4904A808F007FE04A86D
:1059D00001F034FA2800FFF77DFF0500ADE7C0466F
:1059E000C81000205D040100CC10002000C0FEFFA4
:1059F000070401004904010070B50020FFF704FF0F
:105A000004000120FFF700FF844200DA04000A4B83
:105A10001D686A42554128001D60FFF7E5FEA0227F
:105A20006B4252021340054A28009B18044A611C2D
:105A30001360FFF70DFF70BDC81000200480010047
:105A4000CC100020F8B50020FFF7DEFE0700012093
:105A5000FFF7DAFE3E00204D0643204C0DD1802199
:105A6000C020C9024002FFF7A1FE01213000FFF76C
:105A7000EFFE1B4B2E6023601DE0874209DD0023F3
:105A8000B0212B60164B890223602368002001257A
:105A900017E0012380212B60124BC9022360F4E739
:105AA000120E522A08D0002800D023600E4801F0C0
:105AB000C5F9FFF7A1FFF8BD28005A68023292002D
:105AC0009B188B4205D21A68561CE9D10028F2D0E7
:105AD000D1E72160EFE7C046C8100020CC100020BD
:105AE0000480010004C002002204010070B50020FF
:105AF000FFF7F0FEFF260500002801D1280070BD49
:105B000003681C143440FFF7E5FEDA2CF4D10500DD
:105B1000F2E70000FF2270B51F4CD20000212000E8
:105B200008F018FAFF25FFF7E1FF0026002818D13A
:105B3000F0210A22194849420B00962553432D01B2
:105B40001B185D192D78002D07D0154D154E5D19C8
:105B50009B191B78DB00E3582B60013A002AEBD13C
:105B600070BD03681A142A400A2A0AD11A122A4060
:105B7000FF2A03D0D200A1180B71A050FFF7AAFE94
:105B8000D4E7132AFAD11B122B40FF2BF6D0DB00EF
:105B9000E2181671E650F1E764250020041C00208D
:105BA000680900006109000010B59AB0FFF74AFFCC
:105BB000FFF7B0FF00231A000A48D900415801330B
:105BC0004C1EA1415218FF2BF7D1074901A808F03C
:105BD00005FD01A801F032F9044801F02FF91AB0CF
:105BE00010BDC0466425002092040100A6040100F7
:105BF0008022F0B55200A1B00021684808F0AAF94F
:105C0000802200215200664808F0A4F9654BFF2766
:105C10001B681A00049353425A4110000592FFF783
:105C2000E3FD049C0020631E9C415F4B64421C40CA
:105C30005E4BE418FFF75AFF0600002E2FD10498A0
:105C4000FFF7E2FD411C0598FFF702FE059A554B50
:105C5000574D1A602C60FFF75DFFFEF79FFB514B1D
:105C600064201B68A0215A4253414F4A5B421340B3
:105C7000B0222C6892029B18E41A6043490206F095
:105C800025F8A0225202030000924A49220007A8E8
:105C900008F0A4FC07A801F0D1F821B0F0BD3268EB
:105CA000131412123A403B4003921A000A3A092A8E
:105CB00049D83A4B039A995C002931D110223E48C9
:105CC00008F048F935002B6803991A123A409142BE
:105CD00009D11A143A400B2A27D0132A2DD00A2AA8
:105CE00001D1354B1D602800FFF7F4FD051EEAD1F8
:105CF000314B196800290FD02000FFF7DFFD0400A9
:105D00002D4B5B195968002903D02000FFF7D6FD01
:105D1000040004350C2DF3D1204B0121039A995432
:105D20003000FFF7D7FD060087E73B40022BDADCA7
:105D3000214A9B00D3185D60D5E7102200211E4840
:105D400008F008F9CFE71A00153A082AE8D8144AEB
:105D50000399525C002AE3D13500152B00D01500C1
:105D6000300003681A143A40152A0FD01D2A00D1BA
:105D70000025FFF7AFFD0028F3D1002D04D020004F
:105D80002900FFF79BFD0400054BC6E7039A1B1291
:105D90003B409A42EDD10500EBE7C046C80F00201A
:105DA000D0100020C810002000C0FEFF04C0020078
:105DB000CC100020EC030100EC2E002010B5FFF702
:105DC00017FF10BDF0B585B0039203220333DC1733
:105DD000294D1440E4182B68284F5A425341802221
:105DE0005B42D202A4103B409B18A21C0291244E9D
:105DF000910000910190316800980A18934215D2E1
:105E0000FFF7F6FE2B685A42534180225B421F4047
:105E1000D202BF183368009A9B189F4206D21948D5
:105E200001F00CF80025280005B0F0BD029B356894
:105E300019066B461A7BA423DB051343FF222F00B0
:105E4000090C1943019B12041B0413401943280039
:105E5000FFF7ECFC0837281D21003760FFF7E6FC50
:105E6000002C04D00A9A21003800FFF705FD009BA2
:105E7000083BFF183760D6E7C810002000C0FEFFBF
:105E8000CC100020C6030100704770470021094B69
:105E9000094A59600131516059680029FCD000213C
:105EA0001961012393600222044B8131FF315A5062
:105EB0001A607047FC1000400010004000E100E054
:105EC0000222064B0121DA670022054B5A61054A7E
:105ED00011615A69002AFCD07047C04604E100E015
:105EE000FC1000400010004010B5044C2378002B3B
:105EF00001D0FFF7E5FF0020207010BDD111002078
:105F00000120024B1B685B001843704754120020AD
:105F10000120024B1B685B001843704728000020DB
:105F20001FB5064B06491A6801A808F057FB08215F
:105F300001A8FEF7C7FC05B000BDC04658120020FE
:105F4000340501001FB580235B051A6E044901A8C2
:105F500008F044FB082101A8FEF7B4FC05B000BD21
:105F60003405010010B5044C200008F07DFB010051
:105F70002000FEF7A7FC10BD5D1200200E4B10B5EF
:105F80001B680E4C5A1C0FD00D4C002B0CD00D4C26
:105F9000012B09D00C4C022B06D0094C042B03D04A
:105FA0000A4C052B00D1074C200008F05DFB0100D6
:105FB0002000FEF787FC10BD2C00002039050100F1
:105FC00060FA00004405010067FA00003E05010088
:105FD00070B504000D001600FDF7D2FF80230122EA
:105FE00000215B051B6E6270E270020AA271020C56
:105FF000E2711A0A60716372000EA2721A0C1B0E13
:1060000026702571A1702072E272237370BD0000AA
:1060100070B5214C2278002A3DD1204B01215A60D5
:106020008022D20511605A68002AFCD00022072085
:106030001B4B1C4901255A500439585008315A50FD
:1060400019481A4958501A491A485A501A495A5068
:10605000A622D2009D50082218495A5004315850A7
:106060000220174958501749174858501748043903
:106070005850182016495850C12189005A500539E6
:10608000FF395858921802435A501249124A9950EF
:10609000FFF7FCFE257070BDD1110020FC00004010
:1060A000001000400C050000746962751C050000BA
:1060B00024050000200004022C0500001405000047
:1060C000340500003C050000FFFF00002110010026
:1060D00054050000D21100200405000013B5094B3F
:1060E00004000093084B019307280AD8074B1B783C
:1060F000002B01D1FFF78CFF6B46054A1957054B62
:10610000D15013BDE2ECF0F4F8FC0004D1110020F2
:10611000001000400C05000070B50E4B06001B7807
:10612000002B01D1FFF774FF00200B4D2C78844227
:106130000ED00A4B202219780323091B1940084B63
:106140004901C918300007F0E9FE0120013C2C701C
:1061500070BDC046D11100205C120020D01100207B
:10616000D2110020002370B588B0984235DD0D684B
:1061700001262C0034409C422FD12300042D2CD921
:106180000F222B681A402300092A26D16A683F2A69
:1061900023DD6846FFF7C0FF230000281DD06B46B3
:1061A00019783300A14203DB6B461B5D5B00334370
:1061B000A200AA1801349360202CF2D1092169446D
:1061C0004A780B7812021A438B781B041A43CB7857
:1061D0001B061343024A13600423180008B070BD65
:1061E0005812002070B5454B8AB01B78002B01D1A6
:1061F000FFF70EFF02AC2000FFF78EFF002802D150
:1062000000200AB070BD23780B2BF9D96378012BDD
:10621000F6D1E378012BF3D100231120384E394D0C
:1062200033602B7068442379374A417813600278D1
:1062300009021143827812041143C27812060A43FC
:1062400032490A60002B0ED1152169444A780B7837
:1062500012021A438B781B041A43CB781B06134394
:106260003360002318E0012B1AD1152169444A78C4
:106270000B7812021A438B781B041A43CB781A212D
:106280001B06134333600E23627C6944934200DD96
:10629000130000229A422CD100220420EA54B0E7D5
:1062A000022B03D1627B10331621EEE7042B0DD1B4
:1062B000152108226944684607F030FE00980199CC
:1062C00003F080F907F0DCFC3060CAE7052BC8D189
:1062D000152108226944684607F020FE00980199BC
:1062E00003F070F907F0CCFC3060627D0A231E21B8
:1062F000CBE7885CA8540132CCE7C046D11100201E
:10630000541200205D1200202C00002058120020A2
:1063100010B5134B04001B78002B01D1FFF778FE5A
:10632000FFF7CEFD00200F4A0F49104B5450586024
:106330000130106058680028FCD00020186101303E
:10634000906018690028FCD0094B0A481B785B0153
:106350001B185350FFF7B4FDFFF798FD10BDC04662
:10636000D11100200010004004050000FC10004086
:10637000D0110020D211002010B588B000281DDDFA
:106380000A68012113000B4018D1042A16D90F20E6
:1063900014682040092811D150683F280EDD98006C
:1063A000101880680024084201D04010C4B268462A
:1063B000C4540133202BF2D1FFF7AAFF002008B00C
:1063C00010BD000010B5002813DD0C68E30710D5E0
:1063D0006410532C0DD8084B1B78002B01D1FFF70C
:1063E00017FEFFF76DFDA123044ADB00D450FFF731
:1063F0004DFD002010BDC046D1110020001000400E
:1064000010B500280EDD0C68E3070BD56410FF2CD7
:1064100008D8054B1B78002B01D1FFF7F9FD034A83
:10642000034BD450002010BDD111002000100040BB
:106430002405000010B5002805DD0868C30702D553
:106440004010FFF74BFE002010BD70B588B000284B
:1064500020DD0124086804401CD104281AD90F2328
:1064600002681340042B15D1FEF70CF8060008F063
:10647000FBF80500122800D912252A0002210D324E
:106480006846FFF7A5FD6B465D73A54205DC6846CF
:10649000FFF73EFF002008B070BD2300325D6B4463
:1064A0009A730134F1E7F0B50D008BB0012832DDAD
:1064B00008680122040014402DD104282BD90F2391
:1064C00001680B40042B26D16B68134223D0FDF7E3
:1064D000D9FF6E6807007310019308F0C5F8050036
:1064E0000E2800D90E252A000121113202A8FFF73B
:1064F0006FFD6A46127902AB5A7302AA7312937344
:10650000019B76141B0ED67313745574A54205DCDB
:1065100002A8FFF7FDFE00200BB0F0BD3A5D02A916
:1065200063189A740134F1E730B589B0002814DD9E
:106530000C68E30711D5102268460021FFF748FDDB
:106540006B466A4665105D73684663122D0E6414CF
:106550009373D4731574FFF7DBFE002009B030BDD0
:10656000174B184A5968002903D00021596001319E
:106570009160196900291FD0002018618023DB0079
:10658000D3581149012B18D1A923DB00D3585B4202
:106590000B600E490B78032B01D801330B700320DD
:1065A0000B490B78013303400B700A495B015B1800
:1065B000094953500123936070470860FAE7C046C9
:1065C000FC10004000100040280000205C12002059
:1065D000D0110020D21100200405000010B50A4B94
:1065E0001B78002B0ED0FFF76BFCA1230722074C72
:1065F000DB00E250FFF74AFC0022054B0620E25088
:10660000FFF76CFD10BDC046D11100200010004006
:106610002405000010B5034A1021034800F092F849
:1066200010BDC046B4040100AE040100044A05498F
:106630001368C85401339B059B0D13607047C04617
:106640008C1600208C12002070B5124C124A236860
:10665000834202DC0023236018E0115C451C0E001D
:10666000FA3E012E07D8AB4211DD515D002902D060
:1066700028399F2901D82800EAE70100151A565C3D
:106680006E5401318B42FADC181A206070BD117013
:10669000FAE7C046981A00209816002010B5FDF7BA
:1066A00065FC064B1A68824201D900221A601B68F9
:1066B000C31A034898428041404210BD881200200E
:1066C000204E000010B5094C094A23681268934215
:1066D00000D110BD074AD05CFDF758FE0028F8D065
:1066E000236801339B059B0D2360ECE79016002087
:1066F0008C1600208C12002010B50400064B074AAF
:106700001B6812689B1ADB439B059B0DA34200DBB1
:1067100010BDFFF7D7FFF1E78C1600209016002080
:1067200070B5FFF7E3F9FF250400002801D1200030
:1067300070BD03681B142B401D2B00D10400FFF714
:10674000C9F8F2E770B5074E33680E2B08DC0C254C
:106750005D43054C0133285164196160A2603360C8
:1067600070BDC04694160020FC2E0020F0B5B7B0D6
:10677000040007F079FF012802D8002037B0F0BDEF
:1067800023785B2BF9D1013825182B785D2BF4D1B8
:1067900001343A21200007F04FFF061EEDD0071B01
:1067A000002FEADD210000243A0004A807F074FF5E
:1067B00004AB711CDC556F1AA742DEDD1DAD3A003B
:1067C000280007F069FF134BEC551B6803950193F4
:1067D000019BA342D1DD0C2666430F4B04A9F6189A
:1067E000306807F037FF051E05D17368B66802935D
:1067F000029B9D4201DB0134EAE73068039907F010
:1068000029FF37000836002801D17868B6E701353E
:10681000EEE7C04694160020FC2E002010B5FAF7D3
:10682000F3FDFEF7B7FFFAF719FEFDF741FDFEF79E
:1068300081FAFEF723FBFFF7EDFE01F011F901F0FD
:106840003DFD01F06FFD01F0B9FFFAF725FEFEF7FF
:1068500033FB10BD962210B512010021034807F04A
:1068600079FB0022024B1A6010BDC046041C0020B8
:10687000DC05002070B514007F22174BC000C05803
:106880000D00836813401C2B01D0002070BDC3682D
:10689000190011400429F8D101690A40192AF4D1DC
:1068A0001B0A01339B000C30C018FDF7EBFD037889
:1068B00006000120002BE9D0300007F0D5FE0023B0
:1068C000A042E2D1A34201DB0120DFE7F15CEA5CF8
:1068D0009142DAD10133F5E764250020064B074ADF
:1068E0001B6812689B1ADB439B059B0D01228342A8
:1068F00000DC0022100070478C160020901600204B
:10690000F8B505000C0016001F1E0ED10320FFF77E
:10691000E5FF002808D0FA20FFF788FEE8B2FFF76D
:1069200085FEE0B2FFF782FEF8BD501DFFF7D6FFEF
:106930000028F9D0FB20FFF779FEE8B2FFF776FEDA
:10694000E0B2FFF773FEF0B2FFF770FE3012C0B294
:10695000FFF76CFE3C00E31B9E42E5DD2078FFF76D
:1069600065FE0134F7E7000070B50024F0250B4BFD
:106970001B68A34202DCFFF76DFF70BD2B00634371
:10698000074A9B181A78002A05D05978002311204D
:106990001A00FFF7B5FF0134E9E7C046DC05002027
:1069A000041C0020F8B507000024F0252B006343E9
:1069B0000C4A01349E18B74211D0317800290BD00F
:1069C0000133D15C002311201A00FFF799FF2A0040
:1069D0000021300007F0BEFA0A2CE7D1F8BD024BC7
:1069E0001C60F9E7041C0020DC050020F0B5150050
:1069F00001222F007A4C1740A54401900291002FEC
:106A000011D005AB1A706A105A70120E1A71052255
:106A1000691299706D140299DD70FFF771FFCF2331
:106A20009B009D44F0BD042D2AD90F242868044002
:106A3000042C32D1022304AA28001371FDF722FD91
:106A4000050007F011FEC82302009B00984200DDFC
:106A50001A007C1C97420DD1984206D9614804ABBC
:106A600003226149C01807F059FA220005AB0299C8
:106A70000198D2E72700611E695C05ACE155E8E7A3
:106A8000042D00D0A7E0032304AA043D13716B4238
:106A90005D4105AB55710222E9E7092C7ED1042244
:106AA00005AB1A706A685110009169465212097854
:106AB0009A70009A59701F2A01DD202200926A46BE
:106AC000127806ACDA70009BBB4202DC05ABE21A1E
:106AD000CDE70126BB00EB189868064006D10428D4
:106AE00037D90F210368194002290CD101232370E3
:106AF0004310637042121B0E4014A270E0702371A9
:106B000005340137DFE7042921D102232370FDF783
:106B1000B9FC039007F0A8FDA31C142809D86070E5
:106B2000864201D19C19ECE7039A925D9A55013691
:106B3000F6E714226270039A925D9A550136112E7F
:106B4000F9D12E23E374237563751634D9E701292F
:106B500007D1032304382370434258416070023444
:106B6000CFE7092909D10423237043685A106270C2
:106B70005B12A370E6700434C3E703290BD105232D
:106B800023700068020992B2430F92000B40D31A9F
:106B900063701B12EDE726700134B2E7032C00D0BE
:106BA0003DE7052205AB01091A7089B2420F890041
:106BB00022408A1A11125A709970642A00DD6422E8
:106BC0000421DA70081F824201DC04324FE7685C5E
:106BD00058540131F6E7002D00D020E753E7C046B6
:106BE000C4FCFFFF220300001AF6000070B502008B
:106BF0000024F0210D4E080060438019457895422D
:106C000003D001340A2CF6D170BDF022002107F028
:106C1000A1F9074A1368013BA34200D11460002385
:106C200029001A001120FFF76BFEEDE7041C00207D
:106C3000DC05002010B5B2B002236A4604001370D0
:106C400007F012FDC72800D9C7200023984207DCAF
:106C5000421C6B46FE211420FFF752FE32B010BDDD
:106C6000694601335A1EA25CCA54EFE7002310B5EF
:106C700001001A001120FFF743FE10BD07B56B4657
:106C8000197069465A7013128B701314120ECB7060
:106C90000A716B46010005221320FFF731FE07BD84
:106CA00010B50A0001001220FFF7A0FE10BD10B5BC
:106CB0000C000300110014202200FFF721FE10BD7C
:106CC000012370B5FF24084A41185B42884201D372
:106CD000D84370BD06781D0A234073409B009B5823
:106CE00001306B40F2E7C0463006010013B50400E6
:106CF000FE2813D80A4BC200D05800280ED0436893
:106D000008309900FFF7DCFF01900920FFF7F4FC41
:106D100001AB042221001720FFF7F2FD13BDC0468E
:106D200064250020F8B500231800254DDA00AA5884
:106D30000133511E8A418018FF2BF7D105244443AB
:106D40000A20FFF7D9FCFB20FFF770FC2720FFF794
:106D50006DFC0020FFF76AFCE0B22412FFF766FC2E
:106D6000E0B2FFF763FC174BFA21186804F0AEFF9E
:106D700000260700F300E85800281CD043680830BC
:106D80009900FFF79DFF04000520FFF7B5FCF0B266
:106D9000FFF74CFCE0B2FFF749FC2004000EFFF7C0
:106DA00045FC2002000EFFF741FC200EFFF73EFCE1
:106DB000380002F0ABF90136FF2EDBD1F8BDC0463A
:106DC0006425002004000020F7B50190FFF7A8FC1F
:106DD00001250400FF276D42002C01D12800FEBDD3
:106DE000266833143B40152B0DD121000198083142
:106DF00007F030FC002801D135123D402000FEF79D
:106E000069FD0400E8E71D2BF8D101256D42F5E787
:106E1000002010B5074C236883420AD0FDF7A6F87E
:106E200022680300904200D3831A0020024A9A424B
:106E3000404110BD88120020BFC62D0030B5B3B050
:106E40000500FFF7E5FF002816D002236A46280058
:106E5000137007F009FC0400C72800D9C7240023D9
:106E6000A3420BDB20003230FFF746FC621C6B466E
:106E7000FF211420FFF744FD33B030BD69460133D4
:106E80005A1EAA5CCA54EBE7F0B5BDB005900C00E1
:106E9000012803DC1B20FAF79FFC55E02C4B086807
:106EA0000393C30709D4042807D90F2302681340AA
:106EB000042B02D1FDF7E6FA0390254B606804939A
:106EC000C30709D4042807D90F2302681340042BF1
:106ED00002D1FDF7D7FA049000261E4B1B680893D9
:106EE000089BB3420BDC049B1B4A0093C821039B05
:106EF0000AA807F041FB0AA8FFF7A0FFCAE70C2584
:106F00007543164B0399ED18286807F0A3FB071E7D
:106F100005D16B68AD680993099B9F4201DB01367F
:106F2000DEE728680499079507F094FB083506907A
:106F300000280BD121000598079B08315B680238B7
:106F40009847074B069A1A603DB0F0BD0137E3E75A
:106F5000F7FB00009416002015060100FC2E00200F
:106F6000A40F0020F7B5234B06001B68F021009307
:106F70000023009A9A4211DC0024F0231A00624395
:106F8000019201991C4A55182F78002F12D0013414
:106F90000A2CF3D11948FFF751FF29E00A005A43A0
:106FA000154882185078B04202D11278002A1FD1B9
:106FB0000133DEE7F0223900280006F0CBFF022380
:106FC0000D4A0199EB6053540D4AF1008A58009B19
:106FD0006E70AE70AA602F616F61A34202DC054B38
:106FE00001341C60002331001A001020FFF788FCD8
:106FF000F7BDC046DC050020041C00205D0A01002E
:107000006425002010B5FFF7AFFCFF24084AE30019
:107010005B429B18074AD35C043B012B03D8E04337
:10702000C0B2FFF79FFF013C002CEFD110BDC0465E
:10703000FC07000064250020F8B505000E00FDF7F0
:1070400041FCFF240D4B18600D4AE3005B429B1886
:107050000C4AD35C062B01D0032B0BD1E743FFB2C4
:10706000320029003800FFF705FC002802D0380064
:10707000FFF778FF013C002CE6D1F8BD08000020A6
:10708000FC0700006425002070B50500FF24084AB5
:10709000E3005B429B18074AD35CAB4203D1E04359
:1070A000C0B2FFF75FFF013C002CF0D170BDC046BD
:1070B000FC07000064250020F7B5FCF757FF574B8D
:1070C0001A68824201D900221A601A685449821A49
:1070D0008A420DD9FF2253491860D3005248CB1A77
:1070E0001B181B78073B022B0CD9013A002AF4D15C
:1070F000F7BD0720FFF7C8FF4C4B27E00820FFF73C
:10710000C3FF38E0FCF73CFF071E00D10127002039
:10711000FCF7FCFF01900020FDF70CF8019B0090AC
:10712000434C444D002B12D02368002B6ED12B68AA
:107130002760002B6ED0404B01261B78002BD8D146
:107140000920FFF7A1FF394B1E703B4B1E70009BBF
:10715000002B12D02B68002B0FD123682F60002B3F
:107160001ED0324B01261B78002BC7D10920FFF718
:107170008BFF2E4B1E70304B1E702368002B0FD0E0
:107180002A4E3278002A0BD19F4200D22760236812
:10719000FB1A312B04D90720FFF776FF0123337048
:1071A0002B68002B0FD0244E3278002A0BD1BB4223
:1071B00000D92F602B68FF1A312F04D90820FFF760
:1071C00063FF012333702368002B0CD0019B002B3D
:1071D00009D1164E3378002B02D10720FFF754FF58
:1071E0000023236033702B68002B00D180E7009BC5
:1071F000002B00D07CE7104C2378002B02D1082014
:10720000FFF742FF00232B60237071E7009A002AEA
:10721000A0D1B5E7009B002B9FD1AEE784120020E0
:107220000F27000064250020FC07000078120020D2
:10723000741200207C1200208012002013B504007C
:10724000FFF792FBFEF721FE00230093134B1B6810
:10725000002B02D16846FCF741FF042301A901205D
:107260000193FDF77BFF00210800FDF731FFFEF7DA
:107270003FF9FFF7B3F9FCF771FFFCF7F5FFFDF7F6
:107280000FF8FEF77BFAFCF79DFE002C04D0FDF70B
:10729000A7F80348FFF7D2FD13BDC046B01A00207F
:1072A0004E0A010070B50D003235060028000C00B2
:1072B000FFF714FB002806D1FFF7AAFD002808D02D
:1072C0002800FFF719FA3300220000211B20FFF7E6
:1072D00017FB70BDF0B5A1B0FFF7F4F98021A94C00
:1072E000A94F2068C900091AC019FDF735F82368AD
:1072F000C0182060002811D0FCF738FEA34B18609E
:107300003B78FA2B00D04FE12368022B08DCFFF713
:10731000C5F9002802D00120FFF796F921B0F0BD91
:107320007B78BC78981E242800D91FE104F03AFC31
:10733000250038003C00400043004C001E01560070
:10734000880092009900AF00EE0005011E011E01A9
:107350001E011E011E011E011E011E011E011E0135
:1073600019011E011E011E011E011E011E011E012A
:107370001E011E011E011E019600FF2C0ED02000D2
:10738000FFF734FC0022824BE100CA505B181A71EF
:107390002100009213001320FEF714FD0320BBE729
:1073A0002000FFF7DFFDF9E72000FFF71FFCF5E7FE
:1073B000FFF728FEF2E7FFF7D7FA0020FFF73EFFBE
:1073C0007448FFF73BFDE9E7632CE7D8724BA20056
:1073D000D25821001520FFF709FBDFE7FFF7A0F9DE
:1073E000FF270400002CD9D025682B143B40152B17
:1073F00004D02000FEF76EFA0400F3E72000083006
:1074000007F032F906000530FFF776F9FB20FFF7A9
:107410000DF92D121D20FFF709F9E8B2FFF706F963
:10742000F0B2FFF703F93012C0B2FFF7FFF8250002
:107430002B1B9E42DDDD287AFFF7F8F80135F7E7D0
:1074400000211D2000910B000A00FEF7BBFCFCF799
:10745000C7FFA3E72000FFF749FC9FE7FFF762FCA7
:107460009CE7FCF79BFD07AC4C4A642100904C4B19
:10747000200007F081F802232000237007F0F4F8C1
:107480002300020000211620FFF73AFA86E7454B59
:10749000FA21186804F01AFC002604903C4AF30014
:1074A0009B181C68002C28D01B790593636808344E
:1074B0009F00B81D0393FFF71FF9FB20FFF7B6F8F5
:1074C00001207D1CFFF7B2F8F0B2FFF7AFF8E8B289
:1074D0002D12FFF7ABF8E8B2FFF7A8F80598FFF711
:1074E000A5F8E719A7420CD8FFF7ECF8049B03981E
:1074F000584301F00BFEFFF7E5F80136FF2ECDD122
:107500004CE72078FFF792F80134EBE70024FFF70F
:107510002BFA2300220021000094DA20FEF752FC0F
:10752000FF222100D2001A4806F014FDFCF758FF94
:1075300021002000FDF7CCFD30E7012C02D1FEF741
:10754000F3F92BE7022C02D1FEF738FC26E7032CD7
:1075500003D100210800FDF7BBFD0120FFF76EFEFF
:107560001CE7002321001A001A208DE71A00C83AF0
:10757000052A00D912E7002218001100F9F77AFF56
:107580000CE7C046981A00209816002088120020A8
:1075900064250020300A01005C2D0020470A01000C
:1075A000420A010004000020FB2B00D0B3E6226851
:1075B000042A00DCABE63E79F878614B36020643DC
:1075C0009E4200DDA7E6331D9A4200DC9FE6FB5C8D
:1075D000FE2B00D09FE67878BC78751E1B2869D0FA
:1075E0001AD807284FD0082824D0012819D1FF2CF9
:1075F00010D02000FFF7FAFA7D79524AB31E0092AC
:1076000021002A000A20FEF7DDFB4F4BE400E0508A
:107610001B191D71701D7FE61D285DD04FD31E28DC
:1076200071D00300C83B052BF4D8484A2900F9F76C
:1076300021FFEFE7632CEDD87A79022A13D0032AD1
:107640001BD0012AE6D1F979BB79090219433B7AAB
:10765000A4001B0419437B7A1B060B435B001343F6
:107660003B4AA350D6E7002DD4DDB11E3548FDF7C7
:1076700029F9374BA400E050CCE7BB79A4005A1E8F
:1076800093419B00ECE7632DC4DC07AF2A002F4930
:10769000380006F043FC002338007B55FFF794FBCD
:1076A0000028B7DB2A4B8000C25821001520FFF7C5
:1076B0009DF9AFE729002548FFF7BEFCAAE7FF2C9C
:1076C000A8D07A79022AA5D81E490B200091210062
:1076D000B31EFEF777FB9DE7632D00DD63250023D6
:1076E00007A99D420ADCEB430022DB172B40CB1895
:1076F0001A70152000916B1C2100EAE7FA185279E4
:10770000CA540133EDE7022C13D0032C14D0012C02
:1077100000D07FE7002D00DC7CE77B79002B03D0D5
:107720001C00322B00DD322464235C43094B1C60B7
:1077300070E7FEF7A9FB6DE7FEF7A7FB6AE7C04617
:10774000F60300009E160020642500209D160020F0
:107750005C2D0020040000200120704710B5064C6D
:10776000200001F03FF90549200001F06FF90122E6
:10777000034B1A6010BDC046D41A0020801A0600C0
:107780009C1A00201FB500211020FCF70DFC0121E0
:107790001620FCF709FC01211120FCF705FC1C4C0C
:1077A000200001F07DF81B4B1B4A1B6812681B4927
:1077B000D2B28B420BD880239B04019301AB1A7188
:1077C0000199029A0023200001F086F81FBD144998
:1077D0008B4202D88023DB04EFE712498B4202D8A8
:1077E00080231B05E9E710498B4202D880235B0503
:1077F000E3E70E498B4202D880239B05DDE70C4965
:107800008B4202D88023DB05D7E780231B06D4E711
:10781000B41A0020340000203000002048E80100A5
:1078200090D0030020A1070040420F0080841E007A
:1078300000093D0010B5002815DD01240B68234226
:1078400011D023410C4A13600C4AA04209D04B6866
:10785000234206D02341022B09D0032B09D0A34297
:1078600003D002231360002010BD0023FAE7032396
:10787000F8E71460F7E7C04634000020300000202D
:1078800070B5002812DD0C68E3070FD56410012CD9
:107890000CDD074D2B68002B01D1FFF75FFF2B6834
:1078A000002B03D02100034801F0D0F8002070BD68
:1078B0009C1A0020D41A0020F8B501250868284237
:1078C00003D10D20F9F788FFF8BD4010FCF790FBBD
:1078D000041E14DBFCF766FBA04210DB0221200033
:1078E000FCF762FBFA222900D200200001F040FCE4
:1078F0000025A84205D101002000FCF755FB00201F
:10790000E2E700270726FA2201219200200001F079
:107910002FFC0028F3D0282802DD0123B3401F43A9
:10792000013EF0D20E4EAF550135052DE9D10021B3
:107930002000FCF739FB012206210920FCF744FF57
:107940000028DCD00B23012443600023F25C990063
:1079500052004118224301338A60052BF6D1B3E768
:10796000A01A002070B500281EDD0D68EB071BD49F
:10797000042D19D90F242B681C40032C14D11A098B
:1079800092B25B0F92001C40141B2E00FFF7FAFE10
:10799000731B06489C4205DD317900F0A3FF0136D8
:1079A000F070F5E700F09DFF002070BDB41A0020D4
:1079B00010B504680D20E30703D56410FF2C03D92C
:1079C0001720F9F709FF10BDFFF7DCFEE1B2044C08
:1079D000200000F087FF200000F083FF0020F2E786
:1079E000B41A002070B5FFF7CDFE064D0021280027
:1079F00000F078FF0400280000F073FF012064000D
:107A0000204370BDB41A0020A02101220B4BC900F5
:107A10005A500B480B4958500B491A604A68002AC3
:107A2000FCD000224A60A121C900585801215960A8
:107A3000A021C9005A50054BC01870470070004083
:107A40006A10000004050000FC700040FBFDFFFF11
:107A500010B5FFF7D9FF43000120184310BD000007
:107A600010B5034A0F210348FEF76CFE10BDC04657
:107A7000740A0100EC0A0100F8B50E4F04003B68DF
:107A80000E001500002B01D1FFF768FE3B68002BAC
:107A90000FD0E1B2084C200001F06FF8F1B22000E5
:107AA00000F06CFFE9B2200000F068FF200001F058
:107AB000CFF8F8BD9C1A0020D41A002010B501247C
:107AC0000368234205D04168214202D082682242E5
:107AD00003D10D20F9F780FE10BD5810802801D980
:107AE0001520F7E74910FF2901D91620F2E75210B7
:107AF000FF2A01D91720EDE7FFF7BEFF0020EBE7D3
:107B000010B5002803DC1C20F9F766FE10BD0B68D9
:107B1000DA0701D40D20F7E75B100322012B06DD05
:107B20000522022B03D00C22042B00DC08220F219B
:107B30001820FFF7A1FF022001F0E8FA0020E5E796
:107B4000F7B5012203001000934211DD0E683242A6
:107B50000ED0394D16412B684C68002B01D1FFF730
:107B6000FDFD2B68002B04D12320F9F735FE002002
:107B7000FEBDF1B2314E2700300000F0FEFF0122C1
:107B800017400FD01441FF2C02D91720F9F724FE1B
:107B9000E1B2300000F0F2FE300001F059F80028A8
:107BA000E6D0E1E7042CF7D90F2523681D40092D05
:107BB0001CD1636801925B100093009BBB42EBDD1C
:107BC000BB00E3189D68019B1D420BD06D10FF2D7B
:107BD00002D91720F9F700FEE9B2300000F0CEFE1E
:107BE0000137EAE71720F9F7F7FDF9E7032D0FD181
:107BF00027001A0992B25B0F92001D40551B3B1BD8
:107C00009D42C9DD3979300000F0B8FE0137F6E752
:107C1000042DC1D12000FCF735FC0500200006F042
:107C200023FD2C000700631B9F42B5DD2178300047
:107C300000F0A4FE0134F6E79C1A0020D41A0020BC
:107C400070B5174C050023680E00002B01D1FFF71B
:107C500085FD2368002B21D0124CEDB229002000B5
:107C600000F08BFFF1B2200000F088FE0021200020
:107C700000F08EFF002801D040420EE072B60122D3
:107C80002900200000F074FF62B6200000F067FEBB
:107C9000002802D0200000F067FE70BD6420EBE7F2
:107CA0009C1A0020D41A002010B501240368234236
:107CB00002D04168214203D10D20F9F78DFD10BD9E
:107CC0005810802801D91520F7E74910FF2901D95C
:107CD0001620F2E7FFF7B4FF40002043EFE7000073
:107CE00070B5284D04002B68002B08D10521182001
:107CF000FFF7A6FF022001F009FA01232B60012CF7
:107D000014D105211820FFF79BFF7F282BDC0300EF
:107D10007F3301DA7F204042C8235B4258437F21F2
:107D200003F0D4FF052C00D1404270BD032C11D1CB
:107D300021001820FFF784FF7F2814DC03007F3325
:107D400001DA7F204042C8235B4258437F2103F081
:107D5000BDFFEAE70020052CF5D107211830FFF719
:107D60006FFF7F2802DD0138FF38D0E703007F3343
:107D700001DA7F204042C8235B4258437F2103F051
:107D8000A5FFD1E7A81A002010B50120FFF7A8FF32
:107D900043000120184310BD10B50320FFF7A0FFDA
:107DA00043000120184310BD10B50520FFF798FFD0
:107DB00043000120184310BD10B508211820FFF71B
:107DC0003FFF0300C00FC0180123401015304000D2
:107DD000184310BDF8B5514B05001B68002B01D1AD
:107DE000FFF7BCFC4E4C23787F2B00D892E0072194
:107DF0000E20FFF725FFC42833D101220E26494B60
:107E000010211A70484B30001A702670FFF734FEAC
:107E1000802211213000FFF72FFE0021615600293A
:107E20001EDB424EC9B2300000F0A7FE3D4B3000D1
:107E3000197800F0A3FD300000F00AFF2178062237
:107E4000300000F095FEAC1D300000F088FD0028E9
:107E500006D0300000F088FD28700135A542F3D12E
:107E6000F8BD0F211920FFF7EBFE33280FD1682250
:107E70002C4B1E261A7000222B4B60211A703000EA
:107E80000C322670FFF7F8FD02226121C2E70021C3
:107E90001820FFF7D5FEFA281CD14222214B1026CC
:107EA0001A700022204B4B211A70300001322670CC
:107EB000FFF7E2FD042001F029F938224C213000BF
:107EC000FFF7DAFD0F2251213000FFF7D5FD1B220D
:107ED00052219FE70F211C20FFF7B2FE3D289CD1C5
:107EE00028221C2600270F4B20211A700E4B263A01
:107EF00030001F702670FFF7BFFD3A0022213000CE
:107F0000FFF7BAFD3A0023213000FFF7B5FD40220C
:107F100024217FE70021615683E7C0469C1A002098
:107F2000380000203A00002039000020D41A002038
:107F300073B5002606220021684606F00BF8684655
:107F4000FFF748FFFFF7C6F91A4B6A469E576C4683
:107F50006B4691781878D5785B7812796479002E21
:107F60001FD000020902034329431BB209B21202C7
:107F700011482243007812B240B2102802D15210A8
:107F8000DB10C910D8171B184340C8170918414007
:107F900001205918D317D2185A408A18520010439A
:107FA00076BD1B022D02034329431BB209B22402F2
:107FB000DEE7C0463900002038000020F7B5012870
:107FC00001DC0120FEBD01250B6801932B42F8D096
:107FD0004E683540F5D1042EF3D90F233268134093
:107FE000092BEED173685C10002CEADD174F3B685B
:107FF000002B01D1FFF7B2FB3B68002BE1D0202C16
:1080000000DD202472B6019B114F5910C9B2220025
:10801000380000F0ADFD62B6380000F0A0FC00288A
:1080200003D16D0001302843CCE7380000F09CFC00
:108030000122AB004000F3181043AD189860A54230
:10804000EADB944010002043BCE7C0469C1A0020A5
:10805000D41A002070B52B4B86B01B68002B02D1C0
:108060000120FFF73DFE01AD14220021280005F09C
:1080700071FF254E1821300000F07FFD03213000F4
:1080800000F07CFC0021300000F082FD041E13D1C2
:1080900072B605221821300000F06AFD62B6300089
:1080A00000F05DFC002802D0300000F05DFCA30071
:1080B0000134E850052CF2D1019B7F2B01DD013BFF
:1080C000FF3BAA687F2A01DD013AFF3A29697F292F
:1080D00001DD0139FF39C820434342434843DB11E6
:1080E000D2115243C0115B4340439B18181805F04E
:1080F000FDFD01F051FD05F0C3FD430001201843D3
:1081000006B070BDA81A0020D41A002010B5054C86
:108110002368002B02D01B20F9F75EFB00202060B3
:1081200010BDC046AC1A002010B5002803DC1C208E
:10813000F9F752FB10BD0B68DA0706D4042B04D9FB
:108140000F221B681340032B01D02420F0E7034BC0
:1081500025201B68002BEBD01B20E9E7AC1A002080
:1081600010B5002803DC1C20F9F736FB10BD0B68A6
:10817000DB0701D40D20F7E71B20F9F72DFB0020CA
:10818000F4E700001D4B70B51B680C00002B03D1F9
:108190002520F9F721FB70BD012801DC1C20F8E740
:1081A00008680121084207D1042805D90F23026875
:1081B0001340DD1E8D4201D92420EAE765680D4297
:1081C00001D11120E5E7042B0BD1FCF75BF906F098
:1081D0004BFA63685B10013B01D4834208DB122039
:1081E000D7E7100980B252008000920F801AF0E7A2
:1081F0001B20F9F7F1FA0120CDE7C046AC1A0020A8
:1082000010B50400802803DD2620F9F7E5FA10BD3B
:10821000002CFCDD1B20F9F7DFFAFEF74DFFFFF71E
:1082200059F8012000F072FFF2E7000010B50028B5
:1082300005DC1C20F9F7D0FA0400200010BD184B13
:108240001B68002B01D12520F4E7012408680440B5
:108250000FD04010FF2801D92820EBE71B20F9F7A9
:10826000BBFAFEF729FFFFF735F8012000F04EFFBB
:10827000F4E70428E1D90F2102681140042906D14E
:10828000FCF700F906F0F0F9FFF7BAFFD5E703298C
:10829000D3D1100980B2520F80000A40801AF3E750
:1082A000AC1A0020044B10B51B682520002B00D011
:1082B0001B20F9F791FA10BDAC1A002010B5034A43
:1082C00006210348FEF73EFA10BDC046980B010098
:1082D000C80B010000207047012070470020704744
:1082E0000020704701207047002070470020704731
:1082F0000020704700207047002070470020704722
:108300000020704700207047002070470020704711
:10831000002070470020704700207047704770476A
:108320007047704710B5034A12210348FEF70AFA56
:1083300010BDC046E80B0100780C01000378013B3A
:108340001F2B00D970470130F8E710B5FFF7F6FF93
:108350000378002B0BD00130222B11D10378002B96
:1083600003D0421C222B03D11000FFF7E7FF10BD02
:108370005C2B03D14378002B00D0821C1000EDE76A
:108380003A2BF2D02C2BF0D07B2B0BD1FFF7D6FF62
:108390000378002BE9D07D2B01D10130E5E7FFF711
:1083A000D4FFF5E720225B2B14D1FFF7C7FF03783A
:1083B000002BDAD05D2BF0D0FFF7C7FFF7E7202BBB
:1083C000D3DD2C2BD3D0190091435D29CFD0222BA4
:1083D000CDD001300378002BF1D1C6E7002210B5D3
:1083E000904216D0FFF7AAFF03780422222B10D068
:1083F000023A7B2B0DD0013A5B2B0AD019003039A1
:108400000232092905D92D2B05D1417830390929A6
:108410000AD8100010BD0522742BFAD00132662B49
:10842000F7D001326E2BF4D0581E83415A42F0E748
:1084300070B5FFF783FF037801222D2B01D180183F
:10844000023A00230A2502E06B430130CB18017881
:108450003039CCB2092CF7D95A43100070BDF8B5A9
:108460000C001500FFF76AFF0378222B02D00023CF
:108470002370F8BD0D236A1E210008250C260A274B
:108480009C4601300378222B02D100230B70F0E7C9
:10849000002BFAD0441C5C2B0BD14378841C622B3C
:1084A0000ED0662B0ED06E2B0ED0722B0ED0742BEE
:1084B0000ED0002AE9DD0B70013A01312000E1E71E
:1084C0002B00F6E73300F4E73B00F2E76346F0E702
:1084D0000923EEE710B50400FFF737FFA04203D9E8
:1084E0000378013B1F2B00D910BD0138F6E710B50A
:1084F000002815D00378002B13D0FFF71FFF202191
:10850000037802008B4300205D2B09D01000FFF799
:108510001CFF03782C3B5A425341C018FFF70EFF53
:1085200010BD1800FCE70300002070B50C0081426C
:108530000EDD1A785B2A0BD1581CFFF7FFFE0125D0
:10854000AC4205D0FFF7D3FF002801D00135F7E793
:1085500070BD70B50C001500002901D000230B7010
:10856000002820D00378002B1ED0FFF7E7FE037809
:1085700006002C2B03D10130FFF7E0FE0600337814
:1085800000207D2B0FD0844204D02A00210030002F
:10859000FFF765FF3000FFF7D8FE03783A2B02D1D2
:1085A0000130FFF7CBFE70BD1800FCE7F0B50D0001
:1085B00004009DB02E78002E35D02E21280006F024
:1085C0003BF8071E14D0431B0193303E092E14D8EC
:1085D0002800FFF72DFF01002000FFF7A4FF040093
:1085E000002C20D0002F1ED0019B0133ED18E1E7B5
:1085F000280006F039F80190E7E723787B2B11D1AA
:10860000601C642203A9FFF7A4FF041E0BD0019A8B
:10861000290003A806F02FF80028E1D02000FFF77A
:1086200094FEEEE7002420001DB0F0BD70B50500FB
:1086300000200C0081421DDD2800FFF7CFFE030063
:10864000681C012B14D00020022B13D10022681CBF
:108650001100FFF77EFF012C0CD0FFF748FF00222E
:108660001100FFF776FF013CF5E7FFF740FF013C03
:10867000012CFAD170BDF8B5050000200C001600E1
:108680001F0081420DDD2800FFF7A8FE0300002037
:10869000022B06D1681C3A003100FFF75AFF012C6B
:1086A00000D1F8BDFFF723FF3A003100FFF751FF7B
:1086B000013CF4E710B50024A04218D0FFF73EFEBD
:1086C00003787B2B0AD1013000221100FFF741FF14
:1086D00000280CD0FFF739FE0134F5E75B2B06D1FB
:1086E0000130FFF704FF002801D00134F9E7200032
:1086F00010BDF8B5002816DD0D68EB0713D56D1019
:10870000013D0124FDF7F2F90026FF27644200280D
:108710000CD1002E21D0300005F0A6FF0100300062
:10872000FCF7D0F8F8BD01256D42EAE703681A149A
:108730003A40152A0BD11B123B409C4200DA1C0028
:108740009D4201D106000836FDF7C4F8DFE71D2A77
:10875000FAD1012400266442F6E7012001346400C6
:108760002043DFE710B508680C00FBF78BFEFEF72F
:108770002BFB002803DB6268024B8000C250002004
:1087800010BDC0465C2D002010B50868FBF77AFECE
:10879000FEF71AFB0123002802DB024B8000C358BE
:1087A000180010BD5C2D002010B50868FBF76AFEAC
:1087B000FEF70AFBC043C00F800010BD10B5034A8E
:1087C00004210348FDF7BEFF10BDC046380D01006F
:1087D000320D010010B5FBF777FDFBF725FEFEF724
:1087E0001DF80448FEF72AFBFDF7DEF9FEF70AFC48
:1087F00010BDC046870D010010B5FBF79BF810BDFA
:1088000070B5002504AC24780573A94205D10A4B44
:108810000A4A25210A4805F013FB01600949920024
:1088200052589B0002715B58A400837163588560A5
:1088300043710223C37170BD9F0D0100FE0D010045
:10884000AD0D01005C0E0100037B002B04D14373CE
:108850008373036101330373704700001FB50191F7
:10886000A02100240068C900D2B24450012A10D0CF
:10887000A24209D0032A0AD0074A8350074B019A23
:10888000C250012343501FBD02221343F4E70422C8
:10889000FBE70622F9E7C046540500002405000066
:1088A00010B50400FFF7D0FFA1222368A179D20000
:1088B00099506179064A20009950217904329950E3
:1088C000044B19685A689B68FFF7C8FF10BDC04683
:1088D0000C050000C81A00201FB5FFF7BFFF05B048
:1088E00000BD70470368074A99501A00FC32D168EE
:1088F0000029FCD0A321C90058580023C0B2D3607E
:108900007047C0461C05000007B58022074BD20502
:108910001A6000229A6002321A7111230E320093FB
:10892000034905330348FFF76BFF07BDC81A002052
:1089300000300040B41A0020F8B505000E00170002
:108940000024BC4208D02B68315D1B682800984782
:10895000002801D00134F4E72000F8BD704710B5BD
:108960001C3000F0AFF910BD10B51C3000F09CF9C0
:1089700010BD10B51C3000F0ABF910BD70B5437ED2
:108980000D00002B01D1002070BD6430040000F008
:10899000A8F90028F7D12000290000F076F901207D
:1089A000F2E70000F7B50193FA23002504009B00CD
:1089B00083600B4B4560083303601C300F001600CA
:1089C00000F058F92000643000F054F96B461B7930
:1089D000276166756576A5762000A375FEBDC04645
:1089E0003C0E0100012330B5A024C375837D1349DB
:1089F0009B005A58437DC132114DFF32E40592006D
:108A00009B005B581551CC22C133FF339B001D5195
:108A100004690C4B5204E25005220469243BE250E5
:108A2000837D04699B005A58A123DB00E250437DFB
:108A300002699B005958044BD15030BD5C0E0100B7
:108A40000C060000240500000C050000A0220023F5
:108A500010B50469D200A3500A4CA1420FD90A4CA8
:108A60008C425B4109495B420B40CD21C9045B1834
:108A700004690749635005210369995010BDCC234F
:108A80005B04F5E7A086010090D00300000098FD8C
:108A900024050000F7B5040000200D000193824278
:108AA00065D01600402A00D9402627001C37380020
:108AB00000F0F6F8B1232269DB00D55080220123B3
:108AC000216992008B50A27E002A03D12269136291
:108AD000226913600025731EAB4207D1019B002B56
:108AE00004D0802202212369920099500122236937
:108AF0001A622369FC33DA68002A02D19A6A002AD2
:108B0000F9D09A6A002A0BD1DA60A3232269DB002C
:108B1000D1583800C9B2013500F0B7F8B542DAD300
:108B2000019B2269002B0FD11300FC339B6A002BA1
:108B30000AD10133A376D3612369FC33DA6C002AAE
:108B4000FCD00022DA640AE000230121A3765161FF
:108B50001A002369FC3399680029FCD09A602369C4
:108B6000FC339A6A002A01D000229A62E8B2FEBD64
:108B700010B50123FFF78EFF10BD0300AC3310B515
:108B800004001970643000F08BF80123637610BD87
:108B90000023020070B5AC3243760D001178B1228B
:108BA00004000069D20081508022216992008B501C
:108BB0002269013313622269936026006436300013
:108BC00000F080F8002812D0300000F06DF81E4B45
:108BD0002269D0502369FC331A6A002A02D19A6AAA
:108BE000002AF9D09A6A002A01D11A62E5E72369BE
:108BF0000122002D0DD11900FC31896A002908D10C
:108C0000DA612369FC33DA6C002AFCD00022DA64D2
:108C100007E05A612369FC339A68002AFCD00022DD
:108C20009A6000202369FC339A6A82420BD09862D2
:108C30002169064A8B588B501800022B03D0181F4D
:108C4000431E9841033070BD1C050000C4040000A1
:108C500010B50121FFF79CFF10BD000010B51323D4
:108C6000122202490248FFF79DFE10BD004000405D
:108C7000D41A002010B540220021040005F06AF942
:108C8000002320002364636410BD10B53F24026CF0
:108C9000531C2340446C9C4201D08154036410BD9A
:108CA0000023036443647047436C026C934206D014
:108CB0003F21C25C01330B40436410007047012028
:108CC0004042FBE7036C406C181A00D540307047F7
:108CD000436C026C934201D0C05C7047012040425B
:108CE000FBE73F22036C406C01331340181A4342E8
:108CF0005841C0B27047000003210A4802680A4385
:108D00000260094802680A4302600849084A094BA0
:108D10009B1A03DD043BC858D050FBDC00F012F86E
:108D2000F7F7F2F92405004054050040A8130100AC
:108D30000000002074020020FEE7FEE7FEE7FEE7E9
:108D4000FEE7FEE7014B024A1A6070473C00002034
:108D50000024F4000120704710B503681322DB697A
:108D6000984710BD70470000054B0269D150036958
:108D7000FC331A6A002AFCD0002201201A627047D4
:108D80001C050000030010B55C331A781F231A403D
:108D90001E3B19009140114AD167C2220421046987
:108DA0009200A150026953600269D360A02300229F
:108DB0000169DB00CA5001230169094A5B428B50FB
:108DC0000169084A8B5001690C3A8B5001690832DD
:108DD0008B501430FFF764FF10BDC04604E100E083
:108DE0000C0500001405000010B51430FFF76AFFF1
:108DF00010BD10B51430FFF76BFF10BD10B5143067
:108E0000FFF752FF10BD0000030070B55E331A7803
:108E10000469724BE25003005D331A780469704BA9
:108E2000E250030061331C7802696E4B012C00D0C4
:108E30009EE005005F352E78A225ED005651020018
:108E400060321578A1220669D200B5500269D4506B
:108E50009623DB00994200D88CE096231B019942AF
:108E600000D88AE096235B01994200D888E09623D7
:108E70009B01994200D885E0E1239B01994200D8EB
:108E800082E09623DB01994200D880E0E123DB01F8
:108E9000994200D87DE096231B02994200D87AE0DF
:108EA000E1231B02994200D877E096235B029942A6
:108EB00000D874E0E1235B02994200D871E0E1231D
:108EC0009B02994200D86EE0474B994200D86CE073
:108ED000E123DB02994200D86AE0E1220023120379
:108EE0008A425B41414A5B421340802252059B18F3
:108EF00001693F4A8B50A02304220169DB00CA505C
:108F000000210369FC33D9600369FC331962012332
:108F100001690B6001698B60C1210469890062509D
:108F20001F215C3002780A4093406231314AFF31A0
:108F300053500021415600293CDA0F230B40083BD7
:108F40002D4C9B089B001B1903242140A140FC349D
:108F50008C40DD69A5432C00C0258D4029002143AC
:108F6000D9611F23017819401E3B8B40136070BDEF
:108F700000246CE79E23DB02BAE79D231B03B7E7BF
:108F80001E4BB5E71E4BB3E7EC239B03B0E71D4B2D
:108F9000AEE71D4BACE71D4BAAE71D4BA8E71D4BE9
:108FA000A6E71D4BA4E71D4BA2E78023DB049FE748
:108FB0001B4B9DE78C080F4BA400E41803230B40C8
:108FC000FF21C025DB009940AD0066598E4331007A
:108FD000C0269E4033000B436351C2E70C050000DE
:108FE000140500006C05000090D0030000D0BEFE08
:108FF0002405000000E100E000ED00E000B01300F7
:109000000050270000A04E0000F0750000509D00A9
:1090100000F0EB0000903A0100E0D70100B0AF0390
:1090200000705F07F7B5009308AB1B78002501932C
:10903000FA2304009B0083600E4B456008330360F5
:1090400014300F001600FFF715FE23005C33276174
:109050001E70009B084A9B00995823005D331970CD
:10906000019B20009B009A5823005E33DD701A702C
:10907000FEBDC046D80E01005C0E0100036910B5AC
:109080001A00FC32D2680400002A0AD0A322D200BF
:1090900099581430C9B2FFF7F8FD00222369FC3358
:1090A000DA6010BD10B50248FFF7E8FF10BDC046FA
:1090B0008C1B00201D2307B50222009302490133B7
:1090C0000248FFF7AFFF07BD002000408C1B0020C7
:1090D00010B5002801D005F0F9F910BD0849094A7A
:1090E000094B10B51B688858FA22190A1B06184349
:1090F0009200002302F022FF4904C00B084310BD78
:109100000010014004050000F01B002070B5041E93
:1091100009D0FFF7E3FF050000F014F8FFF7DEFFCA
:10912000401BA042F8D370BD0022044B9A60044A51
:1091300013680133DBB213607047C046FC10014076
:10914000F01B00207047704710B500F05FF8FFF784
:10915000FAFF0120FFF7DAFFFFF73CFBFFF74CFBBC
:10916000024B002BFAD000E000BFF7E70000000040
:10917000F8B54C1EA1410125104B114F8000C3587A
:109180004C4238680F499D40160002F015FD0A2137
:10919000704302F011FD2C400300220029000A4810
:1091A00000F016F8FA21094C89004443386802F0AF
:1091B00003FD0100200002F0FFFCF8BD5C0E010081
:1091C0003C00002040420F00100500501027000016
:1091D00030B504680C40944206D1013B002BF8D115
:1091E00012E0013B002B0FD004680C409442F8D1F0
:1091F000002405680D40954204D101349C42F8D109
:10920000002002E0201C00E0181C30BDC420114BDF
:1092100080001A5810491140C02212020A431A5005
:10922000C0218022490092025A501A608023A32252
:109230000021DB05D20099500122F9309A60074BDA
:10924000FF301950C12002318000195040301950B0
:109250001A60704700E100E0FF00FFFF00100140CE
:10926000014B18607047C04688000020F7B5002306
:109270001E285AD8384B8000C258042A5BD007D821
:10928000022A54D055D80423012A09D000234CE0E7
:10929000062A54D051D31A2A53D002231B2AF5D1BF
:1092A0002E4A116808294ED909294FD00A240226CE
:1092B000A02001252A4AC00015502A482A4D0768D7
:1092C0001C20BF00074029480197006857590090AB
:1092D00027481B0207401F43C02300989B020340FE
:1092E000FF2057515759000207401F43019B1F435E
:1092F000009B58016023184007433E435651012507
:109300001C4B156058680028FCD000205860A12331
:109310000125DB00D3585560A025ED0050511BB24C
:10932000A14202D015D2611ACB401800FEBD08231D
:10933000B6E71023B4E72023B2E74023B0E7802349
:10934000AEE70123ACE708240026B1E70C000126B4
:10935000AEE7091B8B40E8E75C0E010084000020AB
:109360000070004040000020040500004400002080
:10937000FF00FFFFFC700040F0B51E285BD8364BA5
:109380008000C258354B1E68002E30D1C227344BA6
:10939000BF00D859334C03250440C02000022043AD
:1093A000D851C02480206400800018512E4F1860CE
:1093B0002E4B803CD859FF3CA043D8510437D85994
:1093C000A8432043D8510837D8590C35A8438446C0
:1093D000072065462843D851A820C0001E50C12050
:1093E0008026800076021E501C601C4B1C601425D9
:1093F00000202B001E4C2E0046433659771C1BD1F3
:109400004343E250A0230325C132FF329200DB0523
:10941000D550184B1A68082A14D114234343E31873
:109420009A6812485132FF32920059601150DA683E
:10943000C1239B00C250F0BD9642E1D00130032809
:10944000D9D1F8E7082A02D9083AD140E5E708233C
:109450009A1A9140E1E7C0465C0E0100F41B00201F
:1094600000E100E0FF00FFFF040500000090004065
:1094700048000020880000202149F0B54A6C2148AE
:10948000002A14D0A025A12600230124ED05F60012
:10949000C258571C06D0C7187F68002F02D027007B
:1094A0009740AF5114333C2BF2D100234B64A023DF
:1094B0000121DB0500260F009C4614234B43C318F3
:1094C0001A1F1268104C0E4D920014195219526C4A
:1094D000002A10D01A00143A1268551C09D0103B0B
:1094E0001B68FF2B05D03B00934065461A00074BD5
:1094F000EA50FC34666401310429DED1F0BDC04677
:10950000FC90004048000020009000400C05000046
:1095100000B51E2810D80C4A8000835803290BD8A8
:10952000A0220800C133FF33D2059B0002F030FBBC
:10953000020905070021D15000BD0C21FBE70421E1
:10954000F9E70321F7E7C0465C0E01001E280AD8A0
:10955000074B8000C25801239340A022D205002966
:1095600002D1044953507047A121C900FAE7C0460F
:109570005C0E01000C050000030000201E2B0AD821
:10958000A021A222C905D2008858034A9B009B58FB
:10959000D8400123184070475C0E0100F7B5060063
:1095A0000D000C008B180193019B671B9C4207D098
:1095B000336821781B683000984701340028F3D1C4
:1095C0003800FEBDF0B5C64600B5CB0F9846404A00
:1095D0004B005B0D9A1882B00D000400132A2FDC9B
:1095E000002A49DB3B4F17413E000E40064323D083
:1095F0007F08390029400C430AD03749BD438C46C7
:1096000063445C425C418023DB021341E4071D4359
:109610004146CE0031492B008E192200346875680E
:109620002000290002F030FE00900191009801997D
:1096300022002B0003F0C0FF02B004BC9046F0BD36
:10964000332A08DD8023DB009A42F5D102000B00AB
:1096500002F01AFEF0E7224A944601226344524285
:10966000DA400242E8D052080242D1D0944380222C
:10967000D2051A411443CBE74B005B080343DBD010
:109680000B031B0B1C436342234380244D0C240318
:109690001B0B23406D042B4319004346DA000F4B8C
:1096A0009B181C685D6802000B002000290002F076
:1096B000EBFD009001910098019922002B0003F02E
:1096C0007BFF42464B005B08D60733431900B3E7E4
:1096D00001FCFFFFFFFF0F00EEFBFFFF080F010083
:1096E000EDFBFFFFF8B5274A4B005B0D9A180C0005
:1096F0000700132A10DC002A36DB234B13410B42F0
:109700003AD0802424031441002064189C430600AE
:10971000250030002900F8BD332A0EDD8023060025
:10972000DB000D009A42F4D102000B00380021004A
:1097300002F0AAFD06000D00EBE7144D0600AC4652
:10974000012563446D42DD40AC4663460D00034293
:10975000DFD033239A1A323B93401818874200D93E
:109760004C1C63469843D2E7C90FCC070020531C1A
:10977000CDD1074B1C43CAE706000D000028C0D11D
:10978000C7E7C04601FCFFFFFFFF0F00EDFBFFFF37
:109790000000F03F30B5214A4B0087B05B08934290
:1097A0001EDD1F4A934205DD02000B0003F004FF9B
:1097B00007B030BD02AA00F0B5FF03231840049A99
:1097C000059B012813D002281DD0002814D0029830
:1097D000039901F08FFA80231B069C466144E7E75A
:1097E000002300220093002301F0FEFFE0E702982F
:1097F000039901F07FFADBE70124029803990094B2
:1098000001F0F2FFD4E7012402980399009401F0DB
:10981000EBFF80231B069C466144C9E7FB21E93F1F
:10982000FFFFEF7FF0B557464E46DE464546E0B5B2
:109830008FB01D0006000F00140000F00DFACE4B93
:10984000009001919A461B785BB2994601333ED055
:1098500022002B002000290004F0F6F9834600289E
:1098600035D132003B003000390004F0EDF9002220
:109870000390002800D06FE000233000390002F090
:109880002FFB00282CD0002200232000290002F00A
:1098900027FB8346002800D192E004AB98460123C1
:1098A00042460493B54B53604346039A1C615D6185
:1098B0001A629E60DF604246002300249361D461F7
:1098C0004B46002B67D00023AD4C009301940098C9
:1098D00001990FB03CBC90469946A246AB46F0BDFC
:1098E0000098019902F036F88146002800D19AE0EC
:1098F000009801990022002302F0F2FA0028E6D035
:109900003000390002F026F80028E0D020002900BD
:1099100002F020F80028DAD004AB9846042342462F
:109920000493964B14615561536000230024136225
:1099300000239361D46153461B789660D7605BB275
:10994000022B04D0404602F0ABF8002829D104F0E5
:1099500095FA2223036024E000232000290002F06E
:10996000BFFA0028B3D004AB9846012342460493C3
:10997000824B4146536043465A461A6200229E601B
:10998000DF601C615D617E4B8A61CB610092019357
:109990004B46022B9BD0404602F082F8002800D1B3
:1099A0008AE043461B6A002B04D004F067FA434662
:1099B0001B6A03604346DC699B690093019486E758
:1099C0002000290001F0C6FF002800D17FE7002217
:1099D00000232000290002F089FA002800D176E750
:1099E00004AB9846012342460493644B53604346BC
:1099F0005A469E60DF601A621C615D6153461B78A7
:109A00005BB2002B5DD0002042465E499061D1617F
:109A1000022B5BD104F032FA2123036043461B6A18
:109A2000002BC7D0C1E73000390001F093FF0028B8
:109A300000D15DE72000290001F08CFF002800D153
:109A400056E70098019953461B7802005BB29B468B
:109A50000B0004F0F9F804AB9846002862D1032308
:109A600042460493454B1461556153601062966001
:109A7000D760454B20002900002203F02BFB5B46FA
:109A800004000D00002B27D1E02241463F4B120677
:109A90008A61CB61300000220023390002F026FAEF
:109AA00000282AD1404601F0FBFF0028B6D104F07F
:109AB000E5F922230360B1E704F0E0F92123036014
:109AC0006FE74246002300249361D461404601F0D1
:109AD000E7FF0028A2D19DE7002241462C4B300031
:109AE0008A61CB6100220023390002F0FFF90028CF
:109AF00035D15B46022BDAD0D4E720002900FFF7EE
:109B000061FD22002B0002F0EBF9002805D1E022D4
:109B1000204B120641468A61CB6153461B785BB2EB
:109B20009B46E6E7012342460493144B53604346A9
:109B30004A469E60DF601A621C615D615B46002BD5
:109B4000BFD0002300221900100002F0B9FE4346E6
:109B50009861D9615B46022B00D15BE7B6E7200034
:109B60002900FFF72FFD22002B0002F0B9F9002891
:109B7000D3D10022034BCDE78C000020180F010049
:109B80000000F03F0000F0FF0000E03FFFFFEF4764
:109B90000000F07FFFFFEFC7F0B54746CE4680B527
:109BA0008DB004000D0000F0CDFF294B06001B789E
:109BB0000F005BB29846013310D022002B0020002A
:109BC000290004F041F88146002807D10022002333
:109BD0002000290002F08AF9002806D1300039005F
:109BE0000DB00CBC90469946F0BD01230293194B71
:109BF0000694079503934B460A93434604940595B0
:109C0000002B15D0002300221900100002F058FE8E
:109C1000434608900991022B0ED104F02FF921231D
:109C200003600A9B0193002B0CD1089E099FD5E786
:109C3000002300240893099402A801F031FF0028B2
:109C4000EFD1EAE704F01AF90A9B01930360ECE70D
:109C50008C0000201C0F0100F0B55746DE464E4632
:109C600045465C006408E0B598461F00230093B0A9
:109C700083468A46160013430CD07D4B4D0002915B
:109C800081466D089D4212DD7A4B9C465B466544D9
:109C90001D4361D10023784C0093019400980199F1
:109CA00013B03CBC90469946A246AB46F0BD9D42DF
:109CB00050D09C42E8DC6E4B9C426BD00023049356
:109CC0005346002B69DB002A10D1694B9C424CD0D3
:109CD000694B9C4200D1A3E08023DB05984500D16D
:109CE000BCE0664B984501D100F0D6FB5846514682
:109CF00001F02CFE4B4600900191002B07D1002D66
:109D000067D053465C4A9B009B08934261D0534600
:109D1000DB0F013B99464A46049B134300D190E078
:109D2000574B9C4200DCBBE0564B9C4201DC00F0F0
:109D300010FC554B9D4201DC00F004FC4346002B17
:109D400023DD524A524B1000190003F0C3F9009072
:109D50000191A3E7002805D04E4801F0A3FE009032
:109D600001919BE7AC42F7DCA5E75A46414BEB1863
:109D7000134300D18EE7444B9D4200DC99E34346F8
:109D800000960197002B00DB88E700230024009356
:109D9000019483E7002A91D076E73F4B9C423CDC5C
:109DA000394B9C428FDD3D4923158C466344142B6F
:109DB00000DCB2E33421CB1A3100D94008009840CE
:109DC000904200D07FE70123194001335B1A0493CE
:109DD00079E74346002B07DA009A019B00202649C9
:109DE00002F06EFD00900191029B002B00DB55E715
:109DF000204B9C46049B65441D4301D100F00EFCA2
:109E0000049B012B00D049E7009C019D802122008A
:109E100009066B180092019340E70223049352E76E
:109E200058465146434600900191002B00DB35E730
:109E30005A4653460020104902F042FD009001911D
:109E40002CE75A4653465846514603F0B5FB0200EC
:109E50000B0002F035FD009001911FE75A46534672
:109E60005846514603F036F90090019116E7C04676
:109E70000000F07F000010C00000F03F0000E03F55
:109E80000000E0410000F043FFFFEF3F9C750088B9
:109E90003CE4377E200F0100FFFF3F4301FCFFFF42
:109EA000E44B00229D420ADC009801990022E24B1B
:109EB00003F010F935220D00009001915242DF4964
:109EC0002B158C46634498462D03DD4CDD4B2D0B42
:109ED00090442C439D420ADDDB4B9D4201DC00F0A7
:109EE00001FC01239C46D94BE0449C46644400227B
:109EF00000230E920F931092119300220025D04B55
:109F00000692079300980199069A079B21000890F2
:109F1000099103F051FB069A079B0A900B91089850
:109F2000099902F0B1F902000B000020C44902F0C7
:109F3000C7FC0A00010013000C910D9202000A9860
:109F40000B9903F0C7F80A00010013000291039275
:109F5000002200920193802364109B0523438024F8
:109F60002403A44600206344591904000D00020094
:109F70000B000098019903F0ADF802000B000A985D
:109F80000B9903F019FB069A079B0A900B9120008E
:109F9000290003F011FB02000B000898099903F057
:109FA0000BFB009A019B03F095F802000B000A9846
:109FB0000B9903F001FB0C9A0D9B03F08BF8029CAC
:109FC000039D0890099122002B002000290003F036
:109FD00081F804000D009E4A9E4B03F07BF89E4AD8
:109FE0009E4B02F051F922002B0003F073F89C4ABB
:109FF0009C4B02F049F922002B0003F06BF89A4ABF
:10A000009A4B02F041F922002B0003F063F8984AC2
:10A01000984B02F039F922002B0003F05BF8964AC6
:10A02000964B02F031F92200069007912B00200098
:10A03000290003F04FF802000B000698079903F07F
:10A0400049F8009A019B04000D000298039902F060
:10A050001BF9089A099B03F03DF822002B0002F03F
:10A0600013F9009C019D0A900B9122002B00200007
:10A07000290003F02FF80022814B04000D0002F0AC
:10A0800003F90A9A0B9B02F0FFF800220B00110063
:10A090001A00069107920A000098019903F01AF835
:10A0A00000220C900D9106980799754B03F084FAE5
:10A0B00022002B0003F080FA02000B000A980B9993
:10A0C00003F07AFA029A039B03F004F8069A079BBE
:10A0D00004000D000898099902F0FCFF02000B0033
:10A0E0002000290002F0D0F804000D0002000B004F
:10A0F0000C980D9902F0C8F800221000E022614B84
:10A1000012060090019102F0E5FF0C9A0D9B02905F
:10A1100003910098019903F04FFA02000B00200010
:10A12000290003F049FA584A564B02F0D3FF574A28
:10A1300004000D0000980199554B02F0CBFF02007E
:10A140000B002000290002F09FF8109A119B02F0EA
:10A150009BF806900791404603F0C8FD069A079BBE
:10A1600004000D000298039902F08EF80E9A0F9BDE
:10A1700002F08AF822002B0002F086F8002022006C
:10A180002B000090019103F017FA0E9A0F9B03F039
:10A1900013FA029A039B03F00FFA02000B000698D1
:10A1A000079903F009FA069007914A46049B013B80
:10A1B000134300D188E10023214C02930394002231
:10A1C0003B0030003900140003F0F6F9009A019BBF
:10A1D00002F080FF32003B00049005910698079939
:10A1E00002F078FF02000B000498059902F04CF889
:10A1F0003D0006000F000098019922002B000496F4
:10A20000059702F067FF02000B0030003900009252
:10A21000019302F039F81F4B04000D008B46020039
:10A22000994200DC55E11C4BCB18034300D0FBE105
:10A2300034E0C046FFFF0F000000404301FCFFFF79
:10A240000000F03F8E98030079B60B000000F0FF8D
:10A25000EF4E454A287ECA3F65DBC9934A86CD3F0B
:10A2600001411DA96074D13F4D268F515555D53FF1
:10A27000FFAB6FDBB66DDB3F033333333333E33F89
:10A280000000084009C7EE3FFD033ADCF5015B140E
:10A29000E02F3EBEFFFF8F40000070BF049805997D
:10A2A000E84AE94B01F0F0FF009A019B06000F001D
:10A2B0002000290003F080F902000B003000390073
:10A2C00001F028FEAA46002800D0ADE18024DF4A34
:10A2D00053469446640322001B1563441A4113003D
:10A2E000DB495B445A001E001B038C461B0B2343B7
:10A2F0001424520DD74D62441541A21A13419946B8
:10A300005B46AE4300203100002B02DA4B465B4235
:10A31000994602000B000098019903F04DF94B4655
:10A320001B0500900191020098460B0004980599C6
:10A3300001F0AAFF0D0000240022C74B20002900D5
:10A3400002F0C8FE009A019B0690079120002900A8
:10A3500003F032F902000B000498059903F02CF980
:10A36000BE4ABF4B02F0B6FEBE4A06000F00BE4B0F
:10A370002000290002F0AEFE02000B003000390080
:10A3800001F082FF04000D0002000B0006980799FF
:10A3900001F07AFF069A079B06000F0003F00CF904
:10A3A00002000B002000290003F006F932000090A3
:10A3B00001913B003000390002F08CFE04000D00DA
:10A3C000AA4AAB4B02F086FEAA4AAB4B03F0F4F864
:10A3D00022002B0002F07EFEA84AA94B01F054FF98
:10A3E00022002B0002F076FEA64AA74B03F0E4F809
:10A3F00022002B0002F06EFEA44AA54B01F044FFA0
:10A4000022002B0002F066FE02000B003000390033
:10A4100003F0D2F804000D0002000B0030003900F8
:10A4200002F058FE8023049005910022DB052000F5
:10A43000290003F0C1F802000B000498059902F00E
:10A440003FFA009A019B04000D003000390002F031
:10A4500041FE009A019B01F017FF02000B00200053
:10A46000290003F0A9F832003B0003F0A5F8020030
:10A470000B000020874903F09FF843465B181A152C
:10A48000002A00DC3FE11900029A039B02F022FE41
:10A4900000900191FFF702FC5346002B01DAFFF711
:10A4A00025FC5846514600F04DFB00900191FFF706
:10A4B000F5FB4346002B00DB67E480231B06FB18FB
:10A4C00000960193FFF7EAFB0023734C0293039479
:10A4D00075E64B005B089A46704B9A4500DCF9E044
:10A4E0006F4B5B441A430AD1009A019B03F064F856
:10A4F000049A059B01F018FD002800D1E6E60298B9
:10A500000399684A684B02F0E5FD664A664B02F023
:10A51000E1FD00900191FFF7C1FB002A01D0FFF798
:10A52000E5FB1432D31A22001A4111009940A142CE
:10A5300001D0FFF7CDFB01231A40DB189B1A0493CF
:10A54000FFF7C6FB4346002B01DBFFF71EFCFFF7BE
:10A55000F8FB564B9D42F5DD4E4B9D4201DDFFF76A
:10A56000EDFB0098019900224A4B03F025F8C02228
:10A570004F4BD20504000D0002F0ACFD4D4A029095
:10A5800003914D4B2000290002F0A4FD0022009011
:10A5900001914A4B2000290002F09CFD02000B00B3
:10A5A0004748484903F008F822002B0002F092FDCA
:10A5B00002000B000020444902F0FEFF220006903A
:10A5C00007912B002000290002F084FD02000B00FF
:10A5D0000698079902F07EFD1A4A354B02F07AFD83
:10A5E00002000B000098019902F0E6FF02000B0048
:10A5F00004000D000298039901F046FE029A039BA5
:10A6000000200090019102F0D7FF02000B00200013
:10A61000290002F0D1FF06900791C6E50098019944
:10A6200002000B00FFF711FC284A294B02980399FE
:10A6300002F050FD254A264B02F04CFD009001919E
:10A64000FFF72CFBFE822B654715973C02FCFFFFB2
:10A6500001FCFFFFFFFF0F00432EE63FEF39FAFE3C
:10A66000422EE63F396CA80C615C20BED0A4BE72BD
:10A670006937663EF16BD2C541BDBB3E2CDE25AFCE
:10A680006A56113F93BDBE166CC1663F3E55555587
:10A690005555C53F0000F03F0000F0BFFFCB904094
:10A6A00000346F3F59F3F8C21F6EA501FEFFEF3F64
:10A6B0004715F73F44DF5DF80BAE543E0000D03F36
:10A6C000555555555555D53F0000E03F9C750088C0
:10A6D0003CE4377E00220E4B904691469A4500DCC2
:10A6E00029E6F3E580220B4BD2050E920F930A4A1E
:10A6F0000A4B8025109211930022094BED0206921D
:10A700000793FFF7FFFB4A4601F0D2F9BCE6C046CB
:10A710000000E03F03B8E23F06D0CF43EBFD4C3EE4
:10A720000000F83FF0B54E464546DE465746E0B5D8
:10A73000E14B4C008FB09046894664089C4200DC97
:10A7400087E0DE4B9C4222DCDD4A002900DC92E0FF
:10A75000DC4B02F031FFDB4B06000F009C4200D1C6
:10A760007EE1D94AD94B02F027FF02000B00414697
:10A7700030000A604B60390002F01EFFD34BD24A12
:10A7800002F01AFF434601259860D9606BE0D04B78
:10A790009C4200DC8FE0CF4B9C4200DD55E1CE4A6D
:10A7A000231592469A4451460905631A19001D0063
:10A7B000040003F065FA03F099FA02000B00200090
:10A7C00029000892099302F0F7FE0022C34B02F021
:10A7D00081FC0F00060003F053FA03F087FA04002F
:10A7E0000D0002000B00300039000A940B9502F0B6
:10A7F000E3FE0022B94B02F06DFC002200230C9016
:10A800000D9101F06DFB002800D192E100230022A0
:10A810002000290001F064FB434243410133B04A68
:10A8200041460192022208A80092524600F07CFBA9
:10A830004B460500002B16DA80224346120694464A
:10A8400042465B68454263445360D3686344D360C7
:10A8500009E00B00020041460A604B600022002321
:10A8600000258A60CB6028000FB03CBC904699461A
:10A87000A246AB46F0BD934B01F006FD914B06009E
:10A880000F009C4200D13DE18F4A904B01F0FCFC4F
:10A8900002000B00414630000A604B60390002F0B4
:10A8A0008BFE894A894B01F0EFFC012543466D423E
:10A8B0009860D960D7E701F049F88A4A8A4B0600C8
:10A8C0000F0002F007FC0022884B01F0DDFC03F0D2
:10A8D000D7F9050003F00AFA794A7A4B04900591FA
:10A8E00002F0F8FB02000B003000390002F064FEB9
:10A8F000754A06000F0004980599744B02F0EAFBB4
:10A90000029003911F2D00DCC7E0029A039B3000E8
:10A91000390002F051FE83468A4653465B002415F7
:10A920005B0DE31A102B6CDD04980599D322674B5D
:10A93000520502F0CFFB02000B00300039000292FA
:10A94000039302F039FE0A000100130006910792FA
:10A9500002003900300002F02FFE029A039B02F041
:10A960002BFE06000F0004980599614A614B02F026
:10A97000B1FB32003B0002F01FFE069E079F0B005A
:10A980000200390030000292039302F015FE4B00E2
:10A990005B0D83468A46E41A312C32DD0498059912
:10A9A000B822544B920502F095FB03000C00020004
:10A9B000029303940B000698079902F0FDFD020034
:10A9C0000B0006000F000698079902F0F5FD029AA9
:10A9D000039B02F0F1FD484A029003910498059907
:10A9E000464B02F077FB029A039B02F0E5FD020062
:10A9F0000B00300039000292039302F0DDFD834624
:10AA00008A465A465346414630000A604B60390038
:10AA100002F0D2FD029A039B02F0CEFD44460B00E9
:10AA20000200A260E3604B46002B00DB1BE75B46A5
:10AA3000236080231B065344636080231B069C46CF
:10AA40006144A060E1606D420DE70B00020002F07E
:10AA5000B3FD434600259860D9601860596002E74D
:10AA6000D3221A4B520502F0A7FD214A214B0D00BB
:10AA7000040002F0A1FD02000B00414620000A6024
:10AA80004B60290002F098FD1A4B194A02F094FD20
:10AA9000434601259860D960E5E602000B003000CE
:10AAA000390002F089FD6B1E154A9B009B588346B6
:10AAB0008A46A342A5D130E7FB21E93F7BD902407A
:10AAC00000004054FB21F93F3163621A61B4D03D6C
:10AAD000FB213941FFFFEF7FEAFBFFFF00007041E0
:10AAE000A40F010083C8C96D305FE43F0000E03F60
:10AAF0007370032E8A19A33BC14920259A837B39A1
:10AB0000240F0100D3220C4B520501F0BDFB0B4A70
:10AB10000B4B04000D0001F0B7FB02000B00414697
:10AB200020000A604B60290002F046FD034A044BF6
:10AB3000B9E6032373E6C04661B4D03D7370032EBB
:10AB40008A19A33BF8B54746CE46674B80B50A0045
:10AB50000F00190005003940994200D19BE0040024
:10AB60000100002F69DD3F1500D1B4E05F4B1203F7
:10AB70009C468023120B5B0313435B00CA0F6744A0
:10AB80009B184A00F80703D5D20F5B009B188A0078
:10AB900079108C46002180201624894680030D18E8
:10ABA0009D4202DC29185B1B8144D50F5B00013CF0
:10ABB0005B1952004008002CF1D100208046802013
:10ABC00020250027000609E08B425CD0D40F5B00F3
:10ABD000013DE31852004008002D16D0C4198B42E5
:10ABE000F2DD27180E00002C49DB5B1AA2428941D6
:10ABF00049425B1A121BD40F5B00013D80443100B7
:10AC0000E31852004008002DE8D113434ED14346CB
:10AC10005B0837494A468846494652104244C907AC
:10AC200002D5802109060B4361460F05BD181800A7
:10AC300029000CBC90469946F8BD7B005B08034395
:10AC40003900002BF5D0002F3CD1E30A153A6405FA
:10AC5000002BFAD08020400303423FD1002700E0C0
:10AC60000F005B00791C0342FAD0250020208D40A4
:10AC7000401A2900D71B2200C2401A4376E7FE4340
:10AC8000F60F8E19B1E79442A0D82718002CF6DBF6
:10AC90001E000023AEE702003B002800390002F04E
:10ACA00019FA2A003B0001F0EFFAC2E743460133EC
:10ACB00003D0434601335B08ABE7012398460023EA
:10ACC000C144A6E73B00020002F076FC02000B0044
:10ACD00001F0F6FDADE713000022BBE701272100DC
:10ACE00020207F42C6E7C0460000F07F01FCFFFF46
:10ACF0000000E03FF0B54746CE4680B587B00092F1
:10AD00000193754B4F00814688467F089F4263DC64
:10AD100002F0B6FF002800D1D4E04A464346484638
:10AD2000414602F0D7F904000D006C4A6C4B02F06A
:10AD3000D1F96C4A6C4B01F0A7FA22002B0002F00B
:10AD4000C9F96A4A6A4B02F037FC22002B0002F074
:10AD5000C1F9684A684B01F097FA22002B0002F013
:10AD6000B9F9664A664B02F027FC22002B0002F07C
:10AD7000B1F9644A644B01F087FA22002B0002F01B
:10AD8000A9F9029003910022604B2000290002F0F3
:10AD9000A1F9029A039B06000F002000290002F08F
:10ADA00099F9009A019B04000D004846414602F0C3
:10ADB00091F902000B002000290002F0FDFB0200C7
:10ADC0000B003000390002F0F7FB02000B000020FE
:10ADD0004F4902F0F1FB70E002000B0002F07AF93B
:10ADE00004000D003D4A3E4B02F074F93D4A3E4BD3
:10ADF00001F04AFA22002B0002F06CF93B4A3C4B6E
:10AE000002F0DAFB22002B0002F064F9394A3A4BD7
:10AE100001F03AFA22002B0002F05CF9374A384B75
:10AE200002F0CAFB22002B0002F054F9354A364BDF
:10AE300001F02AFA2B00220002F04CF9354B029067
:10AE400003919F429FDD344B00229F423DDC3349FA
:10AE500000207B182E4916001F0002F0ADFB049065
:10AE600005910022294B2000290002F033F932001D
:10AE70003B0002F0A1FB029A039B06000F0020009A
:10AE8000290002F027F9009A019B04000D004846B2
:10AE9000414602F01FF902000B002000290002F0D9
:10AEA0008BFB02000B003000390002F085FB020032
:10AEB0000B000498059902F07FFB07B00CBC90468C
:10AEC0009946F0BD00201249F7E7154B0026049281
:10AED0000593144FC5E7C046FFFF3F3ED43888BEF8
:10AEE000E9FAA8BDC4B1B4BD9EEE213EAD529C802E
:10AEF0004F7E923E9015CB19A001FA3E7751C116B4
:10AF00006CC1563F4C5555555555A53F0000E03F87
:10AF10000000F03F3233D33F0000E93F0000E0FF84
:10AF20000000E73F0000D23FF0B5DE464E46454602
:10AF30005746E0B5DC4CA5440D9114001900A49AC5
:10AF40000993DA4B9200D6584D1E03901821E01E4B
:10AF50000696029500F0BAFEC3430100DB171940C4
:10AF60004B1C9A009B1ADB001B190B9105934C1B81
:10AF7000771918D4A59BA5009C463F1922AE6544BD
:10AF8000013707E0286802F0B1FE013403C604353A
:10AF9000BC4208D0002CF5DA00200021013403C6A1
:10AFA0000435BC42F6D1069B002B01DA00F0FDFB14
:10AFB000069B03990133DB009A46099BDA0094460D
:10AFC00000920022914672AA0492B94A61449346C3
:10AFD00088469AAB63449B44029B002B00DABCE199
:10AFE0005D4600260027039C4D442A686B6803CC0D
:10AFF00002F070F802000B003000390001F044F953
:10B00000083D06000F004445EFD1049B4B441E60F1
:10B010005F6008239C46E144D145DDD10EA80421A0
:10B020008446494261448C46069A93009C4461469A
:10B0300084460A910399083B63448C460C93009B19
:10B04000009263449B46009A0498D10003008C460A
:10B05000634408911E685F68002A33DD9549804685
:10B060008C466244D300984470AB9A460EAB994626
:10B070000022914B3000390002F02CF802F000FE63
:10B0800002F034FE00228D4B04000D0002F022F885
:10B0900002000B003000390002F08EFA02F0F0FDE1
:10B0A0004B4601C39946434620001A685B68290055
:10B0B00001F0EAF808235B429C46E04406000F00DA
:10B0C000D045D5D1059B30001A003900984600F0D4
:10B0D000EFFCFF2300229B0504000D0001F0FAFFA6
:10B0E00000F042FC0022764B01F0F4FF02000B005E
:10B0F0002000290002F060FA0D00040002F0C0FDFB
:10B10000814602F0F3FD02000B002000290002F04E
:10B1100053FA060040460F00002800DCEEE0009BDA
:10B1200018215A1E92000EAB9B58091A1D000D41A2
:10B13000A9448D405D1B0EAB9D5017231B1A1D416A
:10B14000002D2DDD01239C46009BE144002B00DCFB
:10B150001CE20E9C0123002C00D0B5E0009A012ACD
:10B1600009D099000EAA54580133002C00D0ACE04D
:10B17000009A9A42F5D1059B002B0EDD012B00D1E0
:10B18000A8E1022B09D1009B0EA95A1E92000EAB1A
:10B190009B5807939B029B0A8B50022D00D1C1E064
:10B1A000002300223000390000F09AFE009B0028A6
:10B1B00000D194E2069A591E8A4210DC414A0A984C
:10B1C00094460EAA6344944600229B0063441C6884
:10B1D000043B22438342FAD1002A00D0C0E0069B00
:10B1E0000EAA013B9B00D358002B00D0B3E00122F4
:10B1F0000C9B043B596801320029FAD0009B9C4605
:10B200006244110007921A0001338B4246DC0B980E
:10B2100063468046A59C4344A046099C9B00A146EA
:10B220004A449844D30022AA9146049A99449446E9
:10B23000089BA59A63448446614494469A468B00D1
:10B24000634400934346586802F050FD4B46186033
:10B250005960029B002B24DB4D46039C00260027EF
:10B2600001E0286869680CCC01F034FF02000B0093
:10B270003000390001F008F8083D06000F005C4579
:10B28000EFD153469E60DF6004239C460433E044C4
:10B290009C46009BE144E2449845D3D1079B009330
:10B2A000D1E600260027ECE794FDFFFFF010010037
:10B2B00018FEFFFFFFFFFF1F0000703E00007041FF
:10B2C00000002040FFFFFF3F002180225204141B9A
:10B2D0000EAA5450009999420EDD0EA884469B0098
:10B2E0000EAA8900D25861446344CF4800E01A682E
:10B2F000821A04C38B42FAD101243CE7059B002B40
:10B3000006D1009B0EAA013B9B00D558ED1517E70F
:10B310000022C64B300000F007FE002800D024E1D8
:10B3200000253DE732003B000020C14902F044F90E
:10B3300006000F00002C00D132E7059A0020BC491E
:10B3400000F0B6FB02000B003000390002F034F9C7
:10B3500006000F0024E7012250E70026002754E6EC
:10B360004B46059A079388468B000EA9CB58183A8E
:10B3700008950592002B0DD18C464146AD4B4344B8
:10B380009B006344043B58680139183A0028F9D0FF
:10B3900088460592059A0020A54900F089FB43469E
:10B3A00004000D00002B00DA05E29E000EAB9C4667
:10B3B0004346DB0066449C46059370AB9946049F68
:10B3C00067440097306802F091FC22002B0001F0E6
:10B3D00081FE002238607960974B2000290001F03F
:10B3E00079FE083F04000D00043EB945EAD14AAB9E
:10B3F00003939B4600239A46069B42469946434642
:10B400000132029204934B46002B00DAAAE080201E
:10B410008A4B009D9846C0058949002600270024D4
:10B4200008E008239C460835E044544511DC4346B7
:10B43000186859682A686B6801F04CFE02000B001E
:10B440003000390000F020FF013406000F00A14554
:10B45000E7DA5B46C0C39B4601239C46009BE2445F
:10B46000083B0093029B9A45CDD1049B9846A49B30
:10B47000022B00DD8EE0002B37DC1FD1059B00275F
:10B480001D00039B00249C461E006544083E2A685C
:10B490006B683800210000F0F7FE083D07000C0043
:10B4A000AE42F4D1089B002B03D080231B069C46A0
:10B4B00064443A0023000D990A604B600720079B03
:10B4C00018409B239B009D443CBC90469946A24655
:10B4D000AB46F0BD009B0EA95A1E92000EAB9B58C6
:10B4E00007935B025B0A8B5057E64346002B00DA5A
:10B4F00070E100200021DB004AAAD61848AF32686C
:10B500007368083E00F0C0FEB742F8D1089B002BDC
:10B5100000D025E10B0002004A984B990D9C226057
:10B52000636002F049F8434607000C00002B13DD6E
:10B5300001254CAEB14638002E0021004C460136A4
:10B540000CCC00F0A1FEA146B045F7DA089B07003D
:10B550000C00002B00D015E13A0023000D998A6001
:10B56000CB60ABE70026002773E701239C46009BD6
:10B57000E1440225002B00DDEBE532003B0000201A
:10B580002B4902F019F806000F0009E60024F2E545
:10B590004AAB0393A49B032B00D08FE74346002BB9
:10B5A00000DC14E1039ADB009B46130091465B44E8
:10B5B0001E685F68234B43440293DB00994448AB09
:10B5C0009A464B465C681B681800210032003B001D
:10B5D0000090019100F058FE04000D0002000B00E5
:10B5E0000098019901F0E8FF3B00320000F04CFEAA
:10B5F0004B469860D9601C605D6008235B429C46A6
:10B60000E14426002F00CA45DBD14346012B00DC74
:10B61000E3E0039A13005B441E685F68029BDB0053
:10B6200099464A44904610E0FFFFFF000000E03FCB
:10B630000000F03FFFFFFF3F0000703EB010010030
:10B64000FB21F93FFFFFFF1F984643465C681B68DC
:10B650001800210032003B000090019100F014FE20
:10B6600004000D0002000B000098019901F0A4FFF6
:10B6700032003B0000F008FE4346039A9860D96010
:10B680001C605D60083B26002F009A42DCD14D46CD
:10B690009446002600244746083565442A686B68AE
:10B6A0003000210000F0F0FD083D06000C00AF4224
:10B6B000F4D1039B4A9F5D689968D868089B002B6A
:10B6C00065D08022120694460D9B65446044644414
:10B6D0001F605D609960D8601E615C61EEE69A460D
:10B6E0004B460793059B30005A423900089500F0FD
:10B6F000DFF900223A4B06000F0000F015FC00288D
:10B7000024D0384B00223000390001F0E3FC02F075
:10B71000B7FA52460400950002F0E8FA0022304BD6
:10B7200001F0D8FC02000B003000390001F044FFAA
:10B7300002F0A6FA0EAA50510122059B524418337A
:10B740009046059393000EAAD45023E6534630004A
:10B7500039009C0002F094FA0EAB1851D04619E65D
:10B7600080230D9A1B06CB18106053600B0002005B
:10B770004A984B9901F020FF434607000C00002B2C
:10B7800000DDD5E680231B069C466444E4E62B00DE
:10B790003A000D9D2A606B600A000300AA60EB600E
:10B7A000320023002A616B6188E6099BDB0000936D
:10B7B00072AB049332E4A49B022B00DDE8E6002B7D
:10B7C00000DD92E600D079E6002700246AE6002634
:10B7D00000246EE70020002198E60026340068E788
:10B7E000000070410000703EF0B5CE46474680B57F
:10B7F00087B000920193474A4B00814688465B0818
:10B80000934207DC4146484602F03AFA4146031E9D
:10B81000484666D04A4643464846414601F05AFCEF
:10B8200004000D0002000B004846414601F052FCA6
:10B83000394A3A4B06000F002000290001F04AFC6B
:10B84000374A384B01F0B8FE22002B0001F042FCD1
:10B85000354A364B00F018FD22002B0001F03AFC6F
:10B86000334A344B01F0A8FE22002B0001F032FCD9
:10B87000314B324A00F008FD0E9B02900391002BE1
:10B8800034D00098019900222D4B01F023FC029A3C
:10B89000039B049005913000390001F01BFC02006D
:10B8A0000B000498059901F087FE22002B0001F09F
:10B8B00011FC009A019B01F07FFE224A04000D005A
:10B8C000214B3000390001F005FC02000B00200084
:10B8D000290000F0D9FC02000B004846414601F067
:10B8E0006BFE07B00CBC90469946F0BD02000B0001
:10B8F0002000290001F0EEFB124A134B01F05CFE20
:10B9000032003B0001F0E6FB4A46434600F0BCFC37
:10B91000E7E7C046FFFF3F3E7CD5CF5A3AD9E53D29
:10B92000EB9C2B8AE6E55A3E7DFEB157E31DC73EF0
:10B93000D561C119A0012A3F1111813FA6F810114C
:10B940000000E03F495555555555C53F49004B0846
:10B9500019007047034B48009C4640086044C00FE4
:10B960007047C04600001080474AF0B54F469146E8
:10B970004B005B0D99444646D6464A46C0B5050085
:10B980000C000E0088460700132A27DC002A4BDB38
:10B990003E4B13419A460B0052461340034318D0C6
:10B9A0003B4A3C4B2800210000F06EFC00220023A3
:10B9B00000F0B0FA002847D0002C04DA80234A4671
:10B9C0005B03134198444646534600279E43380084
:10B9D00031001CBC90469946A246F0BD332A08DDD2
:10B9E0008023DB009945F4D102000B0000F04CFCF1
:10B9F000EFE7294A9446012263445242DA409246D4
:10BA00000242E6D0224A234B2800210000F03CFCF1
:10BA10000022002300F07EFA002815D0002C1EDB47
:10BA2000534646469F430FE0194A1A4B280021000F
:10BA300000F02AFC0022002300F06CFA002803D05A
:10BA4000002C04DB0027002638003100C1E7640029
:10BA5000640825430027002DF6D0104EF4E74B462E
:10BA6000142B0BD03422D21A012393405D19BD420E
:10BA700008D201239C462F00E044D1E7133B9C46AB
:10BA8000E044CDE72F00CBE701FCFFFFFFFF0F00F5
:10BA90009C7500883CE4377EEDFBFFFF0000F0BFA3
:10BAA00000207047002001497047C0460000F87F21
:10BAB0004B0070B55B0D14000A00002B1AD14B002F
:10BAC0005B08034315D0234B002201F003FB224BFC
:10BAD0009C422DDB0A004B005B0D363B1F4DE318EB
:10BAE000AB422ADC002B0DDD1D4C1B0522401A4306
:10BAF000110070BD1B4DAB42F0D102000B0000F0F5
:10BB0000C3FBF6E71D00353519DA174B02009C42DE
:10BB100009DD0B001548164900F032F8134A144BA2
:10BB200001F0D8FAE5E70B001248134900F028F8B5
:10BB3000104A114B01F0CEFADBE70200E9E7084CAE
:10BB4000363322401B051343190000220B4B01F032
:10BB5000C1FACEE700005043B03CFFFFFE070000F3
:10BB6000FFFF0F80FF07000050C300009C75008896
:10BB70003CE4377E59F3F8C21F6EA5010000903CEB
:10BB800030B54A00DB0FDB0752081A43110030BD05
:10BB900002B4714649084900095C49008E4402BC60
:10BBA0007047C04603B47146490840004900095A2D
:10BBB00049008E4403BC7047002243088B4274D373
:10BBC00003098B425FD3030A8B4244D3030B8B429E
:10BBD00028D3030C8B420DD3FF22090212BA030CA7
:10BBE0008B4202D31212090265D0030B8B4219D388
:10BBF00000E0090AC30B8B4201D3CB03C01A5241A8
:10BC0000830B8B4201D38B03C01A5241430B8B42EF
:10BC100001D34B03C01A5241030B8B4201D30B03D8
:10BC2000C01A5241C30A8B4201D3CB02C01A5241FF
:10BC3000830A8B4201D38B02C01A5241430A8B42C2
:10BC400001D34B02C01A5241030A8B4201D30B02AB
:10BC5000C01A5241CDD2C3098B4201D3CB01C01AC5
:10BC6000524183098B4201D38B01C01A52414309CF
:10BC70008B4201D34B01C01A524103098B4201D3BD
:10BC80000B01C01A5241C3088B4201D3CB00C01A2A
:10BC9000524183088B4201D38B00C01A52414308A2
:10BCA0008B4201D34B00C01A5241411A00D20146C7
:10BCB000524110467047FFE701B5002000F0F0F850
:10BCC00002BDC0460029F7D076E7704703460B4314
:10BCD0007FD4002243088B4274D303098B425FD385
:10BCE000030A8B4244D3030B8B4228D3030C8B42B1
:10BCF0000DD3FF22090212BA030C8B4202D3121297
:10BD0000090265D0030B8B4219D300E0090AC30B6B
:10BD10008B4201D3CB03C01A5241830B8B4201D318
:10BD20008B03C01A5241430B8B4201D34B03C01A01
:10BD30005241030B8B4201D30B03C01A5241C30A79
:10BD40008B4201D3CB02C01A5241830A8B4201D3EA
:10BD50008B02C01A5241430A8B4201D34B02C01AD4
:10BD60005241030A8B4201D30B02C01A5241CDD279
:10BD7000C3098B4201D3CB01C01A524183098B42C4
:10BD800001D38B01C01A524143098B4201D34B01AD
:10BD9000C01A524103098B4201D30B01C01A524110
:10BDA000C3088B4201D3CB00C01A524183088B4297
:10BDB00001D38B00C01A524143088B4201D34B0080
:10BDC000C01A5241411A00D20146524110467047F2
:10BDD0005DE0CA0F00D04942031000D340425340F7
:10BDE00000229C4603098B422DD3030A8B4212D3B7
:10BDF000FC22890112BA030A8B420CD389019211E9
:10BE00008B4208D3890192118B4204D389013AD025
:10BE1000921100E08909C3098B4201D3CB01C01AFA
:10BE2000524183098B4201D38B01C01A524143090D
:10BE30008B4201D34B01C01A524103098B4201D3FB
:10BE40000B01C01A5241C3088B4201D3CB00C01A68
:10BE5000524183088B4201D38B00C01A5241D9D280
:10BE600043088B4201D34B00C01A5241411A00D201
:10BE70000146634652415B10104601D34042002BFD
:10BE800000D54942704763465B1000D3404201B57C
:10BE9000002000F005F802BD0029F8D016E7704731
:10BEA0007047C046D0400B1C1141203A03D49C4639
:10BEB0001341184363465242934018437047C046AB
:10BEC0008446101C62468C46191C634600E0C0463E
:10BED0001FB501F097F8002801D40021C8421FBD0A
:10BEE00010B500F0EFFF4042013010BD10B501F079
:10BEF00089F8002801DB002010BD012010BDC046DC
:10BF000010B501F07FF8002801DD002010BD0120F0
:10BF100010BDC04610B501F011F8002801DC00206A
:10BF200010BD012010BDC04610B501F007F8002873
:10BF300001DA002010BD012010BDC046F0B5CE468C
:10BF4000474615042D0C2E0080B50704140C3F0C39
:10BF50009946030C7E435D43674363437F19340C6A
:10BF6000E4199C46A54203D980235B029846C44449
:10BF70004B4643435143250C36046544360C240498
:10BF8000A4195B19591820000CBC90469946F0BDC5
:10BF9000F0B54E4657464546DE46E0B543025B0ADD
:10BFA000450083B00F1C99462D0EC60F002D57D0AB
:10BFB000FF2D24D08020DB00C004184300238146DD
:10BFC0009A469B467F3D7C027A00FB0F640A120E64
:10BFD000984623D0FF2A4BD0E30080240020E404BD
:10BFE0007F3A1C43AD186B1C47460193534677407C
:10BFF0003A000F2B48D87D499B00CB589F46002B19
:10C0000000D085E008339A46063B9B467C027A00C6
:10C01000FB0FFF25640A120E9846DBD1002C00D0DE
:10C0200090E0524601231A4392460120DBE74C463A
:10C0300058461700022824D0032800D1CFE0002260
:10C04000002301284DD15802D205400AFF071043B2
:10C05000384303B03CBC90469946A246AB46F0BD7F
:10C06000002B5BD104239A46033B00259B46AAE79D
:10C07000FF35002C60D1524602231A43924602201B
:10C08000B1E7FF220023DEE74B461B0C9C464B46E4
:10C090002604360C180461463300220C6446000C5A
:10C0A00043434E435043544380191A0C121896428E
:10C0B00003D9802149028C4664441B041B0C1004E4
:10C0C000C01883015E1EB341800E1843130C1B1968
:10C0D0009B0103431C00230179D5012362081C4006
:10C0E0001443019A7F32002A4DDD630704D00F23E9
:10C0F0002340042B00D00434230103D53C4B019A88
:10C100001C408032FE2ABCDCA3015B0AD2B29AE753
:10C110000C239A46093BFF259B4654E7180001F083
:10C1200071FE4A46431F76259A4000236D42914690
:10C130002D1A9A469B4646E7524603231A439246D7
:10C14000032050E7200001F05DFE431F2D1A9C40A4
:10C15000763D002047E780230027DB03FF2272E7BC
:10C16000424666E74C463200584662E780234A461C
:10C17000DB031A4222D01C4220D123435B025B0A1C
:10C180004746FF225FE701239A1A1B2A21DC23007E
:10C190000199D3409E318C401A0023005C1EA341BC
:10C1A00013435A0704D00F221A40042A00D0043344
:10C1B0005A0111D49B015B0A002244E780234A46BE
:10C1C000DB0313435B025B0A3700FF223BE7019569
:10C1D00087E70022002336E70122002333E780238C
:10C1E000DB0323435B025B0AFF222CE70011010003
:10C1F000FFFFFFF770B500283DD0C317C5185D409D
:10C20000C40F280001F0FEFD9E22121A962A07DCB8
:10C21000D2B2082833DD083885406802400A23E09E
:10C22000992A0BDD052329001B1AD94003001B3373
:10C230009D402B005D1EAB4119430D00052801DD1B
:10C24000431F9D402B000F490B406E0709D00F265E
:10C250003540042D05D004335D0102D59F220B40EB
:10C26000121A9B01580AD2B24002D205400AE407D2
:10C270001043204370BD002400220020F4E7680230
:10C28000400AF1E7FFFFFFFBF0B54F464646D646B2
:10C290000C000903C0B5490A470F5E0039431F036C
:10C2A000DB0F9C4665007B0A570F1F436D0DE40FA3
:10C2B000760DA146C000B846D200AB1B64457BD0CA
:10C2C000002B5FDD002E00D0A4E03E00164300D11D
:10C2D00012E15E1E002E00D09EE1871A4346B8424E
:10C2E00080410125C91A4042091A0B0200D431E1EC
:10C2F00049024E0A002E00D16EE1300001F082FDAD
:10C300000300083B1F2B00DD61E120223900D21A17
:10C310009E40D1409F400E439D4200DD51E15D1B98
:10C320006B1C1F2B00DD7CE12021C91A3D00300071
:10C330008F408840DD40791E8F413100072228431D
:10C34000D940002507433A40002A09D00F233B403B
:10C35000042B05D03B1DBB42BF417F42C9191F00C2
:10C360000B0200D426E26A1CC64B55056D0D9A429D
:10C3700000D106E1C44AFF080A40530752023B437A
:10C38000120B8EE0002B00D0B8E06B1C5B055B0D40
:10C39000012B00DC30E1871A4346B842B641CB1A84
:10C3A00076429E1B330200D54CE13B003343A1D1C2
:10C3B00000220024002570E0002B00DCE5E0002EC8
:10C3C00000D183E0AF4EB54260D0802636043743BB
:10C3D000B846382B00DC3EE1434613431F007A1E6B
:10C3E00097413F1887428041404209180B0200D410
:10C3F000B0E0A44B01359D4200D1C3E0A24A7B08C6
:10C400000A4001210F401F435108D30707221F4351
:10C410003A4099E79B4EB54238D0802636043743E0
:10C42000B846382B00DDDCE01F2B00DC30E11E00BD
:10C430004746203EF740BC46202B04D04026F31A46
:10C4400046469E403243170063467A1E97411F437B
:10C45000CCE0002B00D104E24346134300D159E164
:10C460004B07C00818438023C9081B03194208D092
:10C470004546ED081D4204D14346D00859070843FC
:10C480002900420FC9007F4D1143C0004B07CA0865
:10C490007C49C00803438D4268D012036D05120B1E
:10C4A0006D0D002112031800130B0A0D12051A431B
:10C4B000764B2D0513402B435B00E4075B082343B9
:10C4C00019001CBC90469946A246F0BD3E0016439A
:10C4D00012D05E1E002E00D000E1871887428041F6
:10C4E00041444042091801250B0233D5022585E756
:10C4F00064463300414610001D00C7E7002D00D000
:10C50000DAE00C000443F3D05C1C00D19FE15D4CE9
:10C51000A64200D12FE1DB43382B00DD66E11F2B63
:10C5200000DD83E120240500E41A0F00DD40D9403E
:10C53000A0404346A7405B1A441EA04198462F43A3
:10C540003843171ABA42924143465242991A6446F6
:10C550003500CAE607223A40002A00D0F6E64B072B
:10C56000CA084849FF083B438D4296D11900114340
:10C5700000D19EE1802109030A431203120B414DB1
:10C580008FE71500002200238BE7002B00D0C7E0C7
:10C590006B1C5F057F0D012F00DCF1E0394DAB42D4
:10C5A00000D1B9E085180A008542894142444942D8
:10C5B00051180722CF076D082F4349083A401D0044
:10C5C000C2E607223049ED1A31403A40BCE63E004F
:10C5D0002838864000279FE6380001F013FC203001
:10C5E0008EE6434613431F007A1E9741C71BB8428D
:10C5F00080414042091A78E60E003B00064313438F
:10C60000002D61D1002E00D0F4E0002B00D11BE101
:10C6100064463900100039E71A4FBB427AD0330024
:10C62000FFE630001F3DE840202B03D04021CB1A0D
:10C630009E4037437B1E9F41072207433A4000211B
:10C64000002589E7171A4346BA42B641591A76427D
:10C650008E1B64464EE61F2B00DDADE020264746CC
:10C66000F61AB740B9461700B246DF404E463E4381
:10C6700037005646B240561EB24117434246DA4092
:10C680008918AEE6FF070000FFFF7FFFFFFF0F8066
:10C6900020264746F61AB740B9461700B246DF4093
:10C6A0004E463E4337005646B240561EB2411743EF
:10C6B0004246DA40891A99E77F4CA6425BD0802433
:10C6C00024045B42214327E7002E0CD1002B00D12C
:10C6D000CBE0644639001000774DD7E6764FBB4279
:10C6E00018D0330075E6002B14D04B07C008184350
:10C6F0008023C9081B03194207D0FC081C4204D13F
:10C700007907D0080843E14621004C46420FC90092
:10C710001143C000684DB9E61D0000220023C0E6A9
:10C72000002D5BD10D00054300D1E2E65D1C00D178
:10C73000B0E0614DAE421FD0DB43382B71DC1F2BC4
:10C7400000DD96E020250F00ED1AAF40B946070046
:10C75000AA46DF404D463D432F005546A840D940EC
:10C76000451EA84188440743BF1897429241514251
:10C77000414435003AE6644635004146100085E6FE
:10C780000B000343002D00D063E6002BF5D0434699
:10C79000134300D17AE6871887428041072241443B
:10C7A000404209183A400B0200D4D5E6434B01350C
:10C7B0001940C9E5380069E61E004746203EF740AB
:10C7C000BC46202B04D04026F31A46469E403243F6
:10C7D000170063467A1E97411F4302E6364DAE426C
:10C7E000CAD080252D045B422943A6E70843411E99
:10C7F0008841A6E6002B00D148E6871A4346B84296
:10C80000B641CB1A76429E1B33024BD5171A4346CC
:10C81000BA429241591A5242891A072264463A4052
:10C8200092E501430F00791E8F419DE71C000F0028
:10C83000203CE740202B03D04024E31A99400843D2
:10C84000411E884138437CE60022002425E6171A61
:10C850004346BA429241591A5242891A64463500F7
:10C8600043E541461000144D10E6802200241203D7
:10C8700080E61D000F00203DEF40BC46202B03D07A
:10C880004025EB1A9940084307006346781E87410C
:10C890001F4369E7871897429B4141445B42C9188F
:10C8A0003500A3E53B003343CED0072231003A40A8
:10C8B00052E600231A00F4E5FF070000FFFF7FFFA8
:10C8C000F0B55746DE464E464546E0B5834607007E
:10C8D0000E03480085B092461C00360B400DCD0F6C
:10C8E000002800D19DE0954B984239D08023F60076
:10C8F0001B041E43924A7B0F334399469446030020
:10C900006344009300230026FF00029323031B0BC4
:10C9100098466300E40F52465B0D019400D1B3E0EA
:10C9200086498B4200D19EE04246D100802212040B
:10C930000A435146490F11438B46814952468C4662
:10C9400000996344CB1A0021D20000932B0063406E
:10C950009A460F2E00D905E17A4BB6009B599F46A7
:10C960005B463343994600D0B8E0022308260027EF
:10C9700000900293CAE7CB463A0002990195019BC9
:10C980009A46022927D0032900D180E2012944D008
:10C990006D49009B8C4663441C00002C38DD530716
:10C9A00000D013E2D2085B46DB0109D55946674B3C
:10C9B00019408B468021C9008C46009B63441C00B3
:10C9C000634B9C4207DC5B4664055F075B021743D1
:10C9D0001B0B620D02E000230027584A00211B03B5
:10C9E0001C0B0B0D1B05234314055A4A380013403A
:10C9F0001C4353466400DB0764081C43210005B058
:10CA00003CBC90469946A246AB46F0BD012252423C
:10CA100001231B1B382B00DCADE100220023002783
:10CA2000DCE75B46334399465ED0002E00D18AE1B5
:10CA3000300001F0E7F903000B3B1C2B00DD7BE12C
:10CA40001D22D31A5A460100DA4008398E401300DD
:10CA50005F46334399468F403F4B00261B1A009395
:10CA60000023029352E7414653460B433B499B4602
:10CA70008C46009B634400935B46002B3BD1022312
:10CA800000221E43022161E7434613439B4637D0F1
:10CA90004346002B00D162E1404601F0B3F90300A8
:10CAA0000B3B1C2B00DD53E102004146083A91404C
:10CAB00088461D21CB1A5146D9400B0041460B43F5
:10CAC0009B46534693401A00009B25499C46604470
:10CAD00003008C4663440093002137E70323B146EB
:10CAE00000900C26029311E70023009301330426E3
:10CAF000002702930AE70323C3461E43032125E7C9
:10CB000001331E430022012120E700239A4680239F
:10CB100000271B03094A61E7802349461B0319428A
:10CB200000D1E2E05946194200D0DEE00B431B037E
:10CB300017001B0BA246014A50E7C046FF07000042
:10CB400001FCFFFF40110100FF030000FFFFFFFE9B
:10CB5000FE070000FFFF0F800DFCFFFF01F8FFFF45
:10CB6000F3030000D94500D9CBE000D1C6E03C007A
:10CB700048460027009B013B00935B46160E1B02B4
:10CB80001E431302984633041B0C9946310C019145
:10CB9000FFF798F84A4642430B04210C050019435D
:10CBA0008A4207D98919013D8E4203D88A4201D9A8
:10CBB000851E8919881A0199FFF784F809048C46A3
:10CBC0004A46210464464243090C030021438A4239
:10CBD00004D98919013B8E4200D8F1E02D041D4390
:10CBE000AB464346891A4246280C12041D0C5B468C
:10CBF000140C22001B041B0C5A4303946B43444344
:10CC0000029568431B19150CEB189C4203D980242C
:10CC10006402A44660441C0C15041B042D0C20184F
:10CC20005D19814277D373D00C1AA24A7D1BAF42A3
:10CC3000BF419446009B7F426344E01B1C00864238
:10CC400000D1DBE00199FFF73DF84A4642430B046F
:10CC5000290C070019438A4207D98919013F8E42DE
:10CC600003D88A4201D9871E8919881A0199FFF7CA
:10CC700029F809044A46894629044D464243090CCD
:10CC8000030029438A4207D98919013B8E4203D800
:10CC90008A4201D9831E89193F04891A3A00039FE9
:10CCA0001A43380013041B0C584381460298150C94
:10CCB0006F43434345434846000C8446DB196344B5
:10CCC0009F4203D9802040028446654448461F0C99
:10CCD00000041B04000C7D191818A94200D284E03E
:10CCE00000D17FE001231A4357E680234A461B0305
:10CCF00013431B031B0BAA466F4A6FE6BA4200D9C7
:10CD000035E74B46DC0758087B081C43FF0734E730
:10CD10000024AF4289D247444745A4415B46644260
:10CD2000A4196418013BA6421ED2A0426DD800D1BE
:10CD3000B6E0241A9B4678E703005A46283B9A40FF
:10CD40000027914688E6584601F05CF8203072E6EC
:10CD500003005246283B9A4093460022B4E65046D0
:10CD600001F050F820309AE6A642E2D1B845DCD96D
:10CD7000341A9B4659E71F2B65DC504C0099A4469A
:10CD80005C46614408008C4011008240D940501E2E
:10CD900082410C4314435A46DA401300620709D01B
:10CDA0000F222240042A05D02200141D94428941FA
:10CDB00049425B181A0262D50122002300270DE6C2
:10CDC0008A4200D80AE7831E891907E70F23134018
:10CDD000042B00D1E6E5171D9742924153429B4434
:10CDE000FA08E0E5002800D1D7E57118531EB142DA
:10CDF00027D3A94215D358D01A0073E7002B00DCC3
:10CE000004E6012300229B44CDE502234744474525
:10CE100089415B429C46494289190C19E344241A12
:10CE200003E743465F0047459B41B8465B429E1976
:10CE3000023A8919A94200D054E7404500D051E791
:10CE4000ABE51A00F6E71F215F4649420C1BE7409D
:10CE5000202B07D01A49009B8C46634418005B4680
:10CE600083401A43501E82413A430727002317404C
:10CE700009D00F21002311401400042995D122006C
:10CE80005F075B021B0BD20817430022A6E5802335
:10CE900059461B030B431B0317001B0B064A9DE55A
:10CEA000BD42B2D89B460024BFE68045B9D31A00E4
:10CEB000C3E7C046FF030000FF0700001E04000098
:10CEC0003E040000F0B54F464646D6468446C0B5FF
:10CED0008046194E18030F034D00000B5C0082467C
:10CEE0003F0B6D0DC90F9146640DDB0F0120B5425C
:10CEF0000AD0B44203D0A54201D157450CD01CBC86
:10CF000090469946A246F0BD66463E43F7D1AC42F4
:10CF1000F5D154461443F2D10120C845EFD19942CE
:10CF200007D0002DEBD163461F433800471EB841A0
:10CF3000E5E70020E3E7C046FF070000F0B54F46F5
:10CF40004646D6464D00C0B50E03C90F8A462C4949
:10CF50001F035C008046360B6D0D91463F0B640D40
:10CF6000DB0F8D421ED08C4216D0002D1ED13043D7
:10CF70008446002C01D13A4323D06246002A1AD0BD
:10CF80009A4529D0514602200139084001381CBC7D
:10CF900090469946A246F0BD39001143E5D00220E3
:10CFA0004042F4E73043FAD1AC420FD0002C0FD10D
:10CFB0003A43E7D00CE00122013B934318000130D3
:10CFC000E5E763460020002BE1D0DBE73A43E6D1FA
:10CFD0009A45D7D1A542D5DCA54205DBBE42D1D8C2
:10CFE00008D00020BE42D2D25046012301389843D7
:10CFF0000130CCE7C845C5D80020C845F4D3C6E702
:10D00000FF070000F0B54F464646D6464D00C0B576
:10D010000E03C90F8A462E491F035C008046360B5B
:10D020006D0D91463F0B640DDB0F8D4218D08C4285
:10D0300011D0002D18D130438446002C1ED13A4324
:10D040001CD163460020002B30D05146022001390C
:10D05000084001382AE039001143EAD0022025E0D7
:10D060003043FBD1AC4226D0002C26D13A4324D108
:10D070005146022001390840013817E06246002A73
:10D080000FD09A45E1D1A54205DBBE42DDD819D0CB
:10D090000020BE420AD25046012301389843013095
:10D0A00004E00122013B9343180001301CBC904670
:10D0B0009946A246F0BD3A43D0D19A45C5D1A54282
:10D0C000C3DCE0E7C845C0D80020C845E3D3EDE79E
:10D0D000FF070000F0B55746DE464E464546E0B530
:10D0E000834606000F03480087B092461D003F0BA1
:10D0F000400DCC0F002800D16FE0DE4B984238D0B5
:10D100008023FF001B041F43730F3B430193DA4B43
:10D110000027994600239B46F60081442B036900B3
:10D120001B0B52469846490DED0F002900D185E0B2
:10D13000D04B994200D173E04346DA0080231B04B0
:10D1400013435246CC48520F8446134352460020A4
:10D150006144D20089442100694000918C4601213C
:10D1600049448A460F2F00D990E0C449BF00CF59E7
:10D17000BF465B463B43019300D06AE10223082788
:10D18000002681469B46C9E732005846019B61460E
:10D190000091022800D175E0032800D1FEE10128AA
:10D1A00000D02CE100230027002600253F032A0D94
:10D1B0003F0BB34812053A4302401B051343009A44
:10D1C0005B00D1075B080B433000190007B03CBC83
:10D1D00090469946A246AB46F0BD5B463B43019361
:10D1E00000D12FE1002F00D1A5E1380000F00AFEA8
:10D1F00003000B3B1C2B00DD96E11D22D31A5A467F
:10D200000100DA405E4608398F4013008E403B43F0
:10D2100001939C4B00271B1A994600239B467DE7F0
:10D22000414653460B4393498C46E144002B00D0C2
:10D230001AE102220220174300228CE7134300D197
:10D240000DE14346002B00D181E1404600F0DAFDBC
:10D2500002000B3A1C2A00DD72E101004346083946
:10D260008B4098461D239A1A5346D3401A004346D2
:10D27000134352468A404946081A824989468144E6
:10D28000002068E77B4B002700268EE7140C120471
:10D29000120C1100370C3604350C794328008C46EB
:10D2A0002E0060436044834656432100300C804684
:10D2B0005846794340440291844506D988468021E6
:10D2C00049028C46E044414602913604010C360C7A
:10D2D00000048B4681191E0C1B041B0C03911900C2
:10D2E00079438C46280075436544A8465843050C8D
:10D2F00045447743A94203D9802149028C466744BB
:10D30000290C8C4639000004000C2D042D186144B2
:10D31000AB4405915946049101990F043F0C080C48
:10D32000390051434243904602008C46090C8B461B
:10D3300062437C4344445C44A04503D980214902B4
:10D3400088464244210C884661460904090C8C46F3
:10D3500039005943434370437E430F0CF6182404AD
:10D36000BE19644442448C46B34203D980235B0215
:10D3700098464044029B61469846049B37044344C8
:10D380009B46AB45AD416B420D0405992D0C8C4677
:10D390007F196744FD18A8465D462D19A542A44192
:10D3A00093466442A446C344DC448F42BF4198453F
:10D3B0009B4193459241A445A4415B427F421F4358
:10D3C000360C52426442BF192243BF1862463818D5
:10D3D0004302D20D039913436A020A43501E82414D
:10D3E0006146ED0D2A434E023243D90100D4B3E029
:10D3F0000126500832400243DE0732435B08224CCC
:10D400005444002C62DD510709D00F20104004283D
:10D4100005D0101D9042924152429B180200D90142
:10D4200004D580241948E400034054441848844239
:10D4300000DD27E75E075B02D2081F0B630516437A
:10D440005B0DB2E6002399460133042700269B4674
:10D4500064E60323019781460C279B465EE6012282
:10D4600001201743002276E6032303201F4343468F
:10D4700071E6C046FF07000001FCFFFF80110100BC
:10D48000FFFF0F800DFCFFFFFF030000FFFFFFFE0B
:10D49000FE0700000023802700933F030026434B34
:10D4A00083E6019B3200A446584670E6AC466EE621
:10D4B000802701993F0339422DD03B422BD11F4396
:10D4C0003F033F0B00951600384B6EE601252D1BE0
:10D4D000382D00DD66E61F2D40DC35481C00504429
:10D4E000160082408440EE40501E82413443144373
:10D4F000EB40620709D00F222240042A05D0220007
:10D50000141D9442804140421B181A023ED501234B
:10D510000027002649E68027019B3F031F433F0366
:10D520003F0B0094214B40E603005A46283B9A40AB
:10D53000002601926DE6584600F064FC203057E664
:10D5400003005246283B9A401300002293E65046BF
:10D5500000F058FC20307BE6CA4650E71F201E0032
:10D560004042041BE640202D03D0124C5444A340FB
:10D570001A43501E8241324307260027164009D025
:10D580000F200023104014000428B9D122005E07A8
:10D590005B021F0BD2081643002306E680273F03D9
:10D5A0001F433F033F0B1600004BFEE5FF07000043
:10D5B0001E0400003E040000F8B557464E4645469E
:10D5C000DE460C000903E0B5490A460F5F0031430F
:10D5D0001E03DB0F760A9B46530F3343C84E65008C
:10D5E000C000E40FD2006D0DA24681467F0D9C461F
:10D5F0009046B74200D1B9E05B46012673409B4696
:10D60000EE1BA34500D183E0002E63DD002F00D088
:10D61000B1E06346134300D123E1731E002B00D019
:10D62000BAE1861A6346B04280410125C91A4042D8
:10D63000091A0B0200D447E149024B0A98464346B7
:10D64000002B00D189E1404600F0DCFB0300083BE1
:10D650001F2B00DD7CE120223000D21A4146D04051
:10D66000994002009E400A439D4200DD6AE15D1B35
:10D670006B1C1F2B00DD94E1202110003500C91A1E
:10D680008E40DA408840DD40711E8E411100072235
:10D690002843002506433240002A09D00F23334097
:10D6A000042B05D0331DB342B641764289191E00C2
:10D6B0000B0200D43DE26A1C914B55056D0D9A4258
:10D6C00000D119E18F4AF6080A4057075202374342
:10D6D000120B9BE0002E00D0C5E06E1C7605760D87
:10D6E000012E00DC48E16746861ACB1BB042BF41E1
:10D6F0007F42B8461F004346FF1A3B00B8461B0254
:10D7000000D55FE137439AD100220024002579E05B
:10D71000002E00DCFAE0002F00D18DE0784B9D4216
:10D7200067D0802367461B041F43BC46382E00DCAD
:10D7300052E1634613435A1E93411E1886428041AC
:10D74000404209180B0200D4BEE06D4B01359D42EA
:10D7500000D1D2E06B4A73080A4001210E401E43FB
:10D760005108D30707221E43324095E71E00164397
:10D7700000D045E740E7624B9D423AD080236746A0
:10D780001B041F43BC46382E00DDEBE01F2E00DCDF
:10D790003AE133006746203BDF403B00202E05D0B6
:10D7A0004027BF1B6646BE40324390464646721E27
:10D7B00096413343DAE0002B00D114E26346134371
:10D7C00000D168E180234E07C008C9081B03064347
:10D7D000194208D06046C008184204D163460100CF
:10D7E000D2085E071643F3009946C900720F444DF4
:10D7F00011434B46DE08424B4F073743CA089D4250
:10D8000000D16EE012036D05120B6D0D00211203A5
:10D81000130B0A0D12051A433B4B2D0513402B43E6
:10D820005B00E4075B082343380019003CBC9046CA
:10D830009946A246AB46F8BD6346134311D0731E0A
:10D84000002B00D007E186188642804161444042A7
:10D85000091801250B0237D502257BE73E006146FA
:10D8600091463500C5E75C46002D00D0E1E00B0095
:10D870000343F3D0731C00D1ACE1214B9F4200D194
:10D880003AE1F343382B00DD6FE11F2B00DD8CE123
:10D8900020250E00ED1AAE40B0460600AA46DE4036
:10D8A000454635432E005546D940A8406346451E9F
:10D8B000A8415B1A9C463043161AB2429241634615
:10D8C0005242991A3D00B4E607223240002A00D0A5
:10D8D000E4E60B4BF6084F073743CA089D4200D0D9
:10D8E00090E73B00134300D1A6E180231B031A43BA
:10D8F0001203120B024D89E715000022002785E76D
:10D90000FF070000FFFF7FFFFFFF0F80002E00D00A
:10D91000C7E06B1C5E05760D012E00DCF0E0C84D03
:10D92000AB4200D1B9E085180A00854289416244C2
:10D93000494251180722CE076D082E43490832404C
:10D940001D00A9E6BF49ED1A114007223240A3E6A7
:10D95000320028388240002686E6300000F052FA75
:10D96000203073E6634613435A1E9341C61AB042F1
:10D9700080414042091A5CE60E00674606431743A1
:10D98000002D5ED1002E00D0F3E0002F00D11EE16B
:10D990005C46614691462CE7A94FBE427BD01E00F3
:10D9A000F1E610001F3DE840202B03D04021CB1AA8
:10D9B0009A401643731E9E410722064332400021BF
:10D9C000002583E7161A6346B2428041591A404245
:10D9D0000B1A98465C4632E61F2E00DDABE020278E
:10D9E000BB1B9A4663465746BB40994613004F46B9
:10D9F000F3401F433B005746BA40571EBA411343FA
:10DA00006246F240891898E62027BB1B9A46634677
:10DA10005746BB40994613004F46F3401F433B0017
:10DA20005746BA40571EBA4113436246F240891A1C
:10DA30009CE7834B9F425FD080252D04734229438E
:10DA400020E7002E0CD1002F00D1D0E05C466146CB
:10DA500091467B4DCDE67A4FBE421CD01E0065E656
:10DA6000002F18D0C0084E0706438020C9080003C5
:10DA7000014208D06346DC08044204D12100DA46A2
:10DA8000D2085E071643F300994601245346C900A5
:10DA9000720F11431C406A4DABE61D0000220027A7
:10DAA000B4E6002D59D10B00034300D1D6E6731C18
:10DAB00000D1B2E0624B9F421ED0F343382B6FDCA3
:10DAC0001F2B00DD97E020250E00ED1AAE40B0467A
:10DAD0000600AA46DE40454635432E005546A8407E
:10DAE000D940451EA8418C440643B618964292413F
:10DAF000514261443D0025E63D006146914678E68D
:10DB00000B000343002D00D055E6002BF5D06346F3
:10DB1000134300D16DE6861886428041614440423D
:10DB2000091800220B0200D4D0E6464B01351940FB
:10DB3000B2E5B1465DE633006746203BDF403B007F
:10DB4000202E05D04027BF1B6646BE40324390467C
:10DB50004646721E96413343EFE5394B9F42CBD088
:10DB600080252D0473422943A8E70843411E8841BC
:10DB7000A2E6002F00D13CE66346861ACF1AB042D7
:10DB80009B415B42FB1A98461B024ED5161A634610
:10DB9000B2429241591A5242891A5C4600227BE5F0
:10DBA00001430E00711E8E419FE71D000E00203DB7
:10DBB000EE40B046202B04D04025EB1A9940084394
:10DBC000814648464346411E8841184374E6002278
:10DBD000002417E6161A6346B2429241591A52427D
:10DBE000891A3D0025E561469146154D01E68022E2
:10DBF0000024120379E61D000E00203DEE40B046E1
:10DC0000202B04D04025EB1A9940084381464E460C
:10DC10004346711E8E411E4367E7861896429B411C
:10DC200061445B42C9183D008CE547463743CED07E
:10DC300007224146324049E600273A00E6E5C04661
:10DC4000FF070000FFFF7FFF70B50C4E0D031C03A4
:10DC500049005B002D0B490D240B5B0DB14208D030
:10DC6000064900208B4203D114432000441EA041EA
:10DC700070BD05430120002DFAD1F1E7FF07000038
:10DC800030B5144D0A034B00120B5B0DC90F002475
:10DC9000AB4211DD104CA34210DC8024640322430C
:10DCA0000E4CE41A1F2C0CDD0D48C31ADA40130089
:10DCB0005C42002900D11C00200030BD094BCC186B
:10DCC000FAE7094DE040AC4663449A401300034331
:10DCD000EEE7C046FE0300001D0400003304000010
:10DCE00013040000FFFFFF7FEDFBFFFF70B500286E
:10DCF0002DD0C317C5185D40C40F280000F082F86E
:10DD0000154B1B1A5B055B0D0A2815DD0B3885408A
:10DD100000222D032D0B002110002D030A0D2D0BC9
:10DD200012052A430D4D1B052A4013435B00E407EF
:10DD30005B082343190070BD020029001532914091
:10DD40000A000B21081AC5402D032D0BE3E7002420
:10DD5000002300250022DEE71E040000FFFF0F80E5
:10DD60004100090E4B1C70B5DBB24602750AC40FA8
:10DD7000012B14DDE0239B006D07360BCB1800212F
:10DD80000A0D280012051C4D32435B052A405B0832
:10DD900013435B00E4075B082343190070BD0029AF
:10DDA00014D1002D1ED0280000F02CF80A281CDC0D
:10DDB0000B232A001B1ADA40030015339D400F4B3A
:10DDC00012031B1A5B05160B5B0DD8E7002D06D05E
:10DDD000320B802636036D071643094BCFE7084BFD
:10DDE0000026CCE700230026C9E703002A000B3BEE
:10DDF0009A400025E3E7C046FFFF0F80890300003B
:10DE0000FF0700001C2101231B04984201D3000CD2
:10DE100010391B0A984201D3000A08391B0998429D
:10DE200001D30009043902A2105C40187047C046B3
:10DE300004030202010101010000000000000000D3
:10DE400030B51C00094B05001B6885B0D868084B2D
:10DE5000002A01D1074B1A000292019300912B0076
:10DE60002200054900F026F800F0A6FD90000020F1
:10DE7000C0110100F7FB0000CD110100014B186833
:10DE80007047C04690000020084B10B50400002BDE
:10DE900002D0002100E000BF054B1868836A002B08
:10DEA00000D09847200001F05DFBC0460000000054
:10DEB000FC1101000EB403B5010003AB044804CB10
:10DEC0000068019300F076F802B008BC03B0184770
:10DED0009000002070B500260C4D0D4C641BA41062
:10DEE000A64209D1002601F03FFB0A4D0A4C641BF3
:10DEF000A410A64205D170BDB300EB589847013677
:10DF0000EEE7B300EB5898470136F2E760020020D5
:10DF1000600200206002002070020020002310B583
:10DF20009A4200D110BDCC5CC4540133F8E710B55F
:10DF3000884202D98B18984203D3002307E08B5CF8
:10DF40008354013AFBD210BDCC5CC45401339A42D5
:10DF5000FAD1F8E703001218934200D17047197004
:10DF60000133F9E7936810B5013B9360002B04DAA5
:10DF70009469A34207DB0A2905D01368581C106076
:10DF80001970080010BD00F04BFC0100F9E7F8B56E
:10DF900006000F001400D518AC4201D1002007E0A4
:10DFA00021783A003000FFF7DDFF0134431CF3D144
:10DFB000F8BD0000F0B59FB002900F001600059369
:10DFC000002805D083690493002B01D100F0F4FDF3
:10DFD0007B4B9F425BD1029B5F68BB891B0762D56D
:10DFE0003B69002B5FD0002306AC6361203363766E
:10DFF0001033A37635002B78002B01D0252B5CD174
:10E00000AB1B04930CD0320039000298FFF7BFFF1E
:10E01000431C00D1C4E06269049B9446634463617D
:10E020002B78002B00D1BBE001220023524262601A
:10E0300002A9543252186E1C2360E360A36013706F
:10E04000A365317805225F4800F0D4FE751C0028D6
:10E0500035D12268D30604D5532302A95B182021A9
:10E060001970130704D5532302A95B182B211970CB
:10E0700033782A2B2CD0350000210A20E3682A7837
:10E080006E1C303A092A64D900292ED026E04E4B66
:10E090009F4202D1029B9F689FE74C4B9F429CD1BD
:10E0A000029BDF6899E73900029800F00FFC002816
:10E0B00099D0012040421FB0F0BD01359BE7414B94
:10E0C0002268C01A01238340134323602E00B8E75F
:10E0D000059B191D1B680591002B01DB099304E0CA
:10E0E0005B42E3600223134323602B782E2B0AD17B
:10E0F0006B782A2B35D1059B02351A1D1B680592BA
:10E10000002B2BDB0793324E29780322300000F0DE
:10E1100071FE002806D04023801B83402268013511
:10E1200013432360297806222A486E1C217600F0CA
:10E1300061FE00283AD0284B002B25D10722059BF1
:10E1400007339343083305936369039A9B1863610C
:10E1500050E7434301219B18350090E701235B42C0
:10E16000D0E700230A201A000135636029786E1C6D
:10E170003039092903D9002BC5D00792C3E74243A0
:10E18000012352183500F1E705AB00933A00134B19
:10E190002100029800E000BF0390039B0133D3D11C
:10E1A000BB895B0600D584E70B9884E705AB009339
:10E1B0003A000A4B2100029800F080F8ECE7C046D4
:10E1C0005412010000120100741201003412010007
:10E1D000061201000A120100000000008FDF00009B
:10E1E000F7B5150001938A680B6900900C00934203
:10E1F00000DA130022002B6043321278002A01D08B
:10E2000001332B6023689B0602D52B6802332B60F9
:10E21000062723681F4027D0230043331B785A1E4C
:10E2200093412268920630D422000199433200982B
:10E23000089EB047431C25D0062320682A68E16861
:10E2400003400025042B03D18D1AEB43DB171D403F
:10E25000A3682269934201DD9B1AED180027BD4295
:10E2600020D1002010E00137E3682A689B1ABB42E6
:10E27000D2DD22000123193201990098089EB0478F
:10E28000431CF0D101204042FEBD3020E118433153
:10E29000087021005A1C45310978A2184332023314
:10E2A0001170C1E7220001231A3201990098089EDB
:10E2B000B047431CE6D00137D1E70000F0B589B084
:10E2C00004920A0043320593039002920A7E0C00E6
:10E2D0000E9B6E2A00D186E01FD8632A33D008D85F
:10E2E000002A00D18CE0582A4DD0250042352A70F2
:10E2F00030E0642A01D0692AF7D1196825680A1D1F
:10E30000280629D508681A60002803DA2D23029A06
:10E31000404213706B4E0A274FE0732A74D008D81E
:10E320006F2A1FD0702AE0D1202209680A43226098
:10E3300003E0752A16D0782AD7D1220078214532F9
:10E340001170614E22E025001A684235111D1960D6
:10E3500013682B70012365E008681A606906D3D53D
:10E3600000B2D1E719682568081D186008682E06F4
:10E3700005D5544E08276F2A1BD00A2719E06D06D1
:10E38000F7D580B2F5E745314E4E0A70186822681D
:10E39000011D00681960150621D5D30702D5202379
:10E3A0001A4322601027002803D1202322689A43B1
:10E3B00022602300002243331A706368A360002B9D
:10E3C00058DB0422216891432160002854D1029D2A
:10E3D000002B5AD02500337842352B7055E0550676
:10E3E000DBD580B2D9E71A680D68101D496918603D
:10E3F00013682E0601D5196002E06D06FBD5198061
:10E400000023029D23614FE01A68111D19601568F1
:10E4100000216268280000F0EDFC002801D0401BBC
:10E420006060636823610023029A13703CE02369F3
:10E430002A0004990398059DA847431C3ED02368F1
:10E440009B0715D4079BE068984239DA180037E03B
:10E4500022000123193204990398059EB047431CFA
:10E460002CD00135E368079A9B1AAB42F0DCE9E750
:10E470000025F7E70028ADD0029D3900FDF722FC0A
:10E48000735C013D2B700028F7D1082F09D1236858
:10E49000DB0706D563682269934202DC3023013D25
:10E4A0002B70029B5B1B2361059B07AA0093210035
:10E4B000049B0398FFF794FE431CB8D1012040420F
:10E4C00009B0F0BD11120100221201000D4B70B510
:10E4D0001C680500A36B002B0FD1182000F06EFC08
:10E4E000094BA0630360094B01224360084B836022
:10E4F0000B2383810023026143610022A36B1D6112
:10E500005A6170BD900000200E33CDAB34126DE621
:10E51000ECDE0500124B10B51C68A36B002B0FD16D
:10E52000182000F04BFC0F4BA06303600E4B012240
:10E5300043600E4B83600B238381002302614361A0
:10E54000A46B0B4A206961690A4BFDF7F7FC0122B5
:10E55000002380185941206161614800400810BDC6
:10E56000900000200E33CDAB34126DE6ECDE0500DA
:10E570002D7F954C2DF451580CB430B5164B9DB0F1
:10E580000C1E1D6808DA8B2301202B6040421DB051
:10E5900030BC08BC02B01847822302A99B008B81C3
:10E5A0000023029008619C4200D0631E8B604B6187
:10E5B00001235B42CB81209A21AB2800019300F01C
:10E5C00055FD431C01DA8B232B60002CDFD0002388
:10E5D000029A1370DBE7C046900000200EB400B52D
:10E5E0000B499CB01DAB029006900791049109481D
:10E5F000094904CB0591006802A9019300F036FD9A
:10E600000023029A13701CB008BC03B01847C04620
:10E61000FFFFFF7F900000200802FFFF020010B5FF
:10E620001378541C002B05D1CC5CD4540133002C3E
:10E63000FAD110BD2200F3E7C9B20378002B04D051
:10E640008B4200D170470130F7E74B4259414942B4
:10E650000840F7E702780B78002A03D00130013137
:10E660009A42F7D0D01A70470023C25C0133002AC7
:10E67000FBD1581E7047002330B59A420AD0013AA8
:10E68000C45CCD5CAC4204D1934202D00133002C77
:10E69000F6D1631B180030BD30B50500002A00D14B
:10E6A00030BD0C78013A6B1C2C700131002C05D167
:10E6B0009A189A42F4D01C700133FAE71D00EDE776
:10E6C00010B50378002B0FD10B785A4253415B42AF
:10E6D000184010BD0023CA5C002AFAD0C45C9442E2
:10E6E00001D10133F7E701300378002BF2D1180094
:10E6F000EFE70000F0B51F000E0087B00590019114
:10E7000002920C98347800F0EAFA08220019437853
:10E71000751C134036D12D2C36D1B51C74780126CA
:10E72000002F62D0102F09D1302C07D120222B7856
:10E730009343582B54D110276C7802352D4B390058
:10E74000F31818000393FDF7BDFA0491012100238B
:10E75000494202008C4618002100303909291AD894
:10E760000C00A74223DD591C09D06346824206D320
:10E7700002D10499A14202DB0123784320182C78AE
:10E780000135E9E72E00BCE72B2C01D01E00C7E7BE
:10E79000B51C7478FAE721004139192901D8373CB2
:10E7A000DFE721006139192901D8573CD9E75A1C04
:10E7B00008D1059A23331360029B0398002B09D1DB
:10E7C00007B0F0BD002E00D04042029A002AF7D0D8
:10E7D000002B01D06B1E0193029B019A1A60EFE798
:10E7E0003024002FAAD10827A8E7302C9ED00A2772
:10E7F000A4E7C046FFFFFF7F37B51300064A0500B8
:10E800001068046A002C00D1044C0A00009429000E
:10E81000FFF770FF3EBDC04690000020F4000020CE
:10E82000F8B505000E001400002804D08369002B01
:10E8300001D100F0C1F9224B9C422DD16C68A36933
:10E84000A360A3891B0731D52369002B2ED0236831
:10E850002269F7B2981A6369F6B2834205DC210097
:10E86000280000F03BF9002826D1A3680130013BC5
:10E87000A36023685A1C22601F706369834204D01E
:10E88000A389DB071AD50A2E18D12100280000F031
:10E8900025F9002812D00FE00A4B9C4201D1AC6848
:10E8A000CDE7094B9C42CAD1EC68C8E7210028009B
:10E8B00000F00CF80028CAD0012676423000F8BDDE
:10E8C000541201007412010034120100364B70B56D
:10E8D0001D6806000C00002D05D0AB69002B02D18D
:10E8E000280000F069F9314B9C420FD16C680C2371
:10E8F000E25E93B219072DD4D90611D40923012061
:10E90000336037331343A381404270BD284B9C4290
:10E9100001D1AC68EBE7274B9C42E8D1EC68E6E715
:10E920005B0713D5616B002908D02300443399425B
:10E9300002D0300000F06AFA002363632422A38926
:10E940009343A38100236360236923600823A28982
:10E950001343A3812369002B0BD1A0218022A3891B
:10E96000890092000B40934203D02100300000F058
:10E97000E1F90123A289134011D00023A360636948
:10E980005B42A361002023698342BED10C23E25E77
:10E990001306BAD540231343A3810138B5E7920784
:10E9A00000D46369A360EDE79000002054120100D9
:10E9B000741201003412010010B5062000F090FC22
:10E9C000012000F0CFFD0000F7B58A8905000C009A
:10E9D000130760D44B68002B04DC0B6C002B01DCAC
:10E9E0000020FEBDE76A002FFAD000232E682B60BE
:10E9F00080235B01216A1A4034D0606DA3895B07D4
:10EA000006D56368C01A636B002B01D0236CC01A53
:10EA10000200216A00232800E76AB847A189431C45
:10EA200006D12B681D2B30D82B4ADA40D3072CD5C2
:10EA30000023636023692360CB0405D5431C02D106
:10EA40002B68002B00D16065616B2E600029C7D058
:10EA500023004433994202D0280000F0D7F9002067
:10EA60006063BEE701232800B847431CC6D12B686A
:10EA7000002BC3D01D2B01D0162B01D12E60AFE788
:10EA80004023A2891343A381ABE740230B4301201A
:10EA9000A3814042A5E70F69002FA1D00B680F604A
:10EAA000DB1B01930023920700D14B69A360019BFC
:10EAB000002B00DC94E7019B3A00216A2800A66A3B
:10EAC000B047002803DC4023A2891343DFE7019B02
:10EAD0003F181B1A0193EAE7010040200B6970B54B
:10EAE00005000C00002B01D1002070BD002804D0CF
:10EAF0008369002B01D100F05FF80B4B9C4209D1D8
:10EB00006C680C22A35E002BEED021002800FFF7DA
:10EB10005BFFEAE7054B9C4201D1AC68F1E7044B8F
:10EB20009C42EED1EC68ECE7541201007412010033
:10EB300034120100002310B50400036043608360B9
:10EB400081814366C28103614361836119000822A8
:10EB50005C30FFF7FFF9054B24626362044BA3624C
:10EB6000044BE362044B236310BDC04621F3000055
:10EB700049F3000081F30000ADF3000010B5024935
:10EB800000F08CF810BDC046DDEA000070B56825C5
:10EB90004A1E55430E002900743100F081F9041E0D
:10EBA00008D000212A00016046600C30A060683265
:10EBB000FFF7D0F9200070BD836913B50400002B66
:10EBC00028D18364C3640365134B144A1B688262B3
:10EBD0000193984201D101238361200000F020F8C5
:10EBE0006060200000F01CF8A060200000F018F821
:10EBF0000022E06004216068FFF79CFF01220921E8
:10EC0000A068FFF797FF02221221E068FFF792FF4A
:10EC10000123A36113BDC046FC1101007DEB000080
:10EC2000F8B51C4B07001E68B369002B02D13000F9
:10EC3000FFF7C2FF4836B4687368013B04D53368F8
:10EC4000002B07D03668F6E70C22A55E002D0DD00C
:10EC50006834F2E704213800FFF798FF306000289D
:10EC6000F0D10C2304003B602000F8BD20000A4BCB
:10EC7000656625606560A560E36025616561A561E5
:10EC8000082229005C30FFF765F96563A563A56478
:10EC9000E564E9E7FC1101000100FFFFF7B504009E
:10ECA0000700002601914834002C01D13000FEBD40
:10ECB0006368A5680093009B013B009301D524681D
:10ECC000F2E7AB89012B08D90E22AB5E013304D0E9
:10ECD00029003800019B984706436835EBE7EC3084
:10ECE0000068704770B50E001D000E23C95E96B017
:10ECF0001400002907DA00232B60B3891B0611D406
:10ED00008023DB000FE06A4600F088FB0028F2DB7E
:10ED1000F022019B12021340054A9B185A425341AC
:10ED20002B60EDE740230020236016B070BDC04685
:10ED300000E0FFFFF7B502268B8905000C00334287
:10ED400006D0230047332360236101236361F7BDAD
:10ED500001AB6A46FFF7C6FF00990700280000F0E4
:10ED60009FF8002808D10C22A35E9A05EFD4032255
:10ED700093431E43A681E4E70F4BAB628023A28935
:10ED800020601343A381009B20616361019B002BE2
:10ED90000DD00E23E15E280000F052FB002806D0C3
:10EDA0000322A38993431A0001231343A381A0895B
:10EDB0003843A081CBE7C0467DEB000010B5034B84
:10EDC0000100186800F06CF810BDC04690000020EB
:10EDD00082B0002900D101A9101E06D0002B06D058
:10EDE00013780B601078431E984102B070470220E0
:10EDF0004042FAE7C9B28218904201D10020704720
:10EE000003788B42FBD00130F6E7000070B50500B7
:10EE1000002910D00C1F2368002B00DAE41828000A
:10EE200000F034FB1D4A1368002B05D163601460A9
:10EE3000280000F02CFB70BDA34209D9216860189E
:10EE40008342F3D118685B6841182160EEE7130034
:10EE50005A68002A01D0A242F9D919685818A0426C
:10EE60000BD120680918581819608242E0D1106847
:10EE70005268411819605A60DAE7A04202D90C239F
:10EE80002B60D5E721686018824203D11068526870
:10EE90004118216062605C60CAE7C046F81B002030
:10EEA000032370B5CD1C9D43083506000C2D1ED2E2
:10EEB0000C25A9421DD8300000F0E8FA254A146854
:10EEC0002100002919D1244C2368002B03D13000E4
:10EED00000F0CAF920602900300000F0C5F9431C99
:10EEE0002BD10C233000336000F0D1FA03E0002D69
:10EEF000DFDA0C233360002070BD0B685B1B19D474
:10EF00000B2B03D90B60CC18256003E04B688C42B7
:10EF10000DD11360300000F0BAFA200007220B3048
:10EF2000231D9043C31AE7D05A42E250E4E76360DE
:10EF30000C00EFE70C004968C3E70323C41C9C43A3
:10EF4000A042E1D0211A300000F08EF9431CDBD141
:10EF5000C7E7C046F81B0020FC1B0020F8B50700DF
:10EF60000D001600002905D11100FFF799FF0400DC
:10EF70002000F8BD002A03D1FFF748FF3400F7E76F
:10EF800000F086FA2C00B042F2D231003800FFF7D0
:10EF900087FF041EECD029003200FEF7BFFF2900D6
:10EFA0003800FFF733FFE3E7F0B58E6885B0070060
:10EFB0000C00039201939E423CD890238A89DB0087
:10EFC0001A4234D00325096923685B1A02936369E6
:10EFD00002985D43EB0F5D19019B6D1001331B1807
:10EFE000AB4200D91D00530532D529003800FFF788
:10EFF00057FF061E09D10C233B6040230120A28944
:10F0000040421343A38105B0F0BD029A2169FEF787
:10F0100085FFA389144A1A4080231343A381029BCE
:10F020002661F61826606561019EED1AA560019BB8
:10F030009E4200D9019E320003992068FEF777FFB7
:10F04000A36800209B1BA36023689E192660DAE753
:10F050002A003800FFF782FF061EE0D12169380040
:10F06000FFF7D4FEC7E7C0467FFBFFFFF0B59FB0B8
:10F07000029005938B890F0016001B0611D50B69B2
:10F08000002B0ED14021FFF70BFF386038610028BC
:10F0900005D10C23029A013813601FB0F0BD402344
:10F0A0007B61002306AC6361203363761033A37663
:10F0B00035002B78002B01D0252B46D1AB1B0493B8
:10F0C0000CD0320039000298FFF76EFF431C00D1CC
:10F0D000AEE06269049B9446634463612B78002B25
:10F0E00000D1A5E0012200235242626002A95432FD
:10F0F00052186E1C2360E360A3601370A36531781F
:10F1000005225448FFF776FE751C00281FD122689F
:10F11000D30604D5532302A95B18202119701307C5
:10F1200004D5532302A95B182B21197033782A2B9D
:10F1300016D0350000210A20E3682A786E1C303A88
:10F14000092A4ED9002918D010E00135B1E7414B0A
:10F150002268C01A01238340134323602E00CEE7A8
:10F16000059B191D1B680591002B01DB099304E029
:10F170005B42E3600223134323602B782E2B0AD1DA
:10F180006B782A2B35D1059B02351A1D1B68059219
:10F19000002B2BDB0793304E297803223000FFF73A
:10F1A00029FE002806D04023801B834022680135B9
:10F1B000134323602978062228486E1C2176FFF726
:10F1C00019FE00283CD0264B002B25D10722059B99
:10F1D00007339343083305936369039A9B1863616C
:10F1E00066E7434301219B183500A6E701235B42F4
:10F1F000D0E700230A201A000135636029786E1CCD
:10F200003039092903D9002BC5D00792C3E74243FF
:10F21000012352183500F1E705AB00933A00114B7A
:10F220002100029800E000BF0390039B0133D3D17B
:10F23000BB890B985B0600D42FE7012040422CE7E6
:10F2400005AB00933A00074B21000298FFF736F810
:10F25000EAE7C04600120100061201000A1201008E
:10F2600000000000A9EF0000002370B5064C050067
:10F270000800236000F060F9431C03D12368002BD1
:10F2800000D02B6070BDC046B02F002070B50400C8
:10F290000D001F2904D9162303600120404270BDD0
:10F2A000436C002B04D08A009B181A68002A08D1EE
:10F2B000200000F031F82A000100200000F01AF8C8
:10F2C000EDE70020012AEAD0511C03D116230130BA
:10F2D0002360E4E7002428001C6090472000DEE75C
:10F2E00010B5034B01001868FFF7D0FF10BDC046F2
:10F2F00090000020002370B5064C050008001100A6
:10F30000236000F001F9431C03D12368002B00D0D7
:10F310002B6070BDB02F002010B500F0E5F810BDD7
:10F3200070B50C000E25495F00F0BAF8002803DB29
:10F33000636D1B18636570BDA389024A1340A381E6
:10F34000F9E7C046FFEFFFFFF8B51F008B89050006
:10F350000C001600DB0505D50E23C95E0022022332
:10F3600000F080F8A389054A28001340A3813200E9
:10F370000E23E15E3B0000F02BF8F8BDFFEFFFFF2E
:10F3800070B50C000E25495F00F06CF8A389421C93
:10F3900003D1054A1340A38170BD8022520113435B
:10F3A000A3816065F8E7C046FFEFFFFF10B50E23AD
:10F3B000C95E00F021F810BD0B1E04D0FF2A04D94D
:10F3C0008A2303608B3B180070470A700123FAE719
:10F3D00070B50500080011000022064C22601A00DA
:10F3E00000F0B8F8431C03D12368002B00D02B6039
:10F3F00070BDC046B02F0020002370B5064C05003C
:10F400000800236000F060F8431C03D12368002B40
:10F4100000D02B6070BDC046B02F0020002370B517
:10F42000064C050008001100236000F055F8431C4D
:10F4300003D12368002B00D02B6070BDB02F0020BB
:10F44000002370B5064C05000800236000F054F856
:10F45000431C03D12368002B00D02B6070BDC04635
:10F46000B02F002070B50500080011000022064CE6
:10F4700022601A0000F050F8431C03D12368002BCF
:10F4800000D02B6070BDC046B02F00207047704781
:10F490000B1F1B68181F002B01DA0B58C018704790
:10F4A00070B50500080011000022064C22601A0009
:10F4B00000F03AF8431C03D12368002B00D02B60E6
:10F4C00070BDC046B02F002058220120014B4042A1
:10F4D0001A607047B02F002058220120014B404293
:10F4E0001A607047B02F002058220120014B404283
:10F4F0001A607047B02F00205822024B00201A607B
:10F500007047C046B02F002058220120014B4042D6
:10F510001A607047B02F002058220120014B404252
:10F520001A607047B02F002058220120014B404242
:10F530001A607047B02F0020044A1368002B00D1D6
:10F54000034B1818106018007047C046001C0020BC
:10F55000B82F002058220120014B40421A6070470A
:10F56000B02F0020FEE7C046F8B5C046F8BC08BC86
:10F570009E467047F8B5C046F8BC08BC9E4670472A
:10F5800064617461000000001EF60000EF010000DD
:10F5900027F60000E50A00002DF60000E302000057
:10F5A00035F60000990B00003CF60000D50C000079
:10F5B00041F600000905000047F60000F5060000CE
:10F5C00052F600005303000057F600002D0F000014
:10F5D00063F600001F0200006DF60000110A000033
:10F5E0007BF600009506000088F600008108000008
:10F5F00094F600005506000072616E646F6D006144
:10F600006C6C006C61737400300066616C73650033
:10F610007472756500252E3135732E2E2E006D61A6
:10F620006B654C6973740072616E67650061646438
:10F630004C6173740064656C657465006A6F696E13
:10F640000073706C697400636F707946726F6D54EB
:10F650006F0066696E64006A6F696E537472696EDA
:10F66000677300756E69636F6465417400756E69D8
:10F67000636F6465537472696E67006E6577427973
:10F680007465417272617900617342797465417287
:10F6900072617900667265654D656D6F7279000003
:10F6A0000DF700002114000012F700003F140000C5
:10F6B00035F600004314000018F700002514000080
:10F6C00022F70000471400002BF700004B14000045
:10F6D00035F700004F1400003EF7000053140000FF
:10F6E00049F700005714000055F7000029140000E6
:10F6F0005EF700003714000068F700002D140000CA
:10F7000073F700003B14000066696C65006F70655C
:10F710006E00636C6F736500656E644F6646696C5E
:10F720006500726561644C696E6500726561644272
:10F73000797465730072656164496E746F006170FD
:10F7400070656E644C696E6500617070656E6442D0
:10F75000797465730066696C6553697A65007374C2
:10F760006172744C697374006E657874496E4C698B
:10F7700073740073797374656D496E666F00000071
:10F78000C4F7000077140000CEF7000083140000D7
:10F79000D9F7000087140000E6F700008B14000082
:10F7A000F2F700008F140000FBF700009314000034
:10F7B00003F800007B1400000EF800007F14000026
:10F7C000686964006D6F7573654D6F7665006D6F68
:10F7D0007573655072657373006D6F7573655265EF
:10F7E0006C65617365006D6F7573655363726F6CE3
:10F7F0006C0070726573734B657900686F6C644B55
:10F8000065790072656C656173654B657900726539
:10F810006C656173654B657973000000D418000056
:10F82000E4180000081900006C190000AA19000073
:10F83000E6190000261A0000561A0000A41A00005B
:10F84000F01A00004A1B0000AC1B0000181C00004E
:10F85000561C0000861C0000C81C00001C1D000077
:10F860004C1D0000841D0000BC1D0000F837000086
:10F87000921E00007E1F000008200000642000008F
:10F88000BC200000E82000001621000094220000A7
:10F89000E4220000662300009E230000DA2300001B
:10F8A0001624000088240000FA24000060250000CF
:10F8B000C825000056260000D22600003827000088
:10F8C0009C270000DC2700002C2800007C2800007A
:10F8D000CC2800002A29000088290000D82900002F
:10F8E0006C2A0000AC2A0000FC2A00004C2B00000F
:10F8F0009C2B0000E02B0000302C0000802C00002E
:10F90000282E0000841D0000C81C0000F22C0000FE
:10F91000D4180000322D0000682D0000A82D000032
:10F92000E82D0000D4180000D4180000D4180000FE
:10F93000D4180000AC2E0000F82E00004A2F000062
:10F94000A42F0000DA2F00005E300000B830000065
:10F95000F0300000D4180000D41800001E31000060
:10F9600058310000C8310000083200003C3200006D
:10F970007C320000B0320000E2320000143300009C
:10F980004E33000088330000BC330000F033000029
:10F990002A3400005E340000D4180000D41800009F
:10F9A000D4180000D4180000D418000098340000C7
:10F9B000CE340000043500003A35000070350000F8
:10F9C000B8350000F8350000383600007836000001
:10F9D000AE360000E436000024370000D4180000E2
:10F9E000D4180000D4180000D4180000D418000067
:10F9F000D4180000D4180000D4180000D418000057
:10FA0000D4180000D4180000D41800005A370000A1
:10FA10005A370000AA380000E03800005B25642057
:10FA20006974656D206C6973745D002825642062BB
:10FA3000797465732900286F626A6563742074792C
:10FA400070653A2025642900537461636B20756EDC
:10FA5000646572666C6F7700626F6F6C65616E00D3
:10FA60006E756D62657200737472696E67006C69A1
:10FA700073740062797465206172726179000000AC
:10FA8000070000000300000019FB00000D3A000011
:10FA900021FB0000BD3A00002AFB00004D3F0000A2
:10FAA00033FB0000113A00003CFB0000513F000016
:10FAB00044FB0000793C00004DFB0000353D000098
:10FAC0005BFB0000A93B000066FB00000141000059
:10FAD00071FB00008D3C00007CFB000059400000E1
:10FAE00088FB0000553B000094FB0000D140000063
:10FAF0001C000000010000000200000004000000E3
:10FB000005000000060000001000000011000000C9
:10FB100043616C6C696F706500686173546F6E65EA
:10FB200000706C6179546F6E650068617353657223
:10FB3000766F00736574536572766F006461634914
:10FB40006E697400646163577269746500736F66EF
:10FB50007457726974654279746500737175617266
:10FB6000655761766500736574557365724C4544DD
:10FB700000616E616C6F675265616400616E616CFB
:10FB80006F675772697465006469676974616C5264
:10FB9000656164006469676974616C577269746552
:10FBA00000474320746F6F6B202564207573656375
:10FBB000733B206672656520256420776F726473DD
:10FBC000003C496E74656765723E003C4C69737415
:10FBD0003E003C4F626A6563743E003C4279746546
:10FBE00041727261793E000D0A564D2050616E6976
:10FBF000633A2025730D0A006D69736300000000ED
:10FC00005DFC0000714B000066FC0000694C0000C8
:10FC10006EFC00002D4C000072FC0000014C000046
:10FC200077FC0000C14C00008AFC0000614B000022
:10FC300099FC0000F5170000A8FC0000B54A000080
:10FC4000B0FC00005B4A0000BAFC0000F149000073
:10FC5000C6FC0000F34800006E756C6C00686578A7
:10FC6000546F496E740072657363616C65007369EB
:10FC70006E0073717274007072657373757265547F
:10FC80006F416C74697475646500636F6E6E656353
:10FC9000746564546F4944450062726F61646361C6
:10FCA0007374546F494445006A736F6E47657400FE
:10FCB0006A736F6E436F756E74006A736F6E566110
:10FCC0006C75654174006A736F6E4B6579417400A1
:10FCD000CCFD00004D4D0000D4FD0000514D000052
:10FCE000DEFD00006F4D0000E7FD0000794D0000D3
:10FCF000F2FD0000834D0000FEFD00008D4D000070
:10FD00000CFE0000974D000014FE0000A14D000005
:10FD10001AFE0000AB4D00002FFE0000B54D0000A4
:10FD200044FE0000BF4D000050FE0000C94D000021
:10FD300060FE0000D34D00006CFE0000DD4D0000B1
:10FD400079FE0000E74D000082FE0000F14D00004A
:10FD50008AFE0000FB4D000098FE0000054E0000EA
:10FD6000A9FE00000F4E0000BCFE0000194E00006E
:10FD7000CAFE0000234E0000D9FE00002D4E0000F8
:10FD8000ECFE0000374E000002FF00004B4E00006A
:10FD90000EFF0000554E00001EFF00005F4E0000E9
:10FDA0002DFF0000694E00003BFF0000734E000075
:10FDB00043FF0000414E00004FFF00005B4D00007C
:10FDC00057FF0000654D00006E6574006861735751
:10FDD0006946690073746172745769466900737487
:10FDE0006F70576946690077696669537461747505
:10FDF00073006D7949504164647265737300737464
:10FE0000617274535349447363616E006765745340
:10FE1000534944006D794D414300687474705365D3
:10FE20007276657247657452657175657374007298
:10FE30006573706F6E64546F487474705265717539
:10FE40006573740068747470436F6E6E65637400DC
:10FE5000687474704973436F6E6E65637465640093
:10FE60006874747052657175657374006874747029
:10FE7000526573706F6E7365007564705374617250
:10FE8000740075647053746F700075647053656EA0
:10FE9000645061636B657400756470526563656975
:10FEA00076655061636B65740075647052656D6F43
:10FEB000746549504164647265737300756470526F
:10FEC000656D6F7465506F727400776562536F6310
:10FED0006B6574537461727400776562536F636B02
:10FEE00065744C6173744576656E74007765625312
:10FEF0006F636B657453656E64546F436C69656EB4
:10FF000074004D515454436F6E6E656374004D51CF
:10FF100054544973436F6E6E6563746564004D514C
:10FF20005454446973636F6E6E656374004D51542D
:10FF3000544C6173744576656E74004D5154545041
:10FF40007562004D51545453657457696C6C004D83
:10FF5000515454537562004D515454556E7375622B
:10FF600000000000B2FF0000954E0000B7FF000047
:10FF7000A94E0000C1FF0000AD4E0000CAFF000006
:10FF8000B14E0000D1FF0000B54E0000DBFF0000C5
:10FF9000A14E0000E5FF0000994E0000EEFF0000BA
:10FFA0009D4E0000F3FF0000A54E000031776972FE
:10FFB0006500696E6974007363616E537461727475
:10FFC000007363616E4E6578740073656C6563746D
:10FFD0000073656C656374416C6C0077726974655D
:10FFE0004279746500726561644279746500637278
:10FFF0006338006372633136000D0E0F04050C0B7D
:020000021000EC
:100000000A06070809000000000008080800080A9E
:100010004A4000000A5FEA5FEA0ED92ED36E193219
:100020004489330C924C924D080800000004880863
:1000300008040804848488000A448A4000048EC4AA
:1000400080000000048800000EC0000000000800CE
:1000500001224488100C9252524C048C84848E1CD1
:10006000824C901E1EC244924C06CA525FE21FF0A0
:100070001EC13E02448ED12E1FE24488100ED12EA6
:10008000D12E0ED12EC48800080008000004800480
:10009000880244880482000EC00EC008048244888E
:1000A0000ED126C0040ED135B36C0C925ED2521C18
:1000B000925C925C0ED010100E1C9252525C1ED0BC
:1000C0001C901E1ED01C90100ED013712E12525E6A
:1000D000D2521C8808081C1FE242524C1254981439
:1000E00092101010101E113B75B131113935B371DA
:1000F0000C9252524C1C925C90100C92524C861CEA
:10010000925C92510ED00C825C1FE4848484125263
:1001100052524C1131312A44113135BB7112524CBB
:100120009252112A4484841EC488101E0EC80808E6
:100130000E10080482410EC242424E048A40000062
:10014000000000001F0804800000000ED2524F1073
:10015000101C925C000ED0100E02424ED24E0C9239
:100160005C900E06C81C88080ED24EC24C10101CA3
:1001700092520800080808024002424C10149814D9
:10018000920808080806001B75B131001C925252F3
:10019000000C92524C001C925C90000ED24EC20099
:1001A0000ED010100006C8049808080EC8070012E8
:1001B00052524F0011312A4400113135BB00124C0C
:1001C0008C9200112A4498001EC4881E06C48C8498
:1001D00086080808080818080C881800000C8360B6
:1001E0000000000001000000020000000300000009
:1001F00004000000050000000600000007000000E9
:1002000008000000090000000A0000000B000000C8
:100210000C0000000D0000000E0000000F000000A8
:100220001000000012000000140000001600000082
:10023000180000001A0000001C0000001E00000052
:10024000200000002300000026000000290000001C
:100250002C0000002F0000003200000036000000DB
:100260003A0000003E00000042000000460000008E
:100270004B00000050000000550000005A00000034
:1002800061000000680000006F00000076000000C0
:100290007D000000840000008B0000009200000040
:1002A00099000000A0000000A7000000AE000000C0
:1002B000B5000000BC000000C3000000CA00000040
:1002C000D1000000D8000000DF000000E6000000C0
:1002D000ED000000F4000000FB000000FF00000043
:1002E00040030100D14E00004B030100B15000005B
:1002F00056030100C554000060030100D150000006
:100300006D030100355200007403010085520000A6
:100310007D030100D552000089030100CD5100008A
:100320009A0301005D510000AA030100C5530000BB
:10033000B703010029510000646973706C61790092
:100340006C696768744C6576656C006D62536574A2
:10035000436F6C6F72006D62446973706C617900F9
:100360006D62446973706C61794F6666006D6250AE
:100370006C6F74006D62556E706C6F74006D6244CA
:100380007261775368617065006D62536861706572
:10039000466F724C6574746572006D62456E616281
:1003A0006C65446973706C6179006E656F50697833
:1003B000656C53656E64006E656F506978656C534B
:1003C000657450696E004E6F7420656E6F75676856
:1003D00020726F6F6D206576656E20616674657240
:1003E00020636F6D70616374696F6E00436F6D7031
:1003F000616374656420466C61736820636F646533
:100400002073746F72650A256420627974657320A5
:100410007573656420282564252529206F662025AD
:100420006400426164207265636F726420666F7558
:100430006E6420647572696E6720696E69746961A3
:100440006C697A6174696F6E0025642025642025CB
:10045000642028256420776F726473290025642046
:100460007265636F7264732C20256420776F7264E9
:10047000732C206D617849442025642C20636F6DB6
:1004800070616374696F6E206379636C6573202596
:100490006400526573746F72656420256420736311
:1004A0007269707473005374617274656400726170
:1004B00064696F0049050100E95E0000560501000E
:1004C000E56100006605010065610000740501003A
:1004D000796300007F050100015F00008F050100C6
:1004E0007D5F0000A3050100655F0000B20501000B
:1004F00029650000BE050100A7640000C7050100D2
:100500004B640000D2050100C5630000DD05010059
:1005100001640000E605010035640000EF050100FC
:10052000115F0000FE050100455F000007060100A5
:10053000215F000025303878006E6F6E65006F74A3
:1005400068657200706169720064697361626C65EC
:10055000526164696F006D657373616765526563AD
:100560006569766564007061636B65745265636587
:10057000697665007061636B657453656E640072C3
:1005800065636569766564496E7465676572007256
:10059000656365697665644D6573736167655479F4
:1005A0007065007265636569766564537472696E1F
:1005B000670073656E64496E746567657200736584
:1005C0006E64506169720073656E64537472696E13
:1005D00067007365744368616E6E656C0073657463
:1005E00047726F757000736574506F776572007332
:1005F00069676E616C537472656E677468006465D8
:10060000766963654944006C6173744D6573736109
:100610006765494400556E6B6E6F776E2070726926
:100620006D6974697665205B25733A25735D0000FA
:1006300000000000963007772C610EEEBA51099940
:1006400019C46D078FF46A7035A563E9A395649E9C
:100650003288DB0EA4B8DC791EE9D5E088D9D297C0
:100660002B4CB609BD7CB17E072DB8E7911DBF901C
:100670006410B71DF220B06A4871B9F3DE41BE8440
:100680007DD4DA1AEBE4DD6D51B5D4F4C785D3839C
:1006900056986C13C0A86B647AF962FDECC9658A40
:1006A0004F5C0114D96C0663633D0FFAF50D088D9C
:1006B000C8206E3B5E10694CE44160D5727167A240
:1006C000D1E4033C47D4044BFD850DD26BB50AA59C
:1006D000FAA8B5356C98B242D6C9BBDB40F9BCACC0
:1006E000E36CD832755CDF45CF0DD6DC593DD1AB1C
:1006F000AC30D9263A00DE518051D7C81661D0BF40
:10070000B5F4B42123C4B3569995BACF0FA5BDB89B
:100710009EB802280888055FB2D90CC624E90BB13F
:10072000877C6F2F114C6858AB1D61C13D2D66B69B
:100730009041DC760671DB01BC20D2982A10D5EFFF
:100740008985B1711FB5B606A5E4BF9F33D4B8E85B
:10075000A2C9077834F9000F8EA8099618980EE1FF
:10076000BB0D6A7F2D3D6D08976C6491015C63E65B
:10077000F4516B6B62616C1CD83065854E0062F27F
:10078000ED95066C7BA5011BC1F4088257C40FF5DB
:10079000C6D9B06550E9B712EAB8BE8B7C88B9FCFF
:1007A000DF1DDD62492DDA15F37CD38C654CD4FB5B
:1007B0005861B24DCE51B53A7400BCA3E230BBD4FF
:1007C00041A5DF4AD795D83D6DC4D1A4FBF4D6D35B
:1007D0006AE96943FCD96E34468867ADD0B860DAFF
:1007E000732D0444E51D03335F4C0AAAC97C0DDD5B
:1007F0003C710550AA41022710100BBE86200CC97F
:1008000025B56857B3856F2009D466B99FE461CEDA
:100810000EF9DE5E98C9D9292298D0B0B4A8D7C7FE
:10082000173DB359810DB42E3B5CBDB7AD6CBAC05A
:100830002083B8EDB6B3BF9A0CE2B6039AD2B17476
:100840003947D5EAAF77D29D1526DB048316DC73D2
:10085000120B63E3843B64943E6A6D0DA85A6A7A76
:100860000BCF0EE49DFF099327AE000AB19E077DD2
:1008700044930FF0D2A3088768F2011EFEC20669F6
:100880005D5762F7CB67658071366C19E7066B6E52
:10089000761BD4FEE02BD3895A7ADA10CC4ADD6776
:1008A0006FDFB9F9F9EFBE8E43BEB717D58EB060D2
:1008B000E8A3D6D67E93D1A1C4C2D83852F2DF4F76
:1008C000F167BBD16757BCA6DD06B53F4B36B248D2
:1008D000DA2B0DD84C1B0AAFF64A0336607A044176
:1008E000C3EF60DF55DF67A8EF8E6E3179BE6946D2
:1008F0008CB361CB1A8366BCA0D26F2536E26852F6
:1009000095770CCC03470BBBB91602222F26055551
:10091000BE3BBAC5280BBDB2925AB42B046AB35C75
:10092000A7FFD7C231CFD0B58B9ED92C1DAEDE5BD1
:10093000B0C2649B26F263EC9CA36A750A936D02B5
:10094000A906099C3F360EEB856707721357000511
:10095000824ABF95147AB8E2AE2BB17B381BB60C35
:100960009B8ED2920DBED5E5B7EFDC7C21DFDB0B91
:10097000D4D2D38642E2D4F1F8B3DD686E83DA1FB5
:10098000CD16BE815B26B9F6E177B06F7747B71811
:10099000E65A0888706A0FFFCA3B06665C0B0111B5
:1009A000FF9E658F69AE62F8D3FF6B6145CF6C1611
:1009B00078E20AA0EED20DD75483044EC2B30339B5
:1009C000612667A7F71660D04D476949DB776E3E11
:1009D0004A6AD1AEDC5AD6D9660BDF40F03BD83735
:1009E00053AEBCA9C59EBBDE7FCFB247E9FFB53091
:1009F0001CF2BDBD8AC2BACA3093B353A6A3B424B5
:100A00000536D0BA9306D7CD2957DE54BF67D92310
:100A10002E7A66B3B84A61C4021B685D942B6F2AB4
:100A200037BE0BB4A18E0CC31BDF055A8DEF022D10
:100A3000416C6C207461736B732073746F7070659C
:100A400064007631393100202573202573004D650F
:100A50006D6F727920636C6561726564004E6F2002
:100A600066726565207461736B20656E747269656A
:100A700073000000F40A010055800000010B010022
:100A8000B97D00000D0B0100897D0000130B0100F2
:100A9000997D0000190B0100A97D00001F0B0100CA
:100AA000017B0000350B0100317F0000430B01008A
:100AB000597700004D0B0100BD7F0000550B010070
:100AC000417B00005E0B0100817800006F0B01008C
:100AD000657900007B0B010035780000840B010074
:100AE000B97800008C0B0100517A000073656E73B9
:100AF0006F727300616363656C65726174696F6EB8
:100B00000074656D70657261747572650074696CEE
:100B100074580074696C74590074696C745A007369
:100B20006574416363656C65726F6D65746572525F
:100B3000616E6765006D61676E65746963466965BE
:100B40006C6400746F756368526561640069326338
:100B50005265616400693263577269746500693275
:100B600063536574436C6F636B53706565640073A6
:100B7000706945786368616E676500737069536575
:100B80007475700072656164444854006D696372E5
:100B90006F70686F6E6500000DF7000061810000E6
:100BA00012F700000D810000CF0B0100A5820000AC
:100BB00035F7000029810000D40B01002D820000D0
:100BC000DA0B01008581000073657269616C007247
:100BD0006561640077726974650077726974654253
:100BE00079746573000000007C0C0100D582000060
:100BF000890C0100D9820000920C0100E5820000FE
:100C00009C0C0100E9820000A50C0100ED820000AF
:100C1000AA0C0100F1820000AF0C0100F582000077
:100C2000BB0C0100F9820000C20C0100FD82000033
:100C3000CB0C010001830000D00C010005830000F3
:100C4000DD0C010009830000EB0C01000D830000A6
:100C5000F70C010011830000020D01001583000054
:100C60000D0D010019830000170D0100DD82000049
:100C7000210D0100E1820000746674007365744206
:100C800061636B6C69676874006765745769647445
:100C900068006765744865696768740073657450B7
:100CA0006978656C006C696E6500726563740072CA
:100CB0006F756E6465645265637400636972636C1A
:100CC0006500747269616E676C65007465787400A4
:100CD00064656665725570646174657300726573EE
:100CE000756D6555706461746573006D65726765D7
:100CF0004269746D61700064726177427566666501
:100D00007200746674546F75636865640074667409
:100D1000546F7563685800746674546F75636859CE
:100D200000746674546F756368507265737375727E
:100D30006500766172730000580D0100A9870000FC
:100D4000620D0100898700006B0D010065870000BE
:100D5000770D0100F386000076617245786973743F
:100D600073007661724E616D6564007365745661DF
:100D7000724E616D6564007661724E616D65466F9D
:100D800072496E6465780057656C636F6D65207499
:100D90006F204D6963726F426C6F636B73210070DB
:100DA0005F73706920213D204E554C4C002F686FB9
:100DB0006D652F6769742F2E706C6174666F726D2C
:100DC000696F2F7061636B616765732F6672616D08
:100DD00065776F726B2D61726475696E6F6E6F727D
:100DE0006469636E7266352F6C69627261726965DF
:100DF000732F5350492F5350492E63707000535036
:100E000049436C6173733A3A535049436C6173734D
:100E1000284E52465F5350495F547970652A2C2002
:100E200075696E74385F742C2075696E74385F74E0
:100E30002C2075696E74385F742900000000000072
:100E4000000000007D890000398900005F890000F2
:100E500069890000738900005D89000000000000BE
:100E60000100000002000000160000000400000065
:100E70000500000006000000070000000800000058
:100E8000090000000A0000000B0000000C00000038
:100E90000D0000000E0000000F0000001A0000000E
:100EA0001B000000140000001300000011000000EF
:100EB00017000000100000001C0000001D000000D2
:100EC0001E000000120000001500000003000000DA
:100ED00018000000190000000000000000000000E1
:100EE000698D00009D950000E98D0000FD8D0000DA
:100EF000F38D0000658D0000598D0000098E000003
:100F0000858D0000558D000000000000000030437A
:100F100000000000000030C3706F770073717274BE
:100F200000000000FB21F93FFB2109407CD9124061
:100F3000FB2119407A6A1F407CD92240BBFD254025
:100F4000FB2129403A462C407A6A2F405C473140C9
:100F50007CD932409C6B3440BBFD3540DB8F374041
:100F6000FB2139401BB43A403A463C405AD83D40F8
:100F70007A6A3F404C7E40405C4741406C104240A2
:100F80007CD942408CA243409C6B4440AC344540E9
:100F9000BBFD4540CBC64640DB8F4740EB58484041
:100FA000FB21494083F9A200444E6E00FC29150044
:100FB000D1572700DD34F50062DBC0003C99950075
:100FC000419043006351FE00BBDEAB00B761C5003A
:100FD0003A6E2400D24D42004906E00009EA2E0094
:100FE0001C92D100EB1DFE0029B11C00E83EA700B9
:100FF000F535820044BB2E009CE98400B4267000C5
:10100000417E5F00D6913900538339009CF439004A
:101010008B5F840028F9BD00F81F3B00DEFF9700BE
:101020000F980500112FEF000A5A8B006D1F6D00FD
:10103000CF7E360009CB2700464FB7009E663F00A3
:101040002DEA5F00BA277500E5EBC7003D7BF10094
:10105000F739070092528A00FB6BEA001FB15F006C
:10106000085D8D00300356007BFC4600F0AB6B0042
:1010700020BCCF0036F49A00E3A91D005E61910008
:10108000081BE60085996500A0145F008D4068008C
:1010900080D8FF0027734D0006063100CA561500A0
:1010A000C9A873007BE260006B8CC00000000000E8
:1010B00000000040FB21F93F000000002D44743E79
:1010C000000000809846F83C0000006051CC783B5E
:1010D00000000080831BF0390000004020257A3892
:1010E000000000802282E336000000001DF3693515
:1010F00002000000030000000400000006000000E1
:1011000088C0000032C0000032C0000060C1000092
:101110002EC000002EC0000056C1000060C10000BB
:101120002EC0000056C100002EC0000060C10000AB
:1011300064C1000064C1000064C100006CC1000013
:1011400064CB0000D6C900001ACA00007EC90000A6
:101150001ACA00000ACB00001ACA00007EC90000AB
:10116000D6C90000D6C900000ACB00007EC9000025
:1011700076C9000076C9000076C9000018CB0000CF
:101180008CD200008ED100008ED10000ACD40000C3
:1011900088D1000088D1000094D40000ACD40000B5
:1011A00088D1000094D4000088D10000ACD40000A5
:1011B000A2D40000A2D40000A2D40000B0D4000049
:1011C0002C2066756E6374696F6E3A2000617373CC
:1011D000657274696F6E2022257322206661696CC6
:1011E00065643A2066696C6520222573222C206C88
:1011F000696E65202564257325730A00940000201C
:10120000232D302B2000686C4C00656667454647EF
:101210000030313233343536373839414243444572
:1012200046003031323334353637383961626364E1
:1012300065660000000000000000000000000000E3
:10124000000000000000000000000000000000009E
:10125000000000000000000000000000000000008E
:10126000000000000000000000000000000000007E
:10127000000000000000000000000000000000006E
:10128000000000000000000000000000000000005E
:1012900000000000504F534958000020202020201B
:1012A0002020202028282828282020202020202016
:1012B0002020202020202020202020881010101006
:1012C000101010101010101010101004040404045A
:1012D0000404040404101010101010104141414186
:1012E000414101010101010101010101010101016E
:1012F0000101010101011010101010104242424280
:10130000424202020202020202020202020202023D
:101310000202020202021010101020000000000061
:1013200000000000000000000000000000000000BD
:1013300000000000000000000000000000000000AD
:10134000000000000000000000000000000000009D
:10135000000000000000000000000000000000008D
:10136000000000000000000000000000000000007D
:10137000000000000000000000000000000000006D
:10138000000000000000000000000000000000005D
:10139000000000000000000000000000000000004D
:0813A00068EDFE7F0100000072
:1013A800FFFFFFFFE803000001000000E803DC0581
:1013B800DC05DC05DC050000FFFFFFFFFFFFFFFF8A
:1013C8001800000000FF000019FCFFFFFFFFFFFFEF
:1013D8000200000040420F00FF01FF000024F4005B
:1013E8000200000003000000FFFFFFFF00000000F4
:1013F800010000000000020001000000FFFFFFFFE5
:1014080000000000020000000000040002000000CC
:10141800FFFFFFFF000000000300000000000800BD
:10142800030000000A00000008000000010000009E
:101438009400002000000000541201007412010002
:10144800341201000000000000000000000000004D
:101458000000000000000000000000000000000084
:101468000000000000000000000000000000000074
:101478000000000000000000000000000000000064
:101488000000000000000000000000000000000054
:101498000000000043000000000000000000000001
:1014A8000000000000000000000000000000000034
:1014B80000000000430000000000000000000000E1
:1014C8000000000000000000000000000000000014
:1014D80000000000430000000000000000000000C1
:1014E80000000000000000000000000000000000F4
:1014F80000000000430000000000000000000000A1
:1015080000000000000000000000000000000000D3
:101518000000000043000000000000000000000080
:1015280000000000000000000000000000000000B3
:101538000000000043000000000000000000000060
:101548000000000000000000000000000000000093
:101558000000000043000000000000000000000040
:101568000000000000000000000000000000000073
:1015780000000000B9F30000D1ED000000000000F9
:101588009A1201001CF60000F7FB0000F7FB0000B0
:10159800F7FB0000F7FB0000F7FB0000F7FB00007B
:1015A800F7FB0000F7FB0000F7FB0000FFFFFFFF61
:1015B800FFFFFFFFFFFFFFFFFFFF00000100415398
:1015C800434949000000000000000000000000003E
:1015D800000000000000000000000000000041536F
:1015E800434949000000000000000000000000001E
:1015F80000000000000000000000000000000000E3
:10160800E9000000098900005D8C0000B590000029
:04161800C10000000D
:0400000300008CF974
:00000001FF
